:100000000C94BA080C94D9080C94D9080C9469097A
:100010000C949F090C94D9080C94D9080C94D90815
:100020000C94D9080C94D9080C94D9080C94D908CC
:100030000C94D9080C94D9080C94D9080C94C90CC8
:100040000C94D9080C94D9080C94D9080C94D908AC
:100050000C9424650C94D55C0C94D9080C94D908A4
:100060000C94D9080C94AA5D0C94D9080C949E5D4C
:100070000C94D9080C94D9080C94D9080C94D9087C
:100080000C9457700C94D9080C94D9080C94D90886
:100090000C94E85D0C94D9080C94DC5D0C94D908A0
:1000A0000C94D9080C94D9080C94D9080C94D9084C
:1000B0000C94D9080C94D9080C94D9080C94D9083C
:1000C0000C94D9080C94D9080C94D9080C94D9082C
:1000D0000C94D9080C94D9080C94D9080C94D9081C
:1000E0000C94D9080C94DD640C94E7640C94D364EC
:1000F0000C9493640C9418650C9409650C94FD643D
:100100000C94F1640C94D9080C94D9080C94D90877
:100110000C94D9080C94D9080C94D9080C94D908DB
:100120009079AF792E7A1D7B3D7B5D7B657B127B61
:10013000084AD73B3BCE016E84BCBFFDC12F3D6C4E
:1001400074319ABD56833DDA3D00C77F11BED9E4B4
:10015000BB4C3E916BAAAABE000000803F076342E1
:1001600036B79BD8A71A39685618AEBAAB558C1D4E
:100170003CB7CC5763BD6DEDFD753EF6177231BFD0
:10018000000000803F08000000BE922449123EABF0
:10019000AAAA2ABECDCCCC4C3E00000080BEABAAA1
:1001A000AAAA3E00000000BF000000803F0000003F
:1001B0000000084178D3BB4387D1133D190E3CC3DF
:1001C000BD4282AD2B3E68EC8276BED98FE1A93E5E
:1001D0004C80EFFFBE01C4FF7F3F00000000002500
:1001E000730A005854414C5F5452494D3D256400F8
:1001F00025730A0025730A00546573742036202580
:10020000730A005465737420352025730A00546501
:10021000737420342025730A0054657374203320CE
:1002200025730A005465737420322025730A005424
:1002300065737420312025730A006368616E3D2563
:10024000640A0074787077723D25640A0035303096
:100250006B0A003235306B0A003131356B0A0035DC
:10026000366B0A0033386B0A0025730A0073656E1B
:10027000743D252D75206475703D252D75206967A9
:100280006E6F7265643D252D752074746C5F7A65A0
:10029000726F3D252D750A0025372E3366202537D0
:1002A0002E33660025352E326620004572726F723D
:1002B000203020566F6C74004E6F74207375707010
:1002C0006F727465640A004572726F722030205636
:1002D0006F6C74004572726F72203020566F6C74B0
:1002E0000025630074746C3D252D64200074746CCB
:1002F0003D252D6420004E65772074746C3D252DBE
:100300006420002563004D533536313120503D25A2
:100310002D372E326620252D372E32666D0A00428B
:100320004D5030383520256C642050612020252D1B
:10033000372E32666D00256300545F484541545F97
:100340004944583D252D352E32662000545F4445E2
:10035000573D252D352E3266200041483D252D354F
:100360002E32662000545F53485432583D252D35B7
:100370002E3266200052485F53485432583D252D96
:10038000352E32662000545F52483D252D342E31E3
:1003900066200052483D252D342E3166200025630D
:1003A0000025630025630025630043757272656E46
:1003B00074207265706F727420696E7465727661F4
:1003C0006C3D252D75207365630A004E657720729C
:1003D00065706F727420696E74657276616C3D250C
:1003E0002D75207365630A002563007265706F7256
:1003F000745F616C6C3D007265706F72743D0025B6
:100400006300256300256300256300204F534343A9
:10041000414C3D2564200020467573653A20656592
:100420003D253032782068663D25303278206C6674
:100430003D25303278206C623D25303278004D43C6
:10044000553D2530366C780025630074785F6C6507
:100450006E3D252D6C752C6C6F775F766F6C7461BB
:1004600067653D252D6C750A002563004F4B0A001A
:1004700025630025630025630025630025630025AF
:10048000630064656275675F616C6C3D0064656202
:1004900075673D0064656275673D0025730A0064F9
:1004A0006565700A006E6F6E650A00707772733D45
:1004B00000696E74725F7365635F70313D252D371F
:1004C0002E33660A00696E74725F70313D252D6CA3
:1004D000640A00696E74725F7365635F70303D25F6
:1004E0002D372E33660A00696E74725F70303D25B9
:1004F0002D6C640A00765F6D63753D252D352E32B7
:10050000660A00707077723D25730A006465627533
:10051000673D0025730A006175746F0A006C6F6790
:100520005F6D6F64653D007573625F7077723D2526
:10053000730A007265706F72743D007265706F723D
:10054000745F696E74657276616C3D252D750A0065
:1005500072656C61793D25730A0074746C3D252DBC
:10056000640A0052494D455F616464723D252D6403
:100570002E252D640A006E65696768626F725F746C
:1005800061626C655F73697A653D25640A006C6F12
:10059000775F766F6C746167653D252D332E32660B
:1005A0000A00747870773D25640A006368616E3DC7
:1005B00025640A006932633D0069643D0074787403
:1005C0003D25730A0053797374656D2053756D6D05
:1005D0006172790A00745F686561745F69647800AC
:1005E000745F64657700616800705F6D73353631E4
:1005F000310072685F736874327800745F73687476
:10060000327800706100700061643400616433000E
:100610006164320061643100613300613200613134
:1006200000765F696E00726800757074696D6500B0
:1006300070315F6C73740070315F740070310070E2
:10064000305F6C73740070305F7400703000765FE0
:100650006D637500745F6D637500743100740069BB
:10066000640065363400747874002D002B006175C9
:10067000746F006E6F6E6500706F7765725F736187
:1006800076655F6C656472790072656C61795F6C28
:1006900065647900636F6D70617373006163636596
:1006A0006C007072657300705F70777200616573C3
:1006B0000070315F6C6564790070305F6C656472E6
:1006C000006576656E74006C6564006F7700706B12
:1006D000740074785F6C6564790072785F6C65642F
:1006E00072006F706572006E6F6E65002530327833
:1006F00000765F6164343D252D382E36660020007B
:10070000765F6164333D252D382E366600200076F5
:100710005F6164323D252D382E3666002000765FFD
:100720006164313D252D382E3666002000765F6CE1
:10073000696768743D252D382E3666002000765F87
:1007400061323D252D372E3366002000765F613102
:100750003D252D372E3366002000765F696E3D25DE
:100760002D352E326600204E657665722D757365C7
:100770006420737461636B203E2025642062797469
:1007800065730A00757074696D653D252D642D646F
:100790006179732D253032643A253032643A253040
:1007A00032642D686F7572730A0074657374205B10
:1007B0006F66667C317C327C337C347C355D2020F6
:1007C0002020202020202D2074657374206D6F64FC
:1007D00065730A0D00263A205B545820504B542074
:1007E000434F4E54454E545D202020202020202091
:1007F000202D2073656E6420706B742066726F6D9F
:1008000020636D646C696E652F636861740A0D0006
:10081000776474205B6F6E7C6F66667C746573743E
:100820005D20202020202020202020202D207761E6
:10083000746368646F670A0D00757067722020200A
:1008400020202020202020202020202020202020A8
:1008500020202020202D207265626F6F7420766921
:100860006120626F6F746C6F616465720A0D007550
:10087000617274205B33386B7C35366B7C3131357B
:100880006B7C3235306B7C3530306B5D202D2073C6
:100890006574207465726D2F756172742073706554
:1008A00065640A0D00626F6F7420202020202020D4
:1008B0002020202020202020202020202020202038
:1008C000202D207265626F6F740A0D00707772734D
:1008D000205B646565707C6E6F6E655D20202020F6
:1008E00020202020202020202D206D637520736C77
:1008F000656570206D6F64650A0D00726573742004
:10090000656570726F6D202020202020202020201F
:10091000202020202020202D20726573746F7265A6
:1009200020656570726F6D0A0D0070707772205BC4
:100930006F6E7C6F66665D202020202020202020A6
:100940002020202020202D2070726F6772616D6D35
:1009500061626C65207077720A0D00747874205B98
:10096000737472696E675D20202020202020202073
:10097000202020202020202D2053657420726570B7
:100980006F7274207465787420737472696E670A6C
:100990000D0074787077205B31352D305D2020207C
:1009A00020202020202020202020202020202D203A
:1009B0005458205077722E204869676865737420F8
:1009C0003020283364426D290A0D0074746C205B5A
:1009D000302D31355D202020202020202020202097
:1009E000202020202020202D2074696D652D746F1B
:1009F0002D6C69766520666F72207061636B65741B
:100A0000730A0D0073732020202020202020202036
:100A100020202020202020202020202020202020D6
:100A20002D2073797374656D2073756D6D617279A6
:100A30000A0D00727320202020202020202020205A
:100A40002020202020202020202020202020202D99
:100A500020726164696F2073746174730A0D00728F
:100A600069205B696E745D202020202020202020DA
:100A700020202020202020202020202D2072657082
:100A80006F727420696E74657276616C0A0D007203
:100A900065205B2B7C2D5D205B6D61736B7C6175CC
:100AA000746F2C6D61736B5D2020202D206D6F7431
:100AB00065207265706F7274207365742F6D6F643A
:100AC0006966790A0D006F772020202020202020E1
:100AD0002020202020202020202020202020202016
:100AE00020202D206F6E652D776972652073656EED
:100AF000736F72730A0D006C6F67205B6175746FA2
:100B00007C6F6E7C6F66665D202020202020202078
:100B10002020202D206D6F74657320646174612026
:100B20006F6E205553420A0D006E65205B666C7532
:100B300073685D20202020202020202020202020DD
:100B400020202020202D206E65696768626F72204A
:100B50007461626C650A0D0065727220202020208D
:100B60002020202020202020202020202020202085
:100B7000202020202D206572726F722073746174A2
:100B8000730A0D006D637520202020202020202076
:100B90002020202020202020202020202020202055
:100BA0002D206D637520696E666F0A0D00696420E3
:100BB0005B72657365745D2020202020202020203A
:100BC0002020202020202020202D20696420686102
:100BD0006E646C696E670A0D0068756D20202020B8
:100BE0002020202020202020202020202020202005
:100BF00020202020202D2068756D6964697479207B
:100C000073656E736F720A0D0072656C6179205B9B
:100C10006F6E7C6F66667C73746174735D202020D8
:100C200020202020202D2072656C6179206E657453
:100C3000776F726B207265706F7274730A0D006447
:100C400065205B6D61736B5D2020202020202020BB
:100C500020202020202020202020202D20646562BC
:100C600075670A0D006368616E205B31312D323685
:100C70005D20202020202020202020202020202037
:100C8000202D206368616E2031312D3236202832CC
:100C90002E3430352D32343830204D687A290A0D03
:100CA0000063616C69205B5B765F696E7C61317C9F
:100CB00061325D20766F6C747C72657365747C6ED6
:100CC0006F6E655D202D2063616C69627261746571
:100CD0000A0D006164632020202020202020202095
:100CE0002020202020202020202020202020202DF7
:100CF0002073686F7720765F696E2C2061312C201D
:100D0000613220766F6C74616765730A0D0075201F
:100D100020202020202020202020202020202020D3
:100D2000202020202020202020202D207570746974
:100D30006D650A0D00762020202020202020202014
:100D400020202020202020202020202020202020A3
:100D5000202D2076657273696F6E0A0D0068202061
:100D60002020202020202020202020202020202083
:100D70002020202020202020202D2068656C700A53
:100D80000D00256300756E6B6E6F776E20636D646A
:100D90000A00484D43353838330025730025730069
:100DA000202573002025362E32662000253032782B
:100DB0000074656D705F65787465726E3D252D36C3
:100DC0002E326600202573002025362E3266204FF5
:100DD0006E2D426F61726400253032780074656D4B
:100DE000705F626F6172643D252D362E3266000A97
:100DF00000503A20256C642050612020252D372E8C
:100E00003266206D0A002563002563004932433AAB
:100E10002000452025642E256420636C6F636B20C1
:100E2000256C752063707520256C75206C706D20A5
:100E3000256C752069727120256C7520676C65645E
:100E400020256C7520796C656420256C7520726C8A
:100E5000656420256C7520747820256C75206C697C
:100E60007374656E20256C752073656E736F727375
:100E700020256C752073657269616C20256C750A7C
:100E800000532025642E256420636C6F636B20253E
:100E90006C7520747820256C7520727820256C750F
:100EA0002072747820256C752072727820256C75FC
:100EB000207265786D697420256C752061636B7490
:100EC0007820256C75206E6F61636B747820256CBB
:100ED000752061636B727820256C752074696D656F
:100EE000646F757420256C752062616461636B7238
:100EF0007820256C7520746F6F6C6F6E6720256C81
:100F00007520746F6F73686F727420256C75206222
:100F1000616473796E636820256C75206261646317
:100F2000726320256C7520636F6E74656E74696FD3
:100F30006E64726F7020256C752073656E64696EC7
:100F40006764726F7020256C75206C6C7478202536
:100F50006C75206C6C727820256C750A00257325E1
:100F6000730A004F6E6C696E650A000A002C2063DC
:100F70006865636B207261746520257520487A006E
:100F800025732025732C206368616E6E656C2025A7
:100F90007520706F776572202575000A0025783AF4
:100FA000004D414320616464726573732000526197
:100FB0006E646F6D204555493634206164647265F6
:100FC00073732067656E6572617465640A000A2A2E
:100FD0002A2A2A2A2A2A426F6F74696E672025738B
:100FE0002A2A2A2A2A2A2A0A00454550524F4D20E9
:100FF000697320636F72727570742C2072657772DA
:101000006974696E672077697468206465666175C4
:101010006C74732E0A006C6F63616C686F7374007C
:1010200041544D454741313238726661310002000A
:1010300000FFFE0000016E616E00696E66000040F8
:101040007A10F35A00A0724E18090010A5D4E800D7
:1010500000E87648170000E40B54020000CA9A3BEF
:10106000000000E1F5050000809698000000404275
:101070000F000000A0860100000010270000000003
:10108000E803000000006400000000000A00000007
:1010900000000100000000002C76D888DC674F08B3
:1010A00023DFC1DFAE59E1B1B796E5E3E453C63AB9
:1010B000E651997696E8E6C28426EB898C9B62ED30
:1010C000407C6FFCEFBC9C9F40F2BAA56FA5F490EA
:1010D000055A2AF75C936B6CF9676DC11BFCE0E461
:1010E0000D47FEF520E6B500D0ED902E03009435B7
:1010F00077050080841E080000204E0A000000C80A
:101100000C333333330F986E12831141EF8D21145A
:10111000893BE65516CFFEE6DB18D1844B381BF72A
:101120007C1D901DA4BBE424203284725E228100C9
:10113000C9F124ECA1E53D274E414E494E49545991
:10114000494E46CDCCCC3D0AD7233C17B7D1387792
:10115000CC2B329595E6241FB14F0A0000204100A8
:1011600000C84200401C4620BCBE4CCA1B0E5AAEF2
:10117000C59D740011241FBECFEFD1E4DEBFCDBFEB
:1011800019E0A0E0B2E0E6E1FCE101E00BBF02C043
:1011900007900D92A435B107D9F710E3A4E5B9E0A3
:1011A00001C01D92A33DB107E1F70E94347C0C946D
:1011B000098E0C9400008BEA94E09F938F930E9419
:1011C000118B80914A0290914B020F900F9093FFE8
:1011D00003C085EA94E002C08FE994E09F938F9367
:1011E0000E94118B0F900F900895E091E91AEF7112
:1011F000F0E0E25CF44E80838091E91A8F5F809387
:10120000E91A80910D28886080930D2844E352E00C
:1012100061E1CA010E94C44C80E090E00895CF9340
:10122000DF93EC0180915B0990915C0986FF1DC002
:101230008E811F928F938D811F928F938C811F922D
:101240008F938B811F928F938A811F928F9386E554
:1012500093E09F938F930E94FF8A8DB79EB70C9661
:101260000FB6F8949EBF0FBE8DBFBE0182E999E014
:101270000E94F64DBE0184E092E0DF91CF910C9484
:101280006B4D87EE93E08115910511F00197F1F711
:1012900008958823B9F052985A981DBA8091690030
:1012A000806280936900EA9A53985B98EB9A8091E8
:1012B00069008068809369008091680081608093F4
:1012C00068000895109269005A9AEA985B9AEB9820
:1012D00008951F920F920FB60F9211248F939F9330
:1012E000AF93BF938091680080FF20C08091ED276D
:1012F0009091EE27A091EF27B091F0270196A11DC4
:10130000B11D8093ED279093EE27A093EF27B09324
:10131000F02780915B0990915C0987FF07C0749862
:1013200082E090E090937A0280937902BF91AF912E
:101330009F918F910F900FBE0F901F9018951F9245
:101340000F920FB60F9211248F939F93AF93BF9379
:101350008091680080FF20C08091F1279091F22752
:10136000A091F327B091F4270196A11DB11D8093A0
:10137000F1279093F227A093F327B093F42780915D
:101380005B0990915C0990FF07C0739882E090E040
:1013900090937A0280937902BF91AF919F918F9140
:1013A0000F900FBE0F901F90189580937C00809136
:1013B0007B00877F80937B0080917C00806C809392
:1013C0007C0085E080937A0080917A008068809329
:1013D0007A0080917B0087FFFCCF80917B0085FFA6
:1013E000FCCF80917A00806480937A0080917A00AB
:1013F00086FDFCCF109279001092780084E090E096
:1014000060E070E020917A00206420937A002091BF
:101410007A0026FDFCCF2091780030917900620F90
:10142000731F0197009771F710927C0080917A00EA
:101430008F7780937A00769567957695679580E0AB
:1014400090E00E948A81089580E00E94D509209151
:1014500075023091760240917702509178020E9495
:101460006A8321EE3AE744E95EE30E94238008950F
:1014700080E18093510160E16093510180915101BD
:1014800085FF03C06F5F6F31B9F78BE4689FB001D0
:101490001124882777FD8095982F0E948C8120E069
:1014A00030E64FE954E40E94238020E030E04AE730
:1014B00054E40E94ED800895CF93DF93EC0188817E
:1014C0009981009799F08C309F4021F01982188201
:1014D00083E011C0623171F40E94380A6093912355
:1014E0007093922380939323909394238CE09FE0B6
:1014F0009983888381E0DF91CF91089565FF4BC088
:1015000080917B00886080937B0089EC80937C00D5
:1015100085E080937A0080917A00806880937A00D9
:1015200080917B0087FFFCCF80917B0085FFFCCF03
:1015300080917A00806480937A0080917A0086FDA1
:10154000FCCF80917A00806480937A0080917A0049
:1015500086FDFCCF609178007091790080E090E08A
:101560000E948A8127ED33EA40E95FE30E946A83A3
:1015700026E636E648E853E40E9422806093AE1ADD
:101580007093AF1A8093B01A9093B11A80917A0039
:101590008F7780937A000895BF92CF92DF92EF9277
:1015A000FF920F931F93CF93DF93CDB7DEB72997A9
:1015B0000FB6F894DEBF0FBECDBF6C011092540978
:1015C0008FEF89870AEF1AE1B12C7E0189E0E80EDE
:1015D000F11C89858823E9F1E8E0BE16E1F1BE013E
:1015E0006F5F7F4FC7010E945F5689858F3F11F063
:1015F0008E3F19F4809354092CC0CE010196C1147A
:10160000D10471F40E94785680930A28FE01319625
:10161000A2E0B8E281918D93EE15FF05D9F71DC0C8
:101620000E947856F8018083FE01319620E030E078
:10163000A801485051098191DA01A20FB31F8C9380
:101640002F5F3F4F28303105B1F7B394075F1F4F2D
:10165000C0CF8B2D03C088E001C081E029960FB672
:10166000F894DEBF0FBECDBFDF91CF911F910F91D8
:10167000FF90EF90DF90CF90BF9008958FEE9DE0A8
:101680009F938F930E94118B0F900F9008952F922C
:101690003F924F925F926F927F928F929F92AF9202
:1016A000BF92CF92DF92EF92FF920F931F93CF934F
:1016B000DF93EC014B01009711F427E004C0813067
:1016C000910549F426E04AE250E06BE270E089E2DD
:1016D00090E00E943F55CE010E94CC0A9E012B5AF9
:1016E000364F5901D9018C93CD2B69F09AEFC92E51
:1016F0009AE1D92EC2EFDAE1E12CF12C20EA222E78
:101700002DE0322EA6C082E098E20E94AD57BC01C7
:10171000882777FD8095982F0E948C816B017C0132
:10172000892869F020E030E048EC52E40E94ED8026
:101730009F938F937F936F938DED9DE0ACC0C2E03C
:10174000D8E208ED1DE089911F928F931F930F93AC
:101750000E94118B0F900F900F900F90B8E2CA303B
:10176000DB0789F720E030E048EC52E4C701B6011E
:101770000E94ED809F938F937F936F9388EC9DE001
:101780009F938F930E94118B0F900F900F900F904B
:101790000F900F9080910A28882319F085E893E034
:1017A00002C089EF93E09F938F9384EC9DE09F9319
:1017B0008F930E94118B0F900F900F900F9075C018
:1017C00000E010E0FE01E00FF11F80811F928F9377
:1017D000ACEABDE0BF93AF930E94118B0F5F1F4F28
:1017E0000F900F900F900F900830110559F720E0DF
:1017F00030E048EC52E4C301B2010E94ED809F93B7
:101800008F937F936F93A4EABDE0BF93AF930E9441
:10181000118B0F900F900F900F900F900F90D6019B
:101820008C91882309F455C085E893E09F938F93AA
:101830003F922F920E94118B0E943E0BBFEFEB1A3A
:10184000FB0AE9E0CE0ED11C29960F900F900F9065
:101850000F90D5018C9190E0E816F906ECF5CE01D9
:101860000E94AD57BC01882777FD8095982F0E9474
:101870008C812B013C018114910409F4A1CF20E05B
:1018800030E048EC52E40E94ED809F938F937F9369
:101890006F9381EB9DE09F938F930E94118B0F902C
:1018A0000F900F900F900F900F90DF91CF911F919D
:1018B0000F91FF90EF90DF90CF90BF90AF909F90EF
:1018C0008F907F906F905F904F903F902F900C94EF
:1018D0003E0B89EF93E0AACFDF91CF911F910F913B
:1018E000FF90EF90DF90CF90BF90AF909F908F9040
:1018F0007F906F905F904F903F902F900895CF937F
:10190000DF9300D0CDB7DEB7809103288983809123
:1019100009288A83CE0101960E94B84A0F900F9041
:10192000DF91CF910895CF93DF93EC0120910228AE
:101930003091032840910428509105286091062891
:10194000709107288091082890910928AFEF0E9494
:101950009A86E1F427E04AE250E06BE270E089E227
:1019600090E00E943F5580E090E00E94CC0ACB5A64
:10197000D64F888349E050E06AE070E082E098E268
:101980000E94548CDF91CF910C947F0CDF91CF910A
:1019900008951F920F920FB60F9211240BB60F925B
:1019A0002F933F934F935F936F937F938F939F9367
:1019B000AF93BF93CF93EF93FF9380910D288260F5
:1019C00080930D2880914A0286FD2B9A80914A02CD
:1019D00087FD2B9A8091790290917A021816190648
:1019E00014F4749A739A80915B0990915C0985FF55
:1019F00002C074987398809102029091030201973B
:101A00009093030280930202892B09F050C18091C8
:101A1000690990916A09019690936A09809369090E
:101A20008091952390919623A0919723B09198232C
:101A30000196A11DB11D8093952390939623A093A9
:101A40009723B093982380E190E0909303028093D2
:101A5000020280914A0280FD02C01D9B07C01092C5
:101A600059091092580983B7817F09C081E090E03D
:101A7000909359098093580983B7817F866083BF0B
:101A800080915B0990915C0997FF0BC08091580988
:101A900090915909892B19F0749A739802C0739A1E
:101AA0007498609150027091510261157105B9F0FE
:101AB0008091690990916A0901960E946B84892B33
:101AC00071F4779880915B0990915C0992FF07C04F
:101AD000749884E090E090937A0280937902609108
:101AE00050027091510261157105A1F08091690950
:101AF00090916A0901960E946B84892B59F4109287
:101B0000AC231092AB2342EA53E262E18CE092E014
:101B10000E94C44C60915002709151026115710590
:101B2000B1F18091690990916A090E946B84892BB7
:101B300071F581E08093A223809152028093A323C8
:101B4000809153028093A423809154028093A52313
:101B5000809155028093A623809156028093A723FB
:101B6000809157028093A823809158028093A923E3
:101B7000809159028093AA231092AC231092AB2338
:101B800042EA53E262E18AE292E00E94C44C609130
:101B90004E0270914F0261157105A1F180916909A2
:101BA00090916A090E946B84892B61F58091ED27E1
:101BB0009091EE27A091EF27B091F0274091871BDD
:101BC0005091881B6091891B70918A1B841B950B17
:101BD000A60BB70B8093C11A9093C21AA093C31A95
:101BE000B093C41A8091ED279091EE27A091EF2732
:101BF000B091F0278093871B9093881BA093891B3B
:101C0000B0938A1B60914C0270914D026115710571
:101C1000A1F18091690990916A090E946B84892BD6
:101C200061F58091F1279091F227A091F327B0916F
:101C3000F42740918B1B50918C1B60918D1B7091F0
:101C40008E1B841B950BA60BB70B8093C51A909324
:101C5000C61AA093C71AB093C81A8091F127909121
:101C6000F227A091F327B091F42780938B1B9093D8
:101C70008C1BA0938D1BB0938E1B80914A0286FD16
:101C80002B9880914A0290914B0291FF10C00E94C4
:101C90004F618A3119F0C1E0C80F01C0CBE00E944A
:101CA00009608C2F90E00E9467610E94516040E0C3
:101CB00050E060E08BE792E00E94C44CFF91EF910E
:101CC000CF91BF91AF919F918F917F916F915F91D4
:101CD0004F913F912F910F900BBE0F900FBE0F9021
:101CE0001F9018958091E91A9091A123891B08955E
:101CF0000E94720E882371F0E091A123EF71F0E051
:101D0000E25CF44E808190E02091A1232F5F20932C
:101D1000A12308958FEF9FEF0895CF93DF93EC01F8
:101D20001092860910928509888199810097C1F0E7
:101D30008F35934021F01982188283E0B6C061315B
:101D400009F0B2C0F89478940E94780E9927909385
:101D50008109809380098D3009F441C08F3F49F497
:101D60000E94720E8111EECF8FE593E099838883F4
:101D70009BC08231910509F458C08F37910509F055
:101D800050C080917E0990917F09181619060CF5B4
:101D90006091CD307091CE3088E090E00E94CD8A85
:101DA0006091CD307091CE3080E290E00E94CD8A7B
:101DB0006091CD307091CE3088E090E00E94CD8A65
:101DC00080917E0990917F09019790937F0980937C
:101DD0007E0980917E0990917F09CF9709F6109234
:101DE000A1231092E91A80917E0990917F09FC014C
:101DF000E355FC4D108290938609809385091092DB
:101E00007F0910927E0980910B2890910C280097F1
:101E100009F4A6CF40E050E0609194110E94C44CB8
:101E20009FCF8830910571F5ACCF6091CD30709126
:101E3000CE308DE090E00E94CD8A10927D09109204
:101E40007C0980917C0990917D0920917E093091D7
:101E50007F09821793070CF0BCCFFC01E355FC4DC2
:101E600080816091CD307091CE3090E00E94CD8A1B
:101E700080917C0990917D09019690937D098093D2
:101E80007C09DFCF6091CD307091CE300E94CD8A39
:101E900080917E0990917F0920918009FC01E35592
:101EA000FC4D2083019691CF81E0DF91CF91089581
:101EB0008091580990915909892BB1F080914A027B
:101EC00090914B0293FD10C00E94096083B7817FFF
:101ED000866083BFF89483B7816083BF78948895C8
:101EE00083B78E7F83BF78940895CF93DF93EC01FF
:101EF00088819981009719F081339F4099F40E945D
:101F0000C65E0E94580F40E050E065E8809198114D
:101F1000909199110E94C44C81E39FE0998388833A
:101F200081E003C01982188283E0DF91CF91089588
:101F3000CF93DF9300D0CDB7DEB7892B81F05F93CD
:101F40004F938DE99DE09F938F9369837A830E94DD
:101F5000118B0F900F900F900F907A8169817F9372
:101F60006F938AE99DE09F938F930E94118B0F904E
:101F70000F900F900F900F900F90DF91CF910895D9
:101F8000FF920F931F93CF93DF930E94C65E80EB67
:101F90000E942B5881111CC00E948F5880918F1F66
:101FA0009091901F81609093901F80938F1F8EE877
:101FB00093E09F938F938AE99DE09F938F930E9474
:101FC000118B0F900F900F900F90C1E0D0E002C0E6
:101FD000C0E0D0E0FEB08F2D8470F82E729A0E947F
:101FE000C65E8EE40E942B58811116C00E948F5845
:101FF00080918F1F9091901F82609093901F80938B
:102000008F1F8E010F5F1F4F49EB58E066E973E0A9
:10201000CE010E94980FE801F11001C072980E9451
:10202000C65E8EEE0E942B58811116C00E948F58FA
:1020300080918F1F9091901F84609093901F809348
:102040008F1F8E010F5F1F4F49EB58E06EE973E061
:10205000CE010E94980FE8010E94C65E86EA0E94A7
:102060002B58811116C00E948F5880918F1F90911C
:10207000901F88609093901F80938F1F8E010F5F39
:102080001F4F49EB58E065EA73E0CE010E94980FBC
:10209000E8010E94C65E8CE30E942B5881111EC08D
:1020A0000E948F5880918F1F9091901F8061909314
:1020B000901F80938F1F8E010F5F1F4F49EB58E0D9
:1020C0006DEA73E0CE010E94980F82E99DE09F9334
:1020D0008F930E94118B0F900F90E8010E94C65EB3
:1020E00082ED0E942B58811116C00E948F5880915A
:1020F0008F1F9091901F80629093901F80938F1FED
:102100008E010F5F1F4F49EB58E065EB73E0CE0186
:102110000E94980FE8010E94C65E80E80E942B583A
:10212000811116C00E948F5880918F1F9091901F2F
:1021300091609093901F80938F1F8E010F5F1F4FB0
:1021400049EB58E06EEB73E0CE010E94980FE80176
:102150000E94C65E80ED0E942B58811116C00E941D
:102160008F5880918F1F9091901F80689093901F3F
:1021700080938F1F8E010F5F1F4F49EB58E064EC77
:1021800073E0CE010E94980FE8010E94C65E8CEEBB
:102190000E942B58811116C00E948F5880918F1F6A
:1021A0009091901F92609093901F80938F1F8E014B
:1021B0000F5F1F4F49EB58E06CEC73E0CE010E94BB
:1021C000980FE80107E010E00E94C65E8CE70E94CD
:1021D0002B58811113C00E948F5880918F1F9091AE
:1021E000901F80649093901F80938F1F49EB58E05D
:1021F00063ED73E0CE010E94980F05C001501109F4
:102200000115110509F70E948F58DF91CF911F9199
:102210000F91FF900C943E0BCF93DF9300D0CDB77E
:10222000DEB74A8369830E9466586981862F0E94BF
:1022300097584A81842F0E9497580F900F90DF91F2
:10224000CF910C948F58AF92BF92DF92EF92FF9292
:102250000F931F93CF93DF9300D01F92CDB7DEB7BC
:10226000182FD22E4A835B8369830E946658698146
:10227000862F0E949758812F81600E948D584A8135
:10228000A42E5B81B52E00E010E0ED2CF12C81E056
:10229000E81AF1080D1580F40E151F0519F40E94B7
:1022A000B25802C00E94A858F50180830F5F1F4FEB
:1022B000FFEFAF1ABF0AEECF0F900F900F90DF9194
:1022C000CF911F910F91FF90EF90DF90BF90AF9053
:1022D0000C948F58AF92BF92CF92DF92EF92FF9201
:1022E0000F931F93CF93DF93CDB7DEB760970FB6F1
:1022F000F894DEBF0FBECDBFB82EA42E6623E9F141
:102300008E010F5F1F4F80E1F80111928A95E9F766
:1023100028E0A80168E980EB0E942311BB2041F06E
:102320002CED33E03F932F930E94FF8A0F900F9084
:102330006E01F8E0CF0ED11C43EEE42E43E0F42E04
:10234000F80181918F011F928F93FF92EF920E946B
:10235000FF8A0F900F900F900F900C151D0581F7BD
:1023600088851F928F9328E334E03F932F930E9438
:10237000FF8A0F900F900F900F90AA20E9F18E0125
:102380000F5F1F4F80E1F80111928A95E9F728E06D
:10239000A80160E880EB0E942311BB2041F088EE89
:1023A00093E09F938F930E94FF8A0F900F906E018E
:1023B000F0E1CF0ED11C33EEE32E33E0F32EF80123
:1023C00081918F011F928F93FF92EF920E94FF8A5B
:1023D0000F900F900F900F900C151D0581F78885B9
:1023E0001F928F9388E394E09F938F930E94FF8ABC
:1023F0000F900F900F900F9060960FB6F894DEBF7D
:102400000FBECDBFDF91CF911F910F91FF90EF9045
:10241000DF90CF90BF90AF900895CF93DF9300D01F
:10242000CDB7DEB71A82198222E0AE014F5F5F4F4F
:102430006AEA8EEE0E942311898190E0982F882706
:102440002A81822B90935F1B80935E1B22E0AE015A
:102450004F5F5F4F6CEA8EEE0E942311898190E0FE
:10246000982F88272A81822B9093611B8093601B71
:1024700022E0AE014F5F5F4F6EEA8EEE0E942311A5
:10248000898190E0982F88272A81822B9093631B63
:102490008093621B22E0AE014F5F5F4F60EB8EEED8
:1024A0000E942311898190E0982F88272A81822B0E
:1024B0009093711B8093701B22E0AE014F5F5F4FC2
:1024C00062EB8EEE0E942311898190E0982F88277D
:1024D0002A81822B9093731B8093721B22E0AE01A2
:1024E0004F5F5F4F64EB8EEE0E942311898190E075
:1024F000982F88272A81822B9093751B8093741BB9
:1025000022E0AE014F5F5F4F66EB8EEE0E9423111B
:10251000898190E0982F88272A81822B9093651BD0
:102520008093641B22E0AE014F5F5F4F68EB8EEE3D
:102530000E942311898190E0982F88272A81822B7D
:102540009093671B8093661B22E0AE014F5F5F4F45
:102550006AEB8EEE0E942311898190E0982F8827E4
:102560002A81822B90936B1B80936A1B22E0AE0121
:102570004F5F5F4F6CEB8EEE0E942311898190E0DC
:10258000982F88272A81822B90936D1B80936C1B38
:1025900022E0AE014F5F5F4F6EEB8EEE0E94231183
:1025A000898190E0982F88272A81822B90936F1B36
:1025B00080936E1B0F900F90DF91CF9108952F9213
:1025C0003F924F925F926F927F928F929F92AF92C3
:1025D000BF92CF92DF92EF92FF920F931F93CF9310
:1025E000DF93CDB7DEB76A970FB6F894DEBF0FBEA4
:1025F000CDBF182F488F298F19821A821B82809194
:10260000821B811107C06A8F0E940D1281E08093A6
:10261000821B6A8D662309F46CC04EE264EF8EEE75
:102620000E940C1169E07AE180E090E00E94185865
:1026300022E0AE014F5F5F4F66EF8EEE0E942311E6
:102640002981822F90E0A0E0B0E02227382F492F87
:102650005A2F8A81282B8091741B9091751B281BFF
:10266000390B41095109A091721BB091731B0E9453
:1026700048846B017C018FE0F594E794D794C7946C
:102680008A95D1F760916C1B70916D1B882777FD3F
:102690008095982F2BE0660F771F881F991F2A952A
:1026A000D1F720916E1B30916F1B442737FD409569
:1026B000542F2C0D3D1D4E1D5F1D0E94B584C20E72
:1026C000D31ED092691BC092681B88E0C80ED11C33
:1026D00034E0D594C7943A95E1F7EE24D7FCE09422
:1026E000FE2CC092761BD092771BE092781BF09262
:1026F000791B012F0295000F000F007C0C5CA12FAD
:10270000B0E0BD8BAC8BA3E0B0E0012E02C0AA0FFD
:10271000BB1F0A94E2F725E335E00E944184DC0107
:10272000CB010296A11DB11D8C879D87AE87BF8707
:1027300080E593ECA0E0B0E004C0B595A79597952F
:1027400087951A95D2F7888B998BAA8BBB8B10E053
:10275000188619861A861B86A8E02A2E312CAC8989
:10276000BD892A1A3B0A988D191709F436C1402FE2
:1027700064EF8EEE0E940C116C857D858E859F85A1
:102780000E94185823E0AE014F5F5F4F66EF8EEE58
:102790000E942311E091681BF091691BE05AFF40F1
:1027A0009F01DF010E942A846B017C018091601BE4
:1027B0009091611B9F8B8E8BA0905E1BB0905F1BD6
:1027C0002091621B3091631B0E942A842B013C01E3
:1027D0003DE075946794579447943A95D1F7A0914A
:1027E000641BB091651BA70196016CE05595479558
:1027F000379527956A95D1F70E945384BB2797FD9B
:10280000B095AB2F480E591E6A1E7B1E92E0490EF2
:10281000511C611C711CB2E07594679457944794E5
:10282000BA95D1F7A0E85A0E611C711CA091701BDB
:10283000B091711BA30192010E944884DC01CB017D
:102840002FE0B695A795979587952A95D1F78C8314
:102850009D83AE83BF8329818A8190E0A0E0B0E0B0
:102860004424582E692E7A2E622A8B81482A022C03
:1028700004C075946794579447940A94D2F745011D
:10288000AA2497FCA094BA2C42E0880C991CAA1C9C
:10289000BB1C4A95D1F7A091661BB091671BA7019D
:1028A00096010E9453846B017C0157E1F594E794F3
:1028B000D794C7945A95D1F72E893F89DF010E949A
:1028C0002A84EBE09595879577956795EA95D1F7FA
:1028D000C60ED71EE81EF91E8C0C9D1CAE1CBF1C1C
:1028E0000C8804C0880C991CAA1CBB1C0A94D2F743
:1028F00092E0890E911CA11CB11CF2E0B594A79442
:1029000097948794FA95D1F7481859086A087B0874
:10291000A3019201688979898A899B890E945B84D5
:1029200097FD0DC0660F771F881F991F2C813D8171
:102930004E815F810E94938449015A010CC02C8111
:102940003D814E815F810E94938449015A01880C28
:10295000991CAA1CBB1C9927B7FC9A958B2D7A2D24
:10296000692D9B01AC010E945B849B01AC01AEED23
:10297000BBE00E9448846C01FF24D7FCF094EF2C4C
:10298000A3E4B3EEA50194010E945684BB2797FDF2
:10299000B095AB2FC80ED91EEA1EFB1EAFECCA0EB7
:1029A000AEE0DA1EE11CF11CA4E0F594E794D794A4
:1029B000C794AA95D1F7C80CD91CEA1CFB1C8885C2
:1029C0009985AA85BB858C0D9D1DAE1DBF1D888771
:1029D0009987AA87BB871F5FC6CE112391F0212F4D
:1029E00030E040E050E0688579858A859B850E94CB
:1029F000938420937A1B30937B1B40937C1B5093D2
:102A00007D1BA98DAA2389F160917A1B70917B1B94
:102A100080917C1B90917D1B61157105810591054D
:102A200021F10E948C8120E836EE45EC57E40E94AB
:102A3000ED8021E03EED42E45EE30E94CD839B0108
:102A4000AC0160E070E080E89FE30E9422802BE40C
:102A50003AE34DEB57E30E94ED8060937E1B709349
:102A60007F1B8093801B9093811B6A960FB6F8940E
:102A7000DEBF0FBECDBFDF91CF911F910F91FF90B1
:102A8000EF90DF90CF90BF90AF909F908F907F900E
:102A90006F905F904F903F902F9008950F931F93EA
:102AA000CF93DF9300D000D000D0CDB7DEB78E013A
:102AB0000F5F1F4F86E0F80111928A95E9F7809128
:102AC000B81A811113C040E061E386EA0E940C113C
:102AD0004AE06CE286EA0E940C1181E08093B81A09
:102AE0006CE77EE380E090E00E94185848E06DE2D9
:102AF00086EA0E940C116CE77EE380E090E00E9481
:102B0000185826E0A80162E386EA0E94231147E0F4
:102B10006DE286EA0E940C118A8190E0982F882746
:102B20002981822B9093B31A8093B21A2C8130E0C2
:102B3000322F22274B81242B3093B51A2093B41ABD
:102B40004E8150E0542F44276D81462B5093B71A85
:102B50004093B61A5F934F933F932F939F938F9316
:102B60008CEE93E09F938F930E94FF8A0FB6F894A8
:102B7000DEBF0FBECDBF26960FB6F894DEBF0FBEE8
:102B8000CDBFDF91CF911F910F910895CF92DF922A
:102B9000EF92FF920F931F93CF93DF93CDB7DEB7E2
:102BA0002A970FB6F894DEBF0FBECDBF8E010F5F20
:102BB0001F4F86E0F80111928A95E9F741E062E043
:102BC0008CE30E940C1148E560E08CE30E940C113C
:102BD00062E174E380E090E00E94185826E0A801CA
:102BE00063E08CE30E94231143E062E08CE30E94E7
:102BF0000C11098110E0102F00278A81082B1093F7
:102C00008F1A00938E1AEB80F12CFE2CEE248C810F
:102C1000E82AF092911AE092901ACD80D12CDC2C07
:102C2000CC248E81C82AD092931AC092921AB801ED
:102C3000882777FD8095982F0E948C819B01AC019D
:102C4000B701882777FD8095982F2F83388749878C
:102C50005A870E948C812F81388549855A850E9428
:102C6000968020EE3EE245E652E40E946A8320E030
:102C700030E044E353E40E9423809F938F937F933B
:102C80006F93DF92CF92FF92EF921F930F938AEF91
:102C900093E09F938F930E94FF8A0FB6F894DEBF54
:102CA0000FBECDBF2A960FB6F894DEBF0FBECDBFC4
:102CB000DF91CF911F910F91FF90EF90DF90CF9018
:102CC0000895CF93DF93EC01888199810097F9F003
:102CD0008A319F4021F01982188283E063C08BE61D
:102CE00099E00E946A4F892BE1F080915B099091F5
:102CF0005C0993FD18C080915B0990915C0994FD7B
:102D000043C080915B0990915C0995FD44C060E8E7
:102D100070E08BE699E00E94434F8AE19FE099833F
:102D2000888381E03FC080918F1F82FFE4CF21E044
:102D300048E061E083E00E94DF128091811B8F9365
:102D40008091801B8F9380917F1B8F9380917E1B3E
:102D50008F9380917D1B8F9380917C1B8F938091AB
:102D60007B1B8F9380917A1B8F9381EF9DE09F93C4
:102D70008F930E94118B8DB79EB70A960FB6F89469
:102D80009EBF0FBE8DBFB7CF80918F1F83FFB9CF7E
:102D90000E944E15B6CF80918F1F84FFB8CF0E943E
:102DA000C615B5CFDF91CF910895CF93C82F8CEE84
:102DB0000E948D588C2F0E94975865E375E080E043
:102DC00090E00E9418588DEE0E948D580E94A858DD
:102DD000C82F0E94B2582C2F30E0322F2227A90191
:102DE000482BCA01CF910895CF93DF93C82F8CEE63
:102DF0000E948D588C2F0E94975862E174E380E006
:102E000090E00E9418588CEE0E948D5880E00E943D
:102E1000975865E375E080E090E00E9418588DEEC9
:102E20000E948D580E94A858C82F0E94A858D82FD9
:102E30000E94B2584D2F50E060E070E0762F652F71
:102E4000542F44276C2B482BCB01BA01DF91CF9133
:102E500008952F923F924F925F926F927F928F923E
:102E60009F92AF92BF92CF92DF92EF92FF920F9319
:102E70001F93CF93DF93CDB7DEB7CD54D1090FB6F3
:102E8000F894DEBF0FBECDBF809100029091010289
:102E9000892BD1F110920102109200028CEE0E9457
:102EA0008D588EE10E9497586BE17EE480E090E0BF
:102EB0000E94185882EA0E94D51690936809809360
:102EC000670984EA0E94D516909366098093650984
:102ED00086EA0E94D516909364098093630988EA74
:102EE0000E94D51690936209809361098AEA0E9434
:102EF000D5169093600980935F098CEA0E94D516DD
:102F000090935E0980935D0988E40E94F4166FAB8C
:102F100078AF89AF9AAF88E50E94F4164B015C0147
:102F200080915F099091600920E030E040E050E03E
:102F3000BA0126962FAF269727963FAF2797289658
:102F40004FAF289729965FAF29972A966FAF2A9798
:102F50002B967FAF2B979C0140E050E060E070E043
:102F600080E090E008E00E943C860E94E8853901FC
:102F7000B42FA52FF62FE72F8C019401A50160E057
:102F800070E080E090E05301CB2EDA2EEF2EFE2E83
:102F90000E94738629833A832A011B014C01B101E7
:102FA000C401315041095F4F6F4F7F4F8F4F9F4F8B
:102FB000A1E0B0E02596BFAFAEAF259721153F4FFA
:102FC0004F4F5140610571058105910509F020F4CD
:102FD00025961FAE1EAE259725966EAC7FAC259725
:102FE00080915D0990915E095C01C12CD12CE12C8E
:102FF000F12C00E010E029813A81A201B101C40165
:103000000E940B85D22EE32EF42E052F162FB72FFC
:10301000F82FE92FA0E00E949A8684F4215031090C
:1030200040485F4F6F4F7F4F8F4F9F4FD22EE32E01
:10303000F42E052F162FB72FF82FE92F2D2D3E2D0B
:103040004F2D502F612F7B2F8F2F9E2F07E10E9436
:1030500055862B8F3C8F4D8F5E8F6F8F78A389A302
:103060009AA32053384F4F4F5F4F6F4F7F4F8F4F73
:103070009F4F2B8B3C8B4D8B5E8B6F8B788F898F0B
:103080009A8F2056304F4F4F5F4F6F4F7F4F8F4F6C
:103090009F4F243D30434105510561057105810570
:1030A000910541F038F025966EAC7FAC2597FFEF87
:1030B0006F1A7F0A80916509909166099C0140E032
:1030C00050E060E070E080E090E000E10E943C862B
:1030D0002B833C834D835E836A8779878F839887B0
:1030E0004091610950916209A980BA806201710121
:1030F00084019A0140E050E060E070E080E090E000
:103100000E940B85D22EE32EF42E052F162FB72FFB
:10311000F82FE92FA0E00E949A865CF4AFE70E94A6
:103120007C86D22EE32EF42E052F162FB72FF82FE4
:10313000E92F2D2D3E2D4F2D502F612F7B2F8F2FBF
:103140009E2F07E00E94558659016A017B018C0180
:103150002B813C814D815E816A8579858F8198853F
:103160000E9473862B833C834D835E836F837887B5
:103170008F87988B2E5F3F4F434051096E4F7F4F93
:103180008F4F9F4F22303105494F5F4F644071058B
:103190008105910521F018F01FEF611A710A8091E5
:1031A000670990916809BC0180E090E020E030E878
:1031B00040E050E00E94648529873A874B875C870E
:1031C0006A8B798B8D879E87409163095091640942
:1031D000A980BA806201710184019A0140E050E047
:1031E00060E070E080E090E00E940B85D22EE32E3C
:1031F000F42E052F162FB72FF82FE92FA0E00E94ED
:103200009A8684F421503F4F4F4F5F4F6F4F7F4F4F
:103210008F4F9F4FD22EE32EF42E052F162FB72F50
:10322000F82FE92F2D2D3E2D4F2D502F612F7B2F65
:103230008F2F9E2F08E00E94558659016A017B015D
:103240008C0129853A854B855C856A8979898D85CC
:103250009E850E94738629873A874B875C876D8796
:103260007E87898B9A8B2F5F3F4F414051096109BF
:10327000710981099109213030484C4F5F47614005
:1032800071058105910521F018F0BFEF6B1A7B0ADB
:103290002B893C894D895E896F89788D898D9A8DBE
:1032A0002F3C3740410551056105710581059105A8
:1032B00011F00CF0A5C1A980BA80620171018401EE
:1032C0009501A201B101C4010E940B85A12CB12C72
:1032D000C12C10E8D12EE12CF12C00E010E00E946E
:1032E000CE842BAF3CAF4DAF5EAF6FAF21967FAFBB
:1032F000219722968FAF229723969FAF2397AB8C6F
:10330000BC8CCD8CDE8CEF8CF8A009A11AA19501A4
:10331000A601B701C8010E940B8559016A017B0112
:10332000E82F192F02E00E943C860E2F0E94738620
:1033300069017A01162F272EF82FE92F322E8D2CB6
:10334000942EAF2CB62E072F582EB92FA0E00E9436
:103350009A865CF4A1E00E947C86322E832E942E05
:10336000A52EB62E072F582EB92F232D382D492DD7
:103370005A2D6B2D702F852D9B2F01E00E945586B5
:103380002E962FAF2E972D963FAF2D9749A75AA770
:103390006BA77CA78DA79EA7522E432E4BA35CA3A1
:1033A0006DA37EA38FA398A7B22D9601A701612FCD
:1033B000722D8F2F9E2FA0E00E949A864CF4A3E0DE
:1033C0000E947C8669017A01162FB72FF82FE92F0A
:1033D0009601A701612F7B2F8F2F9E2F02E00E9465
:1033E00055862FA738AB49AB5AAB6BAB7CAB8DABDB
:1033F0009EAB19014A01B62FA72F24968FAF2497B1
:10340000F92F2B893C894D895E896F89788D898D4B
:103410009A8D24323A4F4F4F5F4F6F4F7F4F8F4FF0
:103420009F4F0CF08CC02B8D3C8D4D8D5E8D6F8D24
:1034300078A189A19AA12455324F4F4F5F4F6F4F0A
:103440007F4F8F4F9F4F59016A017B018C010E9472
:103450000B8519014A01B62FA72FFC0103E00E943A
:103460003C8651016401EB2EFA2E8F010E94888662
:1034700059016A017B018C012E962FAD2E972D9656
:103480003FAD2D9749A55AA56BA57CA58DA59EA5F9
:103490000E947386522E432E4BA35CA36DA37EA382
:1034A0008FA398A79101A4016B2F7A2FCF0102E07F
:1034B0000E943C8651016401EB2EFA2E8F010E947E
:1034C000888602E00E943C860E2F0E948886F22E9B
:1034D000032F142FD52EE62EB72FF82FE92FA0E0BB
:1034E0000E949A865CF4A1E00E947C86F22E032F53
:1034F000142FD52EE62EB72FF82FE92F2F2D302F92
:10350000412F5D2D6E2D7B2F8F2F9E2F01E00E946E
:10351000558659016A017B018C012FA538A949A95B
:103520005AA96BA97CA98DA99EA90E94738619012D
:103530004A01B62FA72F24968FAF2497F92F2B81FE
:103540003C814D815E816F8178858F859889A52C1E
:10355000B42CCBA0DCA0EDA0FEA00FA118A50E946A
:1035600088862B833C834D835E836F8378878F8728
:10357000988B29853A854B855C856D857E85898903
:103580009A8951016401EB2EFA2E24960FAD2497EF
:103590001F2F0E94888629873A874B875C876D8713
:1035A0007E87898B9A8B2B893C894D895E896F89AF
:1035B000788D898D9A8DABACBCACCDACDEACEFAC6C
:1035C0002196FFAC219722960FAD229723961FAD2F
:1035D00023970E9488862056304F4F4F5F4F6F4F82
:1035E0007F4F8F4F9F4F243D30434105510561056B
:1035F00071058105910521F018F02FEF621A720A0A
:103600006FA978AD89AD9AADAB01BC0180E090E0C7
:10361000DC0124964FAF249725965FAF2597269619
:103620006FAF269727967FAF279728968FAF28975B
:1036300029969FAF29972A96AFAF2A972B96BFAFAF
:103640002B97A984BA84CB84DC84ED84FE84098919
:103650001A899A01AB0160E070E080E090E00E947E
:103660000B85F22E032F142FD52EE62EB72FF82F11
:10367000E92FA0E00E949A8684F421503109404E3F
:103680005F4F6F4F7F4F8F4F9F4FF22E032F142F9F
:10369000D52EE62EB72FF82FE92F2F2D302F412FC3
:1036A0005D2D6E2D7B2F8F2F9E2F05E10E9455865D
:1036B000AB80BC80CD80DE80EF80F8840F851889D8
:1036C0000E948886F22E032F142FD52EE62EB72FB8
:1036D000F82FE92FA0E00E949A8684F42150304808
:1036E0004F4F5F4F6F4F7F4F8F4F9F4FF22E032FE4
:1036F000142FD52EE62EB72FF82FE92F2F2D302F90
:10370000412F5D2D6E2D7B2F8F2F9E2F0FE00E945E
:10371000558669017A018B018A83998329011A01EF
:103720004B015C01285E334041095109610971096F
:1037300081099109283D304D4140510561057105D0
:103740008105910521F018F0BFEF6B1A7B0A0E94EA
:103750008F58672859F09601A701B8018A8199818D
:103760000E94E88529011A014B015C019201A10127
:10377000B401C5010E94868120E030E048EC52E4AB
:103780000E94ED80C35BDF4F0FB6F894DEBF0FBE23
:10379000CDBFDF91CF911F910F91FF90EF90DF9000
:1037A000CF90BF90AF909F908F907F906F905F90E1
:1037B0004F903F902F9008954F925F926F927F921B
:1037C0008F929F92AF92BF92CF92DF92EF92FF9231
:1037D0002B013C0169017A0123EC35EF4CE851E4FF
:1037E000C701B6010E946A834B015C0128EB3EE1F0
:1037F00043E753E4C701B6010E9423809B01AC015B
:10380000C501B4010E94ED800E945A814B015C0108
:1038100020E030E048EC52E4C301B2010E94ED80A8
:1038200021E835E943EC50E40E946A83A501940144
:103830000E946A834B015C0123E333E948E853E4C7
:10384000C701B6010E9423809B01AC01C501B401F0
:103850000E94ED8023E333EB48E553E40E946A8342
:10386000FF90EF90DF90CF90BF90AF909F908F90A0
:103870007F906F905F904F9008954F925F926F92FC
:103880007F928F929F92AF92BF92CF92DF92EF92F0
:10389000FF9269017A010E94EC8220E030E040E072
:1038A00050E40E94228022E93CE54EED5EE30E9456
:1038B000ED804B015C0123EC35EF4CE851E4C7018E
:1038C000B6010E946A832B013C0128EB3EE143E7ED
:1038D00053E4C701B6010E9423809B01AC01C301E0
:1038E000B2010E94ED809B01AC01C501B4010E94B0
:1038F00023806B017C0128EB3EE143E753E40E9407
:103900006A834B015C01A701960163EC75EF8CE8BB
:1039100091E40E9422809B01AC01C501B4010E9488
:10392000ED80FF90EF90DF90CF90BF90AF909F9091
:103930008F907F906F905F904F9008954F925F921D
:103940006F927F928F929F92AF92BF92CF92DF92AF
:10395000EF92FF922B013C0169017A0123EC35EFD4
:103960004CE851E4C701B6010E946A834B015C0137
:1039700028EB3EE143E753E4C701B6010E942380F0
:103980009B01AC01C501B4010E94ED800E945A81E7
:103990004B015C0120E030E048EC52E4C301B2018D
:1039A0000E94ED80A50194010E946A8320E030E02E
:1039B00040E251E40E94228024EE38E34EE05FE3CF
:1039C0000E946A839B01AC01C701B6010E9423805B
:1039D000FF90EF90DF90CF90BF90AF909F908F902F
:1039E0007F906F905F904F900895CF92DF92EF920B
:1039F000FF920F931F93CF93DF9380E80E948D581F
:103A00008AEF0E9497588FE00E94975865E375E00F
:103A100080E090E00E94185881E80E948D580E9432
:103A2000A858C82F0E94A8580E94A858D82F0E94B2
:103A3000A8580E94A858182F0E94A8580E94B2584F
:103A4000082F0E94B25880E80E948D588CEF0E9487
:103A5000975889EC0E94975865E375E080E090E004
:103A60000E94185881E80E948D580E94A858D82EAC
:103A70000E94A858C82E0E94A8580E94A858F82E44
:103A80000E94A858E82E0E94B2581F92CF921F920F
:103A9000DF921F920F931F921F931F92DF931F922B
:103AA000CF931F92EF921F92FF928FE094E09F932B
:103AB0008F930E94FF8A0E948F588DB79EB74296BF
:103AC0000FB6F8949EBF0FBE8DBF20E030E040E0FF
:103AD00050E060E070E080E090E0DF91CF911F91D6
:103AE0000F91FF90EF90DF90CF9008950F931F9369
:103AF000CF93DF93EC0180E80E948D58209741F02E
:103B000085EE0E94975861E077E980E090E007C079
:103B100083EE0E94975869E97AEB81E090E00E9479
:103B2000185881E80E948D580E94A858182F0E94AA
:103B3000A858082F0E94B2580E948F58602F70E03A
:103B4000712B6C7F80E090E0CD2B69F00E948A8120
:103B500020E030E04AEF5AE30E946A8320E030E040
:103B600040EC50E40CC00E948A8122E538EB4FE221
:103B70005BE30E946A8326E636E64BE352E40E944A
:103B80002280DF91CF911F910F9108950F931F9382
:103B9000CF93DF93729A80914A0283FF08C08EE42C
:103BA0000E942B58811163C0C0E5D0E008C0C0E579
:103BB000D0E00E94410921972097D9F7F0CF0E94C9
:103BC000410921972097D9F78FE40E942B580E9432
:103BD000A858082F0F730E94A858182F0E94A858A1
:103BE000D82F0E94B258C82F0E948F5880914A0245
:103BF00083FF7298602F70E0762F6627610F711D2A
:103C000080E090E00E948A8120E134E048EC5BE3B0
:103C10000E946A836093831B7093841B8093851B2F
:103C20009093861B6D2F70E0762F66276C0F711DA9
:103C3000769567957695679580E090E00E948A81F9
:103C400024EA3CEF44E25CE30E946A8320E030E037
:103C500040E252E40E94228060930E2870930F2865
:103C6000809310289093112880E090E002C081E0BA
:103C700090E0DF91CF911F910F9108957298729A01
:103C80008EE40E942B5880EA0E94975880E00E94A0
:103C9000975880E00E9497588FE40E942B580E940A
:103CA000A8588EE40E942B5880E80E94975880E024
:103CB0000E94975880E00E9497580E948F5880E099
:103CC00090E0089585E89DE09F938F930E94118B6B
:103CD00080916C020F900F90882361F01F928F9358
:103CE00082E89DE09F938F930E94118B0F900F901D
:103CF0000F900F9008958DE59DE09F938F930E9404
:103D0000118B85E39DE09F938F930E94118B8EE032
:103D10009DE09F938F930E94118B83ED9CE09F9376
:103D20008F930E94118B81EA9CE09F938F930E9456
:103D3000118B85E69CE09F938F930E94118B8FE3FC
:103D40009CE09F938F930E94118B89E09CE09F934E
:103D50008F930E94118B80918F1F9091901F827082
:103D600091702DB73EB7205F3F4F0FB6F8943EBF1E
:103D70000FBE2DBF892B41F089ED9BE09F938F9360
:103D80000E94118B0F900F908DEA9BE09F938F9371
:103D90000E94118B84E89BE09F938F930E94118B6C
:103DA00088E59BE09F938F930E94118B89E29BE0B3
:103DB0009F938F930E94118B87EF9AE09F938F932D
:103DC0000E94118B86EC9AE09F938F930E94118B37
:103DD0008FE89AE09F938F930E94118B8FE59AE072
:103DE0009F938F930E94118B83E39AE09F938F930D
:103DF0000E94118B84E09AE09F938F930E94118B15
:103E00008BEC99E09F938F930E94118B82E999E04C
:103E10009F938F930E94118B8BE599E09F938F93D3
:103E20000E94118B8AE299E09F938F930E94118BDD
:103E30008BEF98E09F938F930E94118B8CEC98E00E
:103E40009F938F930E94118B8DB79EB780960FB66C
:103E5000F8949EBF0FBE8DBF85EA98E09F938F9325
:103E60000E94118B8FE698E09F938F930E94118B95
:103E700089E398E09F938F930E94118B80E198E0F3
:103E80009F938F930E94118B85ED97E09F938F9363
:103E90000E94118B8AEA97E09F938F930E94118B67
:103EA0002DB73EB7245F3F4F0FB6F8943EBF0FBE0D
:103EB0002DBF08958EE394E00C94358B4F925F9262
:103EC0006F927F928F929F92AF92BF92CF92DF922A
:103ED000EF92FF92CF93DF93CDB7DEB728970FB65F
:103EE000F894DEBF0FBECDBF8091952390919623AD
:103EF000A0919723B091982389839A83AB83BC8345
:103F0000409095235090962360909723709098232B
:103F10008091952390919623A0919723B091982317
:103F20008D839E83AF83B88760919523709196238C
:103F300080919723909198232CE3822E912CA12C91
:103F4000B12CA50194010E9493847F936F9330E17B
:103F5000C32E3EE0D32EE12CF12C6D817E818F812A
:103F60009885A70196010E949384A50194010E945F
:103F700093843F932F9340E8842E41E5942EAA2406
:103F8000A394B12CC301B201A50194010E949384B2
:103F9000A70196010E9493843F932F9369817A81B0
:103FA0008B819C81A50194010E9493843F932F9360
:103FB00084E897E09F938F930E94118B0FB6F8943B
:103FC000DEBF0FBECDBF28960FB6F894DEBF0FBE82
:103FD000CDBFDF91CF91FF90EF90DF90CF90BF905A
:103FE000AF909F908F907F906F905F904F900895CB
:103FF000E3EDF0E3808191818234924479F0E35DD6
:10400000F043FF93EF9386E697E09F938F930E9490
:10401000118B0F900F900F900F9008953A96E53FF7
:1040200081E4F80738F30895CF93DF93EC018C9A7D
:104030000E94240A9F938F937F936F938AE597E062
:104040009F938F930E94118B0F900F900F900F9062
:104050000F900F90209719F00E943E0B08C088E542
:1040600097E09F938F930E94118B0F900F9081E0A8
:104070000E94D50920917102309172024091730221
:10408000509174020E946A839F938F937F936F93E2
:104090008CE497E09F938F930E94118B0F900F9069
:1040A0000F900F900F900F90209719F00E943E0BE9
:1040B00008C08AE497E09F938F930E94118B0F9022
:1040C0000F9082E00E94D50920916D0230916E021E
:1040D00040916F02509170020E946A839F938F9368
:1040E0007F936F938EE397E09F938F930E94118B42
:1040F0000F900F900F900F900F900F90209719F046
:104100000E943E0B08C08CE397E09F938F930E9420
:10411000118B0F900F9083E00E94D5099F938F938E
:104120007F936F938DE297E09F938F930E94118B03
:104130008C980F900F900F900F900F900F902097EA
:1041400019F00E943E0B08C08BE297E09F938F937B
:104150000E94118B0F900F9080918F1F87FF83C05B
:1041600021E042E161E080ED0E94EF599F938F933F
:104170007F936F938EE197E09F938F930E94118BB3
:104180000F900F900F900F900F900F90209719F0B5
:104190000E943E0B08C08CE197E09F938F930E9492
:1041A000118B0F900F9021E042E162E080ED0E94C0
:1041B000EF599F938F937F936F938FE097E09F9337
:1041C0008F930E94118B0F900F900F900F900F9074
:1041D0000F90209719F00E943E0B08C08DE097E0E9
:1041E0009F938F930E94118B0F900F9021E042E1DB
:1041F00063E080ED0E94EF599F938F937F936F93BD
:1042000080E097E09F938F930E94118B0F900F9007
:104210000F900F900F900F90CD2B19F00E943E0B36
:1042200008C08EEF96E09F938F930E94118B0F90A2
:104230000F9021E042E164E080ED0E94EF599F93EE
:104240008F937F936F9381EF96E09F938F930E945C
:10425000118B0F900F900F900F900F900F90DF9198
:10426000CF910C943E0BCD2BD1F3DF91CF910895DC
:104270000F931F93CF93DF93882389F049E050E099
:104280006FEF70E082E098E20E946D8A49E050E0B2
:104290006AE070E082E098E20E94548C13C0C2E0B1
:1042A000D8E20CEE16E089911F928F931F930F9323
:1042B0000E94118B0F900F900F900F9088E2CA30E0
:1042C000D80789F7DF91CF911F910F910C943E0B86
:1042D000CF92DF92EF92FF92CF93DF936B017C013D
:1042E00060FF11C08BE794E09F938F938AE99DE074
:1042F0009F938F930E94118B0F900F900F900F90B0
:1043000081E090E002C080E090E0C1FE09C0EC01D5
:10431000219649EB58E060E874E00E94980FCE01C6
:10432000C2FE09C0EC01219649EB58E068E874E050
:104330000E94980FCE01C3FE09C0EC01219649EB03
:1043400058E060E974E00E94980FCE01C4FE09C0F5
:10435000EC01219649EB58E064E974E00E94980F63
:10436000CE01C5FE09C0EC01219649EB58E067E992
:1043700074E00E94980FCE01C6FE09C0EC012196A0
:1043800049EB58E06BE974E00E94980FCE01C7FE3C
:1043900009C0EC01219649EB58E061EA74E00E9403
:1043A000980FCE01D0FE09C0EC01219649EB58E0F0
:1043B00069EA74E00E94980FCE01D1FE09C0EC01B9
:1043C000219649EB58E061EB74E00E94980FCE0112
:1043D000D2FE09C0EC01219649EB58E065EB74E090
:1043E0000E94980FCE0120918F1F3091901F247052
:1043F0003270232B59F0D3FE09C0EC01219649EB12
:1044000058E06BEB74E00E94980FCE0120918F1F53
:1044100023FF0BC0D4FE09C0EC01219649EB58E004
:1044200060EC74E00E94980FCE0120918F1F24FF52
:104430000BC0D5FE09C0EC01219649EB58E066ECB3
:1044400074E00E94980FCE01D6FE09C0EC012196BF
:1044500049EB58E06EEC74E00E94980FCE01B70172
:10446000A60144275078452B462B472B61F049EB9A
:1044700058E069ED74E0DF91CF91FF90EF90DF900D
:10448000CF900C94980FCD28CE28CF2841F487EEFA
:1044900096E09F938F930E94118B0F900F90DF9166
:1044A000CF91FF90EF90DF90CF9008950F931F93DF
:1044B000CF93DF938C01C0E0D0E00115110509F422
:1044C0008AC062EE76E0C8010E944C8A892B09F40A
:1044D000C1606AED76E0C8010E944C8A892B09F41C
:1044E000C26062ED76E0C8010E944C8A892B09F413
:1044F000C4606EEC76E0C8010E944C8A892B09F4F6
:10450000C8606BEC76E0C8010E944C8A892B09F4E4
:10451000C06167EC76E0C8010E944C8A892B09F4DF
:10452000C06261EC76E0C8010E944C8A892B09F4D4
:10453000C06469EB76E0C8010E944C8A892B09F4BB
:10454000C06861EB76E0C8010E944C8A892B09F4AF
:10455000D1606DEA76E0C8010E944C8A892B09F48B
:10456000D26067EA76E0C8010E944C8A892B09F480
:10457000D46062EA76E0C8010E944C8A892B09F473
:10458000D8606CE976E0C8010E944C8A892B09F456
:10459000D06164E976E0C8010E944C8A892B09F455
:1045A000D06269E876E0C8010E944C8A892B09F440
:1045B000D06468E776E0C8010E944C8A892B09F430
:1045C000D06860916A0270916B0280E090E00E9476
:1045D000608A8C0172CFCE01DF91CF911F910F9134
:1045E0000895AF92BF92CF92DF92EF92FF920F9316
:1045F0001F93CF93DF93F22E032F142FE52E5B0131
:104600006C01217030E040E050E060E070E080E05C
:1046100090E0A0E00E949A8689F0EAEEF4E0FF9331
:10462000EF93EAE9FDE0FF93EF930E94118B0F9067
:104630000F900F900F90E1E0F0E002C0E0E0F0E0BA
:1046400080918F1F80FF17C02F2D247030E040E035
:1046500050E060E070E080E090E0A0E00E949A8688
:1046600051F0EF01219649EB58E06EEE74E0CF0176
:104670000E94980FFE012F2D227030E040E050E0A4
:1046800060E070E080E090E0A0E00E949A8651F047
:10469000EF01219649EB58E062EF74E0CF010E94F0
:1046A000980FFE012F2D287030E040E050E060E0D0
:1046B00070E080E090E0A0E00E949A8651F0EF0167
:1046C000219649EB58E06AE075E0CF010E94980F0F
:1046D000FE012F2D207130E040E050E060E070E0FE
:1046E00080E090E0A0E00E949A8651F0EF012196D0
:1046F00049EB58E065EF74E0CF010E94980FFE018E
:104700002F2D207230E040E050E060E070E080E06B
:1047100090E0A0E00E949A8651F0EF01219649EBCB
:1047200058E068EF74E0CF010E94980FFE012F2D32
:10473000207430E040E050E060E070E080E090E025
:10474000A0E00E949A8651F0EF01219649EB58E0D3
:104750006EEF74E0CF010E94980FFE012F2D20789C
:1047600030E040E050E060E070E080E090E0A0E009
:104770000E949A8651F0EF01219649EB58E064E0DF
:1047800075E0CF010E94980FFE0120E0302F3170BC
:1047900040E050E060E070E080E090E0A0E00E9447
:1047A0009A8651F0EF01219649EB58E067E075E0F9
:1047B000CF010E94980FFE0120E0302F327040E0C0
:1047C00050E060E070E080E090E0A0E00E949A8617
:1047D00051F0EF01219649EB58E06CE075E0CF0114
:1047E0000E94980FFE0120E0302F347040E050E02E
:1047F00060E070E080E090E0A0E00E949A8651F0D6
:10480000EF01219649EB58E063E175E0CF010E948A
:10481000980FFE0120E0302F387040E050E060E05B
:1048200070E080E090E0A0E00E949A8651F0EF01F5
:10483000219649EB58E066E175E0CF010E94980FA0
:10484000FE0120E0302F307140E050E060E070E089
:1048500080E090E0A0E00E949A8651F0EF0121965E
:1048600049EB58E06BE175E0CF010E94980FFE0123
:1048700020E0302F307240E050E060E070E080E0F7
:1048800090E0A0E00E949A8651F0EF01219649EB5A
:1048900058E062E275E0CF010E94980FFE0180911E
:1048A0008F1F81FF17C020E0302F307440E050E0B0
:1048B00060E070E080E090E0A0E00E949A8651F015
:1048C000EF01219649EB58E069E275E0CF010E94C3
:1048D000980FFE0180918F1F9091901F90FF17C03D
:1048E00020E030E040E05E2D507160E070E080E05C
:1048F00090E0A0E00E949A8651F0EF01219649EBEA
:1049000058E06CE275E0CF010E94980FFE018091A3
:104910008F1F9091901F90FF17C020E030E040E083
:104920005E2D507260E070E080E090E0A0E00E94B8
:104930009A8651F0EF01219649EB58E06FE275E05D
:10494000CF010E94980FFE0180918F1F9091901FC0
:1049500090FF17C020E030E040E05E2D507460E032
:1049600070E080E090E0A0E00E949A8651F0EF01B4
:10497000219649EB58E065E375E0CF010E94980F5E
:10498000FE0120E0302F307840E050E060E070E041
:1049900080E090E0A0E00E949A8651F0EF0121961D
:1049A00049EB58E060E475E0CF010E94980FFE01EA
:1049B00020E030E0412F417050E060E070E080E0A6
:1049C00090E0A0E00E949A8651F0EF01219649EB19
:1049D00058E065E475E0CF010E94980FFE0120E0E9
:1049E00030E0412F427050E060E070E080E090E005
:1049F000A0E00E949A8651F0EF01219649EB58E021
:104A000068E475E0CF010E94980FFE0120E030E0DD
:104A1000412F447050E060E070E080E090E0A0E062
:104A20000E949A8651F0EF01219649EB58E06BE421
:104A300075E0CF010E94980FFE0180918F1F87FFC4
:104A400017C020E030E0412F487050E060E070E097
:104A500080E090E0A0E00E949A8651F0EF0121965C
:104A600049EB58E06EE475E0CF010E94980FFE011B
:104A700080918F1F87FF17C020E030E0412F4071E9
:104A800050E060E070E080E090E0A0E00E949A8654
:104A900051F0EF01219649EB58E062E575E0CF0156
:104AA0000E94980FFE0180918F1F87FF17C020E0A2
:104AB00030E0412F407250E060E070E080E090E034
:104AC000A0E00E949A8651F0EF01219649EB58E050
:104AD00066E575E0CF010E94980FFE0180918F1F5F
:104AE00087FF17C020E030E0412F407450E060E0C5
:104AF00070E080E090E0A0E00E949A8651F0EF0123
:104B0000219649EB58E06AE575E0CF010E94980FC5
:104B1000FE0180918F1F82FF17C020E030E0412FFF
:104B2000407850E060E070E080E090E0A0E00E941B
:104B30009A8651F0EF01219649EB58E069E176E061
:104B4000CF010E94980FFE0180918F1F82FF17C036
:104B500020E030E040E05E2D517060E070E080E0E9
:104B600090E0A0E00E949A8651F0EF01219649EB77
:104B700058E06EE575E0CF010E94980FFE0180912C
:104B80008F1F9091901F90FF17C020E030E040E011
:104B90005E2D527060E070E080E090E0A0E00E9446
:104BA0009A8651F0EF01219649EB58E061E675E0F5
:104BB000CF010E94980FFE0180918F1F9091901F4E
:104BC00090FF17C020E030E040E05E2D547060E0C0
:104BD00070E080E090E0A0E00E949A8651F0EF0142
:104BE000219649EB58E069E675E0CF010E94980FE5
:104BF000FE0180918F1F9091901F91FF1EC020E0B9
:104C000030E040E05E2D587060E070E080E090E0C1
:104C1000A0E00E949A8689F049EB58E062E775E0CF
:104C2000CF01DF91CF911F910F91FF90EF90DF9017
:104C3000CF90BF90AF900C94980F2F2D302F412F15
:104C40005E2DB501C601A0E00E949A8641F483E77B
:104C500096E09F938F930E94118B0F900F90DF919E
:104C6000CF911F910F91FF90EF90DF90CF90BF9069
:104C7000AF900895AF92BF92DF92EF920F931F9380
:104C8000CF93DF93EC015B01FB0110826EE676E0CF
:104C90000E944C8A892B59F580918F1F7DE4D72E75
:104CA000E0E8EE2E82FD02C004E001C004E810E05E
:104CB00081FF02C060ECE62E26E04AE250E06BE2A3
:104CC00070E089E290E00E943F5581E090E00E9410
:104CD000CC0A882311F05DE5D52E80918F1F90912D
:104CE000901F90FD16E091FF06C0186004C0D12C03
:104CF000E12C00E010E06CE676E0CE010E944C8AE8
:104D0000892B61F481E0F501808360916A027091E2
:104D10006B0280E090E00E94608AEC016AE676E037
:104D2000CE010E944C8A892B61F48FEFF5018083BC
:104D300060916A0270916B0280E090E00E94608A4C
:104D4000EC01209709F41AC166E676E0CE010E94D4
:104D50004C8A892B19F4FD2DF160DF2E62E676E096
:104D6000CE010E944C8A892B19F48D2D8460D82E97
:104D70006FE576E0CE010E944C8A892B19F4ED2D67
:104D8000E260DE2E6DE576E0CE010E944C8A892B32
:104D900019F4FD2DF860DF2E6AE576E0CE010E9461
:104DA0004C8A892B19F48D2D8061D82E64E576E02C
:104DB000CE010E944C8A892B19F4ED2DE062DE2E83
:104DC0006EE476E0CE010E944C8A892B19F4FD2D09
:104DD000F064DF2E6BE476E0CE010E944C8A892BD2
:104DE00019F48D2D8068D82E66E476E0CE010E94FD
:104DF0004C8A892B19F4EE2DE160EE2E6FE376E0FC
:104E0000CE010E944C8A892B19F4FE2DF260EF2E00
:104E10006CE376E0CE010E944C8A892B19F48E2D2A
:104E20008460E82E67E376E0CE010E944C8A892BED
:104E300019F4EE2DE860EE2E60E376E0CE010E94DC
:104E40004C8A892B19F4FE2DF061EF2E69E276E091
:104E5000CE010E944C8A892B19F48E2D8062E82E97
:104E600066E276E0CE010E944C8A892B19F4EE2D81
:104E7000E064EE2E61E276E0CE010E944C8A892B3E
:104E800019F4FE2DF068EF2E6EE176E0CE010E945F
:104E90004C8A892B09F401606BE176E0CE010E9417
:104EA0004C8A892B09F4026068E176E0CE010E9409
:104EB0004C8A892B09F4046064E176E0CE010E94FB
:104EC0004C8A892B09F4086060E176E0CE010E94EB
:104ED0004C8A892B09F400616CE076E0CE010E94D7
:104EE0004C8A892B09F4006268E076E0CE010E94CA
:104EF0004C8A892B09F4006466E076E0CE010E94BA
:104F00004C8A892B09F4006863E076E0CE010E94A8
:104F10004C8A892B09F411606BEF75E0CE010E9479
:104F20004C8A892B09F4126062EF75E0CE010E9471
:104F30004C8A892B09F4146069EE75E0CE010E9459
:104F40004C8A892B09F4186066EE75E0CE010E9448
:104F50004C8A892B09F4106160EE75E0CE010E9445
:104F60004C8A892B09F4106265ED75E0CE010E9430
:104F70004C8A892B09F0DCCE1064DACE2D2D3E2D23
:104F8000A80160E070E080E090E0DF91CF911F9198
:104F90000F91EF90DF90BF90AF900895CF9385EC85
:104FA00095E09F938F930E94118B0E945A1F84EA71
:104FB0009AE19F938F938DEB95E09F938F930E943F
:104FC000118B89EB95E09F938F930E94118B80E06A
:104FD0000E94382184EB95E09F938F930E94118B60
:104FE0000E94C00F80918F1F2DB73EB7265F3F4FA5
:104FF0000FB6F8943EBF0FBE2DBF80FF05C041E045
:1050000061E081E00E946A110E945E1F8091490266
:105010001F928F938BEA95E09F938F930E94118B41
:10502000809157091F928F9382EA95E09F938F9307
:105030000E94118BC0E4CF9383E18F9383E38F931E
:105040008F938EE895E09F938F930E94118B1F9210
:10505000CF9386E795E09F938F930E94118B809169
:1050600013281F928F93809112281F928F9383E6AB
:1050700095E09F938F930E94118B809148021F921D
:105080008F938AE595E09F938F930E94118B809177
:105090004A0290914B022DB73EB7245E3F4F0FB6A8
:1050A000F8943EBF0FBE2DBF96FF03C08BE795E07F
:1050B00002C08EE795E09F938F9380E595E09F93E4
:1050C0008F930E94118B809151028F938091500297
:1050D0008F938BE395E09F938F930E94118B83E3D3
:1050E00095E09F938F930E94118B209152023091F3
:1050F00053024091540250915502609156027091B2
:10510000570280915802909159020E94F1220E9408
:105110003E0B8DB79EB70A960FB6F8949EBF0FBE92
:105120008DBF1D9B03C08BE795E002C08EE795E025
:105130009F938F9387E295E09F938F930E94118BAB
:105140008DE195E09F938F930E94118B80914A028D
:105150000F900F900F900F900F900F9081FF09C04C
:1051600087E195E09F938F930E94118B0F900F9092
:1051700013C080FF03C08BE795E002C08EE795E087
:105180009F938F9383E195E09F938F930E94118B60
:105190000F900F900F900F908CE095E09F938F935E
:1051A0000E94118B60915B0970915C0980E090E036
:1051B0000E9468210E943E0B0F900F90779903C0C8
:1051C0008BE795E002C08EE795E09F938F9383E095
:1051D00095E09F938F930E94118B0E94DB08609152
:1051E00052027091530280915402909155020E9494
:1051F0007E0A0E94380A9F938F937F936F9385EF67
:1052000094E09F938F930E94118B81E090E00E9425
:1052100014208091ED279091EE27A091EF27B09177
:10522000F027BF93AF939F938F9387EE94E09F9364
:105230008F930E94118B8091FD278F938091FC2783
:105240008F938091FB278F938091FA278F9383ED23
:1052500094E09F938F930E94118B8091F1279091FE
:10526000F227A091F327B091F427BF93AF939F93B8
:105270008F9385EC94E09F938F930E94118B809184
:1052800001288F93809100288F938091FF278F931F
:105290008091FE278F9381EB94E09F938F930E94E0
:1052A000118B2DB73EB72E5D3F4F0FB6F8943EBF22
:1052B0000FBE2DBF61E070E080E090E00E94470BE0
:1052C00061E070E081E090E0CF910C94470BF8949E
:1052D000E0E0F0E081E2809357008491E2E0F0E0CA
:1052E00041E2409357004491E4E0F0E091E2909372
:1052F0005700E49190E0A0E0B0E0DC019927882716
:1053000050E060E070E0762F652F542F4427840F23
:10531000951FA61FB71F8E0F911DA11DB11D809354
:105320003A1B90933B1BA0933C1BB0933D1B78947E
:105330000895DF92EF92FF920F931F93CF93DF9325
:10534000CDB7DEB769970FB6F894DEBF0FBECDBFFD
:1053500048E050E06AE170E0CE010B960E94368C86
:10536000DB84EC84FD840E851F85B889F989EA8980
:105370002D2D3E2D4F2D502F612F7B2F8F2F9E2FA8
:10538000AFEF0E949A8649F448E050E06AE170E08D
:1053900082E592E00E94548C10C0D0925202E092BA
:1053A0005302F09254020093550210935602B093A8
:1053B0005702F0935802E093590242E050E068E14E
:1053C00070E0CE0147960E94368C8F89988D8F3F72
:1053D0002FEF920779F48CE390E090935102809341
:1053E000500242E050E068E170E080E592E00E9407
:1053F000548C04C0909351028093500242E050E0DC
:1054000066E170E0CE0147960E94368C8F89988DB8
:105410008F3F2FEF920779F48AE090E490934B024C
:1054200080934A0242E050E066E170E08AE492E054
:105430000E94548C04C090934B0280934A0242E035
:1054400050E06EE270E0CE0147960E94368C8F8964
:10545000988D8F3F2FEF920769F410925C0910929C
:105460005B0942E050E06EE270E08BE599E00E945B
:10547000548C04C090935C0980935B0949E050E030
:105480006AE070E082E098E20E94368C0E947F0C15
:1054900044E050E066E270E0CE0143960E94368C14
:1054A0008B899C89AD89BE8944E050E066E270E05A
:1054B0008F3F9F4FAF4FBF4F29F481E792E00E948B
:1054C000548C04C081E792E00E94368C44E050E0A6
:1054D00062E270E0CE0143960E94368C8B899C89F3
:1054E000AD89BE8944E050E062E270E08F3F9F4F9B
:1054F000AF4FBF4F29F48DE692E00E94548C04C058
:105500008DE692E00E94368C44E050E06AE270E062
:10551000CE0143960E94368C8B899C89AD89BE89C9
:1055200044E050E06AE270E08F3F9F4FAF4FBF4FC3
:1055300029F485E792E00E94548C04C085E792E04C
:105540000E94368C41E050E065E170E0CE01499662
:105550000E94368C898D41E050E065E170E08F3F1C
:1055600029F487E599E00E94548C04C087E599E00E
:105570000E94368C41E050E064E170E0CE01499633
:105580000E94368C898D41E050E064E170E08F3FED
:1055900029F489E492E00E94548C04C089E492E0EA
:1055A0000E94368C41E050E063E170E0CE01499604
:1055B0000E94368C898D41E050E063E170E08F3FBE
:1055C00029F488E492E00E94548C04C088E492E0BC
:1055D0000E94368C4AE050E060E070E0CE01019617
:1055E0000E94368C89814AE050E060E070E08F3F95
:1055F00029F484EA9AE10E94548C04C084EA9AE176
:105600000E94368C69960FB6F894DEBF0FBECDBFF0
:10561000DF91CF911F910F91FF90EF90DF90089550
:10562000CF92DF92EF92FF9260916A0270916B02CB
:1056300080E090E00E94608A62E875E00E94748ACF
:10564000892B09F0C0C08DE48093520280E88093DA
:10565000530284E080935402109255021092560235
:1056600010925702109258021092590248E050E0EE
:105670006AE170E082E592E00E94548C8CE390E055
:10568000909351028093500242E050E068E170E054
:1056900080E592E00E94548C8AE090E490934B0263
:1056A00080934A0242E050E066E170E08AE492E0D2
:1056B0000E94548C10925C0910925B0942E050E009
:1056C0006EE270E08BE599E00E94548C32E2C32ECA
:1056D000DD24DA943CECE32E3BE3F32EC09271021E
:1056E000D0927202E0927302F092740244E050E0B1
:1056F00066E270E081E792E00E94548CC0926D02F5
:10570000D0926E02E0926F02F092700244E050E09C
:1057100062E270E08DE692E00E94548C87ED94E3A3
:10572000AFEEBCE38093750290937602A09377026C
:10573000B093780244E050E06AE270E085E792E0DE
:105740000E94548C1092570980E090E00E94AB6256
:1057500041E050E065E170E087E599E00E94548CFB
:105760008AE1809349028AE190E00E94526141E01F
:1057700050E064E170E089E492E00E94548C8FE094
:105780008093480241E050E063E170E088E492E0F9
:105790000E94548C8AE0E4EAFAE1DF011D928A95C6
:1057A000E9F74AE050E060E070E0CF010E94548CDD
:1057B00081E00E94382180E090E0FF90EF90DF9040
:1057C000CF900C94930CFF90EF90DF90CF900895C2
:1057D0002F923F924F925F926F927F928F929F9201
:1057E000AF92BF92CF92DF92EF92FF920F931F93EF
:1057F000CF93DF93CDB7DEB727970FB6F894DEBF10
:105800000FBECDBF9F838E83FC0180819181892B48
:1058100011F00C94263C60916A0270916B028DEA43
:1058200093E20E94608A60E470E08DEA93E20E9455
:10583000938A009759F46091CD307091CE308AE010
:1058400090E00E94CD8A81E00C942B3C8130910540
:1058500049F42090AD23312C412C512C612C712C1A
:105860004301BDC082309105A1F48091AD23209108
:10587000AE2390E0982F8827820F911D1C01892F5D
:10588000880F880B482E582E682E782E882E982E3A
:10589000A6C083309105D1F52091AD231091AE23A0
:1058A000E091AF2330E040E050E060E070E080E065
:1058B00090E000E10E943C86522E632E742E852ECD
:1058C000962EB72FA82FF92F212F30E040E050E07F
:1058D00060E070E080E090E008E00E943C865901C2
:1058E0006A017B018C01252D362D472D582D692D00
:1058F0007B2F8A2F9F2F0E947386AE2EB12CC12C36
:10590000D12CE12CF12C00E010E059C004970CF4EC
:105910005DC02091AD231091AE23E091AF23F091B3
:10592000B02330E040E050E060E070E080E090E0E4
:1059300008E10E943C8629013A014B01B82FA92FAA
:10594000212F30E040E050E060E070E080E090E047
:1059500000E10E943C8659016A017B018C019201A1
:10596000A301B4018B2F9A2F0E947386AF2EB12C06
:10597000C12CD12CE12CF12C00E010E00E947386A8
:10598000522E632E742E852E962EB72FA82FF92F08
:105990002E2F30E040E050E060E070E080E090E0EA
:1059A00008E00E943C8659016A017B018C01252D8B
:1059B000362D472D582D692D7B2F8A2F9F2F0E9422
:1059C000738619012A013B014C0109C06AE0262EA9
:1059D000312C412C512C612C712C812C912C0E944A
:1059E0003E0B9101A201B301C4012736FFE63F0738
:1059F000FCE64F075105610571058105910511F41C
:105A00000C9476362736EFE63E07ECE64E07510556
:105A1000610571058105910511F008F075C1293600
:105A2000F2E73F07410551056105710581059105C3
:105A300011F40C946E392936E2E73E074105510511
:105A4000610571058105910511F008F097C02536B3
:105A5000F4E63F0741055105610571058105910592
:105A600009F42FC52536E4E63E07410551056105D9
:105A700071058105910509F088F5A6E70E949A86CF
:105A800009F4D6C60E949A8609F060F4A8E60E943E
:105A90009A8609F45CC5A5E70E949A8609F4B2C605
:105AA0000C94243C9101A201B301C4012A33F6E213
:105AB0003F0741055105610571058105910509F40F
:105AC000CBC224363146410551056105710581057A
:105AD000910511F40C94DD390C94243C9101A20140
:105AE000B301C4012737FFE63F07410551056105B2
:105AF00071058105910511F40C9493372737EFE672
:105B00003E0741055105610571058105910509F0C3
:105B1000C0F42436F9E63F074105510561057105DA
:105B20008105910509F447C625363E4641055105D4
:105B3000610571058105910511F40C94C7370C942A
:105B4000243C9101A201B301C4012333F1E73F07D3
:105B500041055105610571058105910511F40C940C
:105B6000DD3925363247410551056105710581054D
:105B7000910511F40C9481380C94243C9101A201FC
:105B8000B301C4012236F5E63F07F4E64F0751059D
:105B9000610571058105910509F493C42236E5E696
:105BA0003E07E4E64E075105610571058105910543
:105BB00011F008F051C02133F4E63F07F1E64F073A
:105BC0005105610571058105910509F463C2213311
:105BD000E4E63E07E1E64E075105610571058105E2
:105BE000910509F0C8F42337F2E73F074105510555
:105BF000610571058105910511F40C94B5392337C0
:105C0000334741055105610571058105910511F481
:105C10000C94C9390C94243C9101A201B301C40134
:105C20002336F4E63F07F1E64F075105610571059C
:105C30008105910511F40C94DD392837344641462D
:105C40005105610571058105910511F00C94243C05
:105C50000E944E150C94263C9101A201B301C4018F
:105C60002D36F5E73F07F8E64F0751056105710549
:105C70008105910511F40C94F3392D36E5E73E07C3
:105C8000E8E64E075105610571058105910509F0AA
:105C9000E0F42237F2E73F07F5E64F0751056105CB
:105CA00071058105910511F40C94F83623363D46B3
:105CB00048465105610571058105910511F00C9467
:105CC000243C0E94C6150C94263C9101A201B3010C
:105CD000C4012336F2E33F07F9E64F07510561059A
:105CE00071058105910509F4F5C1243633464C460A
:105CF0005105610571058105910511F00C94243C55
:105D00000E94A0590C94263C9101A201B301C40148
:105D10002037FCE63F07F5E64F07F8E65F07610529
:105D200071058105910509F412C42037ECE63E07A0
:105D3000E5E64E07E8E65E07610571058105910518
:105D400011F008F0C1C02437F8E73F07F4E74F0728
:105D50005105610571058105910509F4D4C5243704
:105D6000E8E73E07E4E74E07510561057105810547
:105D7000910511F008F051C02133F1E33F07F1E73D
:105D80004F075105610571058105910511F40C94CA
:105D90002D372133E1E33E07E1E74E075105610569
:105DA00071058105910509F0D0F42537F3E63F0729
:105DB000FDE64F075105610571058105910511F457
:105DC0000C942D372033314341475105610571054E
:105DD0008105910511F40C94F8360C94243C910142
:105DE000A201B301C4012037F5E63F07F2E74F07F0
:105DF0005105610571058105910511F40C948138F7
:105E00002C363447444751056105710581059105DC
:105E100011F40C94613B0C94243C9101A201B30158
:105E2000C4012936FCE63F07F1E64F07F3E65F07BA
:105E3000610571058105910509F481C12936ECE6FA
:105E40003E07E1E64E07E3E65E0761057105810561
:105E5000910509F0E0F42437F4E63F07F7E74F0730
:105E60005105610571058105910511F40C94AF3B55
:105E700024373F464F46524661057105810591051D
:105E800011F00C94243C0C9400000C94263C9101DD
:105E9000A201B301C4012E36F1E63F07F8E64F0731
:105EA000F3E65F07610571058105910509F400C5F9
:105EB00026333946454755466105710581059105EB
:105EC00009F449C30C94243C9101A201B301C4011B
:105ED0002437F3E73F07F5E64F07F2E75F07610571
:105EE00071058105910511F40C9441382437E3E7DD
:105EF0003E07E5E64E07E2E75E07610571058105AD
:105F0000910511F008F053C02337F5E63F07F2E79B
:105F10004F07F0E75F07610571058105910511F4F1
:105F20000C94A33A2337E5E63E07E2E74E07E0E7A5
:105F30005E07610571058105910509F0D0F42136F0
:105F4000FDE63F07F5E74F07F8E65F0761057105D6
:105F50008105910511F40C94B1372237374740473A
:105F60005047610571058105910509F4B7C00C948E
:105F7000243C9101A201B301C4012337F2E73F079A
:105F8000F7E74F07F0E75F076105710581059105A8
:105F900011F40C94443821363C464546524761057D
:105FA00071058105910509F4F3C20C94243C91011B
:105FB000A201B301C4012437F2E73F07F1E64F071E
:105FC000F5E75F07610571058105910509F469C36E
:105FD0002437E2E73E07E1E64E07E5E75E076105A5
:105FE00071058105910509F0C8F42437F3E73F07EF
:105FF000F5E64F07F4E75F07610571058105910537
:1060000009F4AAC42737304748475447610571054A
:106010008105910509F422C40C94243C9101A2014C
:10602000B301C4012237F7E63F07F0E74F07F5E772
:106030005F07610571058105910509F434C62C36A9
:10604000314644475847610571058105910511F4B2
:106050000C942B3B0C94243C84E08093A22385E099
:106060008093A3231092A4231092A5231092A62319
:1060700081E08093A7231092A8231092A923109265
:10608000AA2342EA53E262E18AE292E00E94C44C0F
:106090000C94263C21E04CE061E080ED0E94EF5939
:1060A00021E04EE061E080ED0E94EF5921E040E107
:1060B00061E080ED0E94EF5921E042E161E080ED76
:1060C0000E94EF5922E040E161E080ED0E94EF592B
:1060D0000C94263C0E94C00F0C94263C60916A02EE
:1060E00070916B0280E090E00E94608A8C016BE707
:1060F00075E00E94748A892B19F477980C94263CD9
:106100006EE775E0C8010E94748A892B19F4779AAA
:106110000C94263C779903C08BE795E002C08EE78C
:1061200095E09F938F938BE994E09F938F930E94C8
:10613000118B0F900F900F900F900C94263C609154
:106140006A0270916B0280E090E00E94608A8C018C
:1061500065E475E00E94748A892B09F077C060912C
:106160006A0270916B0280E090E00E94608A8C016C
:10617000009711F40C94263C69E875E00E94748A3B
:10618000892BB1F482E29FEFACECBBE38093710208
:1061900090937202A0937302B093740244E050E0B3
:1061A00066E270E081E792E00E94548C0C94263CF9
:1061B0006FE875E0C8010E94748A892BB1F482E20D
:1061C0009FEFACECBAE38093710290937202A093BC
:1061D0007302B093740244E050E066E270E081E73D
:1061E00092E00E94548C0C94263CC8010E944A897B
:1061F0002B013C0120E030E0A9010E94E9808823C6
:10620000D9F081E00E94D5099B01AC01C301B20124
:106210000E94ED806093710270937202809373020A
:106220009093740244E050E066E270E081E792E00F
:106230000E94548C0C94263C84ED92E09F938F93A3
:106240000E94118B0F900F900C94263C68E475E02F
:10625000C8010E94748A892B09F077C060916A0294
:1062600070916B0280E090E00E94608A8C01009740
:1062700011F40C94263C69E875E00E94748A892B1D
:10628000B1F482E29FEFACECBBE380936D0290939C
:106290006E02A0936F02B093700244E050E062E29D
:1062A00070E08DE692E00E94548C0C94263C6FE8DE
:1062B00075E0C8010E94748A892BB1F482E29FEFD5
:1062C000ACECBAE380936D0290936E02A0936F02E0
:1062D000B093700244E050E062E270E08DE692E03C
:1062E0000E94548C0C94263CC8010E944A892B01C0
:1062F0003C0120E030E0A9010E94E9808823D9F028
:1063000082E00E94D5099B01AC01C301B2010E9449
:10631000ED8060936D0270936E0280936F02909394
:10632000700244E050E062E270E08DE692E00E948C
:10633000548C0C94263C87EC92E09F938F930E94A0
:10634000118B0F900F900C94263C60E475E0C8010F
:106350000E94748A892B09F073C060916A0270915F
:106360006B0280E090E00E94608A8C01009711F43B
:106370000C94263C69E875E00E94748A892BB1F47C
:1063800087ED94E3AFEEBCE38093750290937602C1
:10639000A0937702B093780244E050E06AE270E0A4
:1063A00085E792E00E94548C0C94263C6FE875E0DF
:1063B000C8010E94748A892B51F488EB92E09F9364
:1063C0008F930E94118B0F900F900C94263CC80164
:1063D0000E944A892B013C0120E030E0A9010E9483
:1063E000E980882319F180E00E94D5094B015C0106
:1063F00021EE3AE744E95EE3C301B2010E94228044
:10640000A50194010E94ED8060937502709376025D
:10641000809377029093780244E050E06AE270E063
:1064200085E792E00E94548C0C94263C8BEA92E023
:106430009F938F930E94118B0F900F900C94263C8A
:106440000E94240A9F938F937F936F9384EA92E034
:106450009F938F930E94118B82E00E94D509209117
:106460006D0230916E0240916F02509170020E9455
:106470006A83162F072FF82EE92E81E00E94D50996
:10648000EF92FF920F931F9320917102309172024D
:1064900040917302509174020E946A839F938F937C
:1064A0007F936F9388E992E09F938F930E94118B63
:1064B0000E943E0B0FB6F894DEBF0FBECDBF0C940A
:1064C000263C60916A0270916B0280E090E00E942D
:1064D000608A0097C1F00E94562220915B0930919A
:1064E0005C098217930709F190935C0980935B091B
:1064F00042E050E06EE270E08BE599E00E94548C3F
:1065000084E994E002C08DE894E09F938F930E9409
:10651000118B60915B0970915C0980E090E00E94B2
:1065200068210E943E0B0F900F9082E894E09F93A9
:106530008F930E94118B6FEF7FEF80E090E00E94BD
:1065400068210E943E0B0F900F900C94263C0E94F5
:106550007B1E0C94263C8091B123843329F440E0C7
:1065600061E080E00E946A1180916C02882311F43E
:106570000C94263C1F928F938FE794E09F938F9308
:106580000E94118B0F900F900F900F900C94263C4F
:106590008091B123893709F070C060916A027091CF
:1065A0006B0280E090E00E94608A8C016BE775E0EE
:1065B0000E94748A892B31F480914A0290914B0297
:1065C00090640CC06EE775E0C8010E94748A892B44
:1065D00091F480914A0290914B029F7B90934B02E1
:1065E00080934A0242E050E066E170E08AE492E083
:1065F0000E94548C42C064E975E0C8010E94748A0C
:10660000892B21F58091C01A8F938091BF1A8F93A7
:106610008091BE1A8F938091BD1A8F938091BC1A7E
:106620008F938091BB1A8F938091BA1A8F93809128
:10663000B91A8F938DE692E09F938F930E94118BEE
:106640000FB6F894DEBF0FBECDBF17C080914A02CF
:1066500090914B0296FF03C08BE795E002C08EE756
:1066600095E09F938F9389E692E09F938F930E948A
:10667000118B0F900F900F900F9080916C028823D8
:1066800011F40C94263C1F928F938CE794E09F9317
:106690008F930E94118B0F900F900F900F900C947E
:1066A000263C60916A0270916B0280E090E00E944B
:1066B000608A5C016AE975E00E94748A892B11F492
:1066C00089E108C06EE975E0C5010E94748A892BD2
:1066D00049F480E18093C4001092C50082E0809369
:1066E000C00055C062EA75E0C5010E94748A892B1A
:1066F00011F488E0EFCF67EA75E0C5010E94748A63
:10670000892B39F06CEA75E0C5010E94748A892BE7
:1067100011F483E0DFCF8091C400893141F484E635
:1067200092E09F938F930E94118B0F900F90809116
:10673000C400803141F48FE592E09F938F930E94D3
:10674000118B0F900F908091C400883041F489E53F
:1067500092E09F938F930E94118B0F900F908091E6
:10676000C400833041F483E592E09F938F930E94AD
:10677000118B0F900F908091C400883041F48DE40C
:1067800092E09F938F930E94118B0F900F908091B6
:106790006C02882311F40C94263C1F928F9389E796
:1067A00094E09F938F930E94118B0F900F900F9006
:1067B0000F900C94263C60916A0270916B0280E00D
:1067C00090E00E94608A69E875E00E94748A892BD3
:1067D00011F481E001C080E00E94382180916C02B8
:1067E000882311F40C94263C1F928F9386E794E043
:1067F0009F938F930E94118B0F900F900F900F908B
:106800000C94263C0E945E1F80916C02882311F438
:106810000C94263C1F928F9383E794E09F938F9371
:106820000E94118B0F900F900F900F900C94263CAC
:106830000E945A1F80916C02882311F40C94263C0C
:106840001F928F9380E794E09F938F930E94118B08
:106850000F900F900F900F900C94263C60916A025D
:1068600070916B0280E090E00E94608A0E944E89E5
:10687000803178F48093570999270E94AB6241E0F8
:1068800050E065E170E087E599E00E94548C0C943B
:10689000263C809157091F928F9383E492E09F9347
:1068A0008F930E94118B0F900F900F900F90CEC777
:1068B00060916A0270916B0280E090E00E94608AB1
:1068C0000E944E8925EF280F203170F480934902F1
:1068D00099270E94526141E050E064E170E089E450
:1068E00092E00E94548CB2C7809149021F928F930C
:1068F0008AE392E09F938F930E94118B0F900F90E9
:106900000F900F90A3C760916A0270916B0280E0B4
:1069100090E00E94608A009781F04AE050E0BC015C
:1069200084EA9AE10E94848A4AE050E060E070E0E4
:1069300084EA9AE10E94548C89C784EA9AE19F9381
:106940008F9381EB95E09F938F930E94FF8A0F9026
:106950000F900F900F907AC760916A0270916B024E
:1069600080E090E00E94608A5C0161ED73E00E942B
:10697000748A892B99F4219A80914A0290914B0252
:10698000806190934B0280934A0242E050E066E1BE
:1069900070E08AE492E00E94548C58C769E475E084
:1069A000C5010E94748A892B99F4229A80914A0227
:1069B00090914B02806290934B0280934A0242E096
:1069C00050E066E170E08AE492E00E94548C3EC799
:1069D00063EB73E0C5010E94748A892B99F4239AB2
:1069E00080914A0290914B02806490934B02809375
:1069F0004A0242E050E066E170E08AE492E00E94E0
:106A0000548C24C760EF74E0C5010E94748A892BFE
:106A100099F4239A80914A0290914B028068909356
:106A20004B0280934A0242E050E066E170E08AE463
:106A300092E00E94548C0AC762E079E0C5010E948E
:106A4000748A892B09F040C081E08093A223809151
:106A500052028093A323809153028093A4238091B8
:106A600054028093A523809155028093A6238091A0
:106A700056028093A723809157028093A823809188
:106A800058028093A923809159028093AA231092DF
:106A9000AC231092AB2380914A0290914B029160FB
:106AA00090934B0280934A0242E050E066E170E02E
:106AB0008AE492E00E94548C42EA53E262E18AE264
:106AC00092E00E94C44CC2C66AED73E0C5010E9408
:106AD000748A892BD1F4E9ECFAE1119211929AE1CE
:106AE000E93EF907D1F780914A0290914B029260FA
:106AF00090934B0280934A0242E050E066E170E0DE
:106B00008AE492E00E94548CA1C66EE775E0C5014C
:106B10000E94748A20914A0230914B02892BA9F479
:106B20002F703C7F30934B0220934A022B9A42E015
:106B300050E066E170E08AE492E00E94548C80911B
:106B4000F92790E00E94676181C624FF03C08BE7AC
:106B500095E002C08EE795E09F938F938FE292E0DD
:106B60009F938F930E94118B80914A020F900F90F8
:106B70000F900F9085FF03C08BE795E002C08EE772
:106B800095E09F938F9384E292E09F938F930E946E
:106B9000118B80914A020F900F900F900F9086FFFB
:106BA00003C08BE795E002C08EE795E09F938F933B
:106BB00089E192E09F938F930E94118B80914A020A
:106BC0000F900F900F900F9087FF03C08BE795E019
:106BD00002C08EE795E09F938F938EE092E09F93A3
:106BE0008F930E94118B80914A0290914B020F90DB
:106BF0000F900F900F9090FF03C08BE795E002C0BD
:106C00008EE795E09F938F9383E092E09F938F931D
:106C10000E94118B80914A0290914B020F900F902D
:106C20000F900F9091FF03C08BE795E002C08EE7B5
:106C300095E09F938F9388EF91E09F938F930E94AD
:106C4000118B80914A0290914B020F900F900F9000
:106C50000F9091FFFBC589EB95E00E94358B49ECC5
:106C6000A42E4AE1B42E0BE010E051EC852E55E045
:106C7000952EF50180819181F2E0AF0EB11C9F93BA
:106C80008F931F930F939F928F920E94FF8A0F5FA3
:106C90001F4F0F900F900F900F900F900F900B3190
:106CA000110539F7D3C58CE694E09F938F930E942A
:106CB000118B80916C020F900F90882361F01F92CE
:106CC0008F9389E694E09F938F930E94118B0F908E
:106CD0000F900F900F9088E10FB6F89480936000AA
:106CE000109260000FBE0C94007CB0C560916A02E7
:106CF00070916B0280E090E00E94608A8C016BE7EB
:106D000075E00E94748A892BA9F40E9451608091D9
:106D10004A0290914B028D7F816090934B02809349
:106D20004A0242E050E066E170E08AE492E00E94AC
:106D3000548C8CC56EE775E0C8010E94748A892B5B
:106D4000A1F40E94096080914A0290914B028C7FCD
:106D500090934B0280934A0242E050E066E170E07B
:106D60008AE492E00E94548C71C56CEC75E0C80115
:106D70000E94748A892BA9F40E94096080914A02BA
:106D800090914B028E7F826090934B0280934A02D7
:106D900042E050E066E170E08AE492E00E94548CA8
:106DA00055C580914A0281FF0FC08CEC95E09F93FE
:106DB0008F9384EF91E09F938F930E94118B0F909C
:106DC0000F900F900F9042C580FF03C08BE795E0B6
:106DD00002C08EE795E09F938F9380EF91E09F93A1
:106DE0008F930E94118B0F900F900F900F902EC5D4
:106DF00080919C238F9380919B238F9380919A23E2
:106E00008F93809199238F938091A0238F9380916A
:106E10009F238F9380919E238F9380919D238F93A7
:106E20008BE494E09F938F930E94118B80916C026E
:106E30000FB6F894DEBF0FBECDBF882309F406C598
:106E40001F928F9388E494E09F938F930E94118BFD
:106E50000F900F900F900F90F9C4F89481E090E09C
:106E600029E0FC0120935700C895E02C80E090E0D9
:106E7000FC0120935700C895F02C7894F89483E097
:106E800090E0FC0120935700C895002D82E090E02F
:106E9000FC0120935700C895102D789480913D1BDC
:106EA0008F9380913C1B8F9380913B1B8F9380919C
:106EB0003A1B8F932EE334E03F932F930E94118B64
:106EC0001F92EF921F92FF921F920F931F921F9398
:106ED00087E194E09F938F930E94118B0E94F81F8B
:106EE000809166001F928F938BE094E09F938F9325
:106EF0000E94118B0E943E0B80916C020FB6F89499
:106F0000DEBF0FBECDBF882309F4A0C41F928F93AC
:106F100088E094E09F938F930E94118B0F900F90C5
:106F20000F900F9093C460E070E080E090E00E94CA
:106F3000470B60E070E081E090E00E94470B809199
:106F40006C02882309F482C41F928F9385E094E039
:106F50009F938F930E94118B0F900F900F900F9023
:106F600075C40E943E1E0E943E0B80916C028823D5
:106F700009F46CC41F928F9382E094E09F938F93E7
:106F80000E94118B0F900F900F900F905FC4609133
:106F90006A0270916B0280E090E00E94608A61ED6D
:106FA00075E00E94748A892B31F5F89482E999E0A2
:106FB0000E94B14D5C01009769F0C5010F960E94D7
:106FC000B550B50184E092E00E946B4DC5010E946E
:106FD000594EF0CF82E999E00E943E4E892B29F06C
:106FE00082E999E00E94EA4DF5CF82E999E00E949A
:106FF000AD4D789434C082E999E00E94B14D5C01B6
:1070000007ED15E0A114B10451F1F50186811F923D
:107010008F9380851F928F9385811F928F93818597
:107020001F928F9387811F928F9384811F928F93DA
:1070300083811F928F9382811F928F9382851F92EB
:107040008F931F930F930E94FF8AC5010E94594E90
:107050005C010FB6F894DEBF0FBECDBFD3CF8091D9
:107060006C02882309F4F2C31F928F938FEF93E091
:107070009F938F930E94118B0F900F900F900F9002
:10708000E5C30E94102BE2C360916A0270916B020B
:1070900080E090E00E94608A8C0166E176E00E94C8
:1070A000748A892B91F480914A0290914B02977FC8
:1070B00090934B0280934A0242E050E066E170E018
:1070C0008AE492E00E94548CC1C36FE875E0C80165
:1070D0000E94748A892B91F480914A0290914B020C
:1070E000986090934B0280934A0242E050E066E140
:1070F00070E08AE492E00E94548CA8C30E94DB08EE
:10710000A5C360916A0270916B0280E090E00E94DA
:10711000608A009709F4A8C01982BE016F5F7F4F93
:107120000E943A2639014A01B62FA72FF82FE92FDE
:1071300020905202309053024090540250905502D9
:10714000309156023A83809157028B839091580276
:107150009C83209159022D839301A4016B2F7A2FD8
:107160008F2F9E2F51016201EA80FB800C811D81CF
:107170000E94918609F48CC0898181110FC06092B0
:107180005202709253028092540290925502B09330
:107190005602A0935702F09358023FC01816DCF431
:1071A000622860925202732870925302842880925F
:1071B00054029528909255023A81B32BB09356020F
:1071C0008B81A82BA09357029C81F92BF093580236
:1071D000FD81EF2B22C06094709480949094B095C0
:1071E000A095F095E0956220609252027320709213
:1071F00053028420809254029520909255022A8155
:10720000B223B09356023B81A323A09357028C81F3
:10721000F823F0935802FD81EF23E093590248E0F0
:1072200050E06AE170E082E592E00E94548C87EFC2
:1072300093E09F938F930E94118B20915202309183
:107240005302409154025091550260915602709140
:10725000570280915802909159020E94F1220E9497
:107260003E0B0F900F9014C02091520230915302A8
:10727000409154025091550260915602709157020C
:1072800080915802909159020E94F1220E943E0B77
:107290008BEE93E09F938F930E94118B2FEF3FEF24
:1072A0004FEF5FEF60E070E080E090E00E94F1223D
:1072B0000E943E0B80916C020F900F90882309F47E
:1072C000C5C21F928F9388EE93E09F938F930E9485
:1072D000118B0F900F900F900F90B8C260916A02BF
:1072E00070916B0280E090E00E94608A0097D9F074
:1072F0004AE050E060E070E00E94368860935002FF
:10730000709351027F936F938BEC93E09F938F93D5
:107310000E94118B42E050E068E170E080E592E06D
:107320000E94548C0CC0809151028F938091500226
:107330008F938AEA93E09F938F930E94118B0F9013
:107340000F900F900F9080916C02882309F47EC2F9
:107350001F928F9387EA93E09F938F930E94118BE4
:107360000F900F900F900F9071C20E94EE5080917D
:107370006C02882309F46AC21F928F9384EA93E017
:107380009F938F930E94118B0F900F900F900F90EF
:107390005DC20E94CE2780916C02882309F456C2F8
:1073A0001F928F9381EA93E09F938F930E94118B9A
:1073B0000F900F900F900F9049C280E090E00E94D4
:1073C000142080916C02882309F440C21F928F938D
:1073D0008EE993E09F938F930E94118B0F900F90F3
:1073E0000F900F9033C280918F1F81FF2DC00E949C
:1073F000C61D892B49F58091861B8F938091851B33
:107400008F938091841B8F938091831B8F9383E94B
:1074100093E09F938F930E94118B809111288F93FB
:10742000809110288F9380910F288F9380910E2840
:107430008F9386E893E09F938F930E94118B0FB6F2
:10744000F894DEBF0FBECDBF0E943E0B80918F1F10
:107450009091901F90FF63C081E090E00E94761DA4
:107460003B014C0180E090E00E94761D1B012C0145
:107470000E94F51C9F928F927F926F9285E793E016
:107480009F938F930E94118B5F924F923F922F9206
:1074900085E693E09F938F930E94118B222D332DCD
:1074A000442D552D662D772D882D992D0E94DC1B9E
:1074B0009F938F937F936F938AE593E09F938F932E
:1074C0000E94118B222D332D442D552D662D772DA5
:1074D000882D992D0E943D1C9F938F937F936F93CE
:1074E0008CE493E09F938F930E94118B222D332D78
:1074F000442D552D662D772D882D992D0E949E1C8B
:107500009F938F937F936F9389E393E09F938F93E0
:107510000E94118B0FB6F894DEBF0FBECDBF0E9444
:107520003E0B80916C02882309F490C11F928F93C7
:1075300086E393E09F938F930E94118B0F900F909F
:107540000F900F9083C180918F1F82FF2BC021E08D
:1075500048E061E083E00E94DF128091811B8F93FD
:107560008091801B8F9380917F1B8F9380917E1BD6
:107570008F9380917D1B8F9380917C1B8F93809143
:107580007B1B8F9380917A1B8F938FE193E09F9366
:107590008F930E94118B0E943E0B0FB6F894DEBFB2
:1075A0000FBECDBF80918F1F9091901F91FF41C062
:1075B0000E942917B62EA72E982E892E20E030E0A3
:1075C00048EC52E4D501F4016B2F7A2F8F2F9E2FB8
:1075D0000E946A8320E836EE45EC57E40E94ED8075
:1075E00021E03EED42E45EE30E94CD839B01AC01CD
:1075F00060E070E080E89FE30E9422802BE43AE3A1
:107600004DEB57E30E94ED809F938F937F936F9391
:107610008F929F92AF92BF9286E093E09F938F9359
:107620000E94118B0E943E0B0FB6F894DEBF0FBE76
:10763000CDBF80916C02882309F408C11F928F93FB
:1076400083E093E09F938F930E94118B0F900F9094
:107650000F900F90FBC060916A0270916B0280E006
:1076600090E00E94608A6BE176E00E94748A892B28
:10767000B1F460916A0270916B0280E090E00E9428
:10768000608A009709F4E2C00E944E89803108F0B8
:10769000DDC090915201982B90935201D7C08091F8
:1076A00052018F701F928F9383EE91E09F938F937F
:1076B0000E94118B0E943E0B0F900F900F900F9025
:1076C000C5C060916A0270916B0280E090E00E94F8
:1076D000608A009711F14AE050E060E070E00E949B
:1076E0000287603198F4609348021F926F9386EF8F
:1076F00092E09F938F930E94118B41E050E063E1F1
:1077000070E088E492E00E94548C11C0809148029D
:107710001F928F938DEE92E006C0809148021F92D7
:107720008F9384EE92E09F938F930E94118B0F9022
:107730000F900F900F900E943E0B80916C02882357
:1077400009F484C01F928F9381EE92E09F938F93F0
:107750000E94118B0F900F900F900F9077C0609147
:107760006A0270916B0280E090E00E94608A8C0156
:107770006BE775E00E94748A892BA1F40E94BA5EBF
:1077800080914A0290914B02906190934B028093BA
:107790004A0242E050E066E170E08AE492E00E9432
:1077A000548C54C06EE775E0C8010E94748A892B1E
:1077B00041F5F8940E94C85E88E10FB6F894809372
:1077C0006000109260000FBE84B7877F84BF8091F5
:1077D00060008861809360001092600078948091CE
:1077E0004A0290914B029F7E90934B0280934A02F3
:1077F00042E050E066E170E08AE492E00E94548C3E
:1078000025C060E276E0C8010E94748A20914A0295
:1078100030914B02892B21F434FF18C0F894FFCF2C
:1078200034FF03C08BE795E002C08EE795E09F939D
:107830008F938FED91E09F938F930E94118B0F9008
:107840000F900F900F9002C00E94621EEE81FF8188
:107850001182108283E027960FB6F894DEBF0FBE28
:10786000CDBFDF91CF911F910F91FF90EF90DF90EF
:10787000CF90BF90AF909F908F907F906F905F90D0
:107880004F903F902F9008950E94AE5E6C9A6B9A35
:107890006A9A6F9A729A749A739A779A809880B358
:1078A000897F80BB8398849887E080937E00549A78
:1078B0000E9467290E94992981E00E94490980E07D
:1078C00090E00E94930C0E94255880914A0286FD08
:1078D000239A0895CF93DF93EC01888199810097D3
:1078E00041F081159F4009F47EC01982188283E01F
:1078F00083C00E94443C80914A0280FD05C081FF04
:1079000001C01D9B0E940960809170008C7F809354
:1079100070008091B60080628093B6001092B20031
:1079200082E08093B1008091B6008770E1F780918A
:10793000700081608093700065EF78E080E090E0F7
:107940000E94985E0E945A1F80E00E9438218CE0BD
:107950009EE09F938F930E94118B0E94C00F809195
:107960008F1F0F900F9086FD0E944C5980915709F0
:1079700090E00E94AB628091490290E00E945261C7
:107980000E944F61809382098091490290E00E9499
:107990005261809157091F928F93809182091F92A3
:1079A0008F9385E296E09F938F930E94FF8A1092B7
:1079B0008409109283090F900F900F900F900F90F1
:1079C0000F908EE392E090930C2880930B2883E233
:1079D00090E0909395118093941180E09FE09983BB
:1079E000888381E009C06332E1F760E070E083E8FA
:1079F00099E00E94E82BE5CFDF91CF91089584367E
:107A0000910514F19F938F9387E396E09F938F9353
:107A10000E94FF8A8091992390919A23A0919B23A1
:107A2000B0919C230196A11DB11D80939923909341
:107A30009A23A0939B23B0939C230F900F900F90B9
:107A40000F9081E090E0089580E090E008952F92FB
:107A50003F924F925F926F927F928F929F92AF92DE
:107A6000BF92CF92DF92EF92FF920F931F93CF932B
:107A7000DF93CDB7DEB7C559D1090FB6F894DEBF95
:107A80000FBECDBFC457DF4F99838883CC58D040F9
:107A9000633871F487E899E0CB56DF4F6883C559A6
:107AA000D0400E94074BCB56DF4F6881C559D0406C
:107AB000C457DF4FE881F981CC58D0402081318113
:107AC000243BFEE03F07F9F040F42115310581F039
:107AD0002D313D4009F485C079C0253C8EE0380742
:107AE00009F455C02C3C3E4011F40C944A486EC039
:107AF0004FED52E061E870E087E899E00E94ED4ABE
:107B00008DE19DE058C000E010E020914A023091E4
:107B10004B0230FF1EC0739880917B098F5F80936A
:107B20007B098A83B8016F5F7F4FCE0101960E9467
:107B3000365487E899E00E94094B40E050E065E840
:107B400080919811909199110E94C44C84EB9EE011
:107B500032C08D2D90E00E946761F0925102E09258
:107B60005002739A8091580990915909892B11F00C
:107B70000E94096080917B098F5F80937B098091CF
:107B80005B0990915C0982FFBBCF739AB9CF83E701
:107B900099E00E946A4F892BB1F00E945160809158
:107BA0004A0287FD2B9860E470E083E799E00E9429
:107BB000434F8CEC9EE0C457DF4FE881F981CC58ED
:107BC000D0409183808381E00C945D48C457DF4F9F
:107BD000E881F981CC58D0401182108283E00C9466
:107BE0005D48623181F780914A0290914B0291FD8C
:107BF00087CF23E333E343E150E460919123709115
:107C0000922380919323909194230E94E98087FF8F
:107C100014C080919D2390919E23A0919F23B091A9
:107C2000A0230196A11DB11D80939D2390939E23B7
:107C3000A0939F23B093A02363CF8091A223813090
:107C400039F58090A3239090A423A090A523B09011
:107C5000A623F091A723C257DF4FF883CE58D04018
:107C60002091A823C157DF4F2883CF58D0403091AF
:107C7000A923C057DF4F3883C059D0404091AA2371
:107C8000CF56DF4F4883C159D040212C312C2FC013
:107C9000823049F58090A3239090A423A090A5233F
:107CA000B090A6235091A723C257DF4F5883CE58D8
:107CB000D0408091A823C157DF4F8883CF58D04050
:107CC0009091A923C057DF4F9883C059D040E091CD
:107CD000AA23CF56DF4FE883C159D0402090AB2371
:107CE0003090AC2304C0843009F00ACFAACFFA2D1B
:107CF000F470C657DF4FF883CA58D04020E030E018
:107D00004F2F50E060E070E080E090E0A0E00E9443
:107D10009A8609F08C9AB401C5010E947E0A292D29
:107D20002074C557DF4F2883CB58D04020E0C5577B
:107D3000DF4F3881CB58D04040E050E060E070E049
:107D400080E090E0A0E00E949A8611F00E94C61D9B
:107D5000392D3078CE56DF4F3883C259D04020E0DD
:107D600040E050E060E070E080E090E0A0E00E9441
:107D70009A8651F00E94240A6093F5277093F627A3
:107D80008093F7279093F827282D217030E040E06A
:107D900050E060E070E080E090E0A0E00E949A8611
:107DA000F1F084EA9AE19F938F938BE496E09F939E
:107DB0008F931F9287E78F93CE0103969F938F93A4
:107DC0000E94628B7C010E94FF3C0FB6F894DEBFDC
:107DD0000FBECDBF892B09F093CE870102C000E012
:107DE00010E0282D227030E040E050E060E070E0CC
:107DF00080E090E0A0E00E949A86C9F1C801029656
:107E000063E576E0E1E0F0E0EC0FFD1F8E0F9F1FD1
:107E10000E947D8A0D5F1F4FA2E0CA2EA8E2DA2ED3
:107E2000B3EEEB2EB3E0FB2E87E7782EF6018191BF
:107E30006F011F928F93FF92EF921F927F92C80162
:107E4000029621E030E02C0F3D1F820F931F9F937D
:107E50008F930E94628B080F191F0FB6F894DEBF34
:107E60000FBECDBF5AE0C51658E2D506F9F6282D4B
:107E7000247030E040E050E060E070E080E090E0AE
:107E8000A0E00E949A8609F446C0C801029667E500
:107E900076E0E1E0F0E0EC0FFD1F8E0F9F1F0E94E7
:107EA0007D8A0C5F1F4F6E01FAE7CF0ED11C80E177
:107EB000F60111928A95E9F728E0A60168E980EBBE
:107EC0000E9423113601F8E06F0E711CE3EEEE2ED6
:107ED000E3E0FE2EF7E75F2EF60181916F011F921E
:107EE0008F93FF92EF921F925F92C801029621E05A
:107EF00030E02C0F3D1F820F931F9F938F930E94A2
:107F0000628B080F191F0FB6F894DEBF0FBECDBFEE
:107F1000C614D70409F75B2D5078CD56DF4F588330
:107F2000C359D04020E030E040E060E070E080E005
:107F300090E0A0E00E949A8601F580915809909106
:107F400059099F938F938CE596E09F938F931F928F
:107F500087E78F93C8010296E1E0F0E0EC0FFD1F88
:107F60008E0F9F1F9F938F930E94628B080F191F84
:107F70000FB6F894DEBF0FBECDBF20E030E040E08A
:107F800050E0C257DF4F6881CE58D040617070E03A
:107F900080E090E0A0E00E949A8609F1E3E0F0E042
:107FA000EC0FFD1FE00FF11F80E28083E0EBF3E2B6
:107FB00080810F5F1F4F882359F08081A1E0B0E0DE
:107FC000AC0FBD1FA00FB11F12968C933196F0CF4E
:107FD000E3E0F0E0EC0FFD1FE00FF11F1082282D11
:107FE000287030E040E050E060E070E080E090E039
:107FF000A0E00E949A86C1F127E04AE250E06BE2DD
:1080000070E089E290E00E943F5582E098E20E9491
:10801000AD57BC01882777FD8095982F0E948C81F1
:1080200020E030E048EC52E40E94ED809F938F9373
:108030007F936F9383E696E09F938F931F9287E7DA
:108040008F93C801029641E050E04C0F5D1F840FF2
:10805000951F9F938F930E94628B080F191F0FB675
:10806000F894DEBF0FBECDBF282D207130E040E078
:1080700050E060E070E080E090E0A0E00E949A862E
:10808000F1F126E04AE250E06BE270E089E290E034
:108090000E943F5581E090E00E94CC0A80935609EF
:1080A00082EF9AE10E94AD57BC01882777FD809549
:1080B000982F0E948C8120E030E048EC52E40E942E
:1080C000ED809F938F937F936F938DE696E09F93C0
:1080D0008F931F9287E78F93C8010296E1E0F0E04B
:1080E000EC0FFD1F8E0F9F1F9F938F930E94628B3B
:1080F000080F191F0FB6F894DEBF0FBECDBF282D95
:10810000207230E040E050E060E070E080E090E01D
:10811000A0E00E949A8631F18091B11A8F938091EC
:10812000B01A8F938091AF1A8F938091AE1A8F936C
:1081300088E796E09F938F931F9287E78F93C801FC
:10814000029641E050E04C0F5D1F840F951F9F93F6
:108150008F930E94628B080F191F0FB6F894DEBF31
:108160000FBECDBF282D207430E040E050E060E02D
:1081700070E080E090E0A0E00E949A8631F180916A
:1081800094238F93809193238F93809192238F9345
:10819000809191238F9386E896E09F938F931F920F
:1081A00087E78F93C8010296E1E0F0E0EC0FFD1F36
:1081B0008E0F9F1F9F938F930E94628B080F191F32
:1081C0000FB6F894DEBF0FBECDBF282D207830E06B
:1081D00040E050E060E070E080E090E0A0E00E94CD
:1081E0009A8641F1F8948091ED279091EE27A09125
:1081F000EF27B091F0277894BF93AF939F938F931D
:1082000084E996E09F938F931F9287E78F93C8012D
:10821000029641E050E04C0F5D1F840F951F9F9325
:108220008F930E94628B080F191F0FB6F894DEBF60
:108230000FBECDBF20E0392D317040E050E060E04E
:1082400070E080E090E0A0E00E949A8609F477C098
:108250008091500290915102892B09F470C0F894DA
:10826000C090ED27D090EE27E090EF27F090F02718
:1082700078948091EA1A9091EB1AA091EC1AB0913F
:10828000ED1AA7019601281B390B4A0B5B0BCA019B
:10829000B9010E948A812B013C01609150027091CA
:1082A000510280E090E00E948A819B01AC01C301F1
:1082B000B2010E94ED803C017F928F937F936F9378
:1082C0008FE996E09F938F931F9287E78F939E018C
:1082D000200F311F2D5F3F4F3F932F93CB56DF4F22
:1082E0006883C559D040CC56DF4F7883C459D040FD
:1082F0000E94628B080F191FCB56DF4F6881C5594A
:10830000D040CC56DF4F7881C459D040862F972F6C
:10831000A62DB72D8093FA279093FB27A093FC27D7
:10832000B093FD27C092EA1AD092EB1AE092EC1AB1
:10833000F092ED1A0FB6F894DEBF0FBECDBF20E06D
:10834000392D327040E050E060E070E080E090E075
:10835000A0E00E949A8691F1809150029091510282
:10836000892B61F1F8948091C11A9091C21AA09161
:10837000C31AB091C41A78949F938F9380914F023F
:108380008F9380914E028F938CEA96E09F938F9308
:108390001F9287E78F93C8010296E1E0F0E0EC0FAF
:1083A000FD1F8E0F9F1F9F938F930E94628B080F5C
:1083B000191F0FB6F894DEBF0FBECDBF20E0392DD8
:1083C000347040E050E060E070E080E090E0A0E0D9
:1083D0000E949A8671F1F8948091F1279091F2278A
:1083E000A091F327B091F4277894BF93AF939F9314
:1083F0008F938CEB96E09F938F931F9287E78F93D9
:10840000C801029641E050E04C0F5D1F840F951F9C
:108410009F938F930E94628B080F191FC8010E94BF
:10842000FF3C0FB6F894DEBF0FBECDBF892B09F01D
:1084300067CB20E0392D387040E050E060E070E01C
:1084400080E090E0A0E00E949A8609F477C08091D5
:10845000500290915102892B09F470C0F894C09099
:10846000F127D090F227E090F327F090F42778944A
:108470008091EE1A9091EF1AA091F01AB091F11A32
:10848000A7019601281B390B4A0B5B0BCA01B901E6
:108490000E948A812B013C0160915002709151022F
:1084A00080E090E00E948A819B01AC01C301B2018F
:1084B0000E94ED803C017F928F937F936F9387ECB6
:1084C00096E09F938F931F9287E78F939E01200FD3
:1084D000311F2D5F3F4F3F932F93CB56DF4F688364
:1084E000C559D040CC56DF4F7883C459D0400E9444
:1084F000628B080F191FCB56DF4F6881C559D040DA
:10850000CC56DF4F7881C459D040862F972FA62DA7
:10851000B72D8093FE279093FF27A0930028B09358
:108520000128C092EE1AD092EF1AE092F01AF0925F
:10853000F11A0FB6F894DEBF0FBECDBF20E0392D83
:10854000307140E050E060E070E080E090E0A0E05A
:108550000E949A8691F18091500290915102892B4C
:1085600061F1F8948091C51A9091C61AA091C71A2A
:10857000B091C81A78949F938F9380914D028F93F6
:1085800080914C028F9384ED96E09F938F931F927E
:1085900087E78F93C8010296E1E0F0E0EC0FFD1F42
:1085A0008E0F9F1F9F938F930E94628B080F191F3E
:1085B0000FB6F894DEBF0FBECDBF20E0392D30726C
:1085C00040E050E060E070E080E090E0A0E00E94D9
:1085D0009A8661F18091952390919623A09197239B
:1085E000B0919823BF93AF939F938F9384EE96E0BF
:1085F0009F938F931F9287E78F93C801029641E064
:1086000050E04C0F5D1F840F951F9F938F930E9426
:10861000628B080F191FC8010E94FF3C0FB6F89427
:10862000DEBF0FBECDBF892B09F06ACA20E0C55757
:10863000DF4F3881CB58D04040E050E060E070E040
:1086400080E090E0A0E00E949A8661F18091861B14
:108650008F938091851B8F938091841B8F93809142
:10866000831B8F938FEE96E09F938F931F9287E7E4
:108670008F93C801029621E030E02C0F3D1F820F3E
:10868000931F9F938F930E94628B080F191FC8013D
:108690000E94FF3C0FB6F894DEBF0FBECDBF892B02
:1086A00009F02ECA20E0CE56DF4F3881C259D040A3
:1086B00040E050E060E070E080E090E0A0E00E94E8
:1086C0009A8661F18091F8278F938091F7278F9395
:1086D0008091F6278F938091F5278F938AEF96E00C
:1086E0009F938F931F9287E78F93C8010296E1E0D3
:1086F000F0E0EC0FFD1F8E0F9F1F9F938F930E9442
:10870000628B080F191FC8010E94FF3C0FB6F89436
:10871000DEBF0FBECDBF892B09F0F2C920E030E0EB
:108720004A2D417050E060E070E080E090E0A0E011
:108730000E949A8689F181E00E94D50920917102F8
:108740003091720240917302509174020E946A83C8
:108750009F938F937F936F9387E097E09F938F937F
:108760001F9287E78F93C801029641E050E04C0FBB
:108770005D1F840F951F9F938F930E94628B080F3C
:10878000191FC8010E94FF3C0FB6F894DEBF0FBE50
:10879000CDBF892B09F0B4C920E030E04A2D4270EA
:1087A00050E060E070E080E090E0A0E00E949A86F7
:1087B00089F182E00E94D50920916D0230916E020C
:1087C00040916F02509170020E946A839F938F9331
:1087D0007F936F9384E197E09F938F931F9287E736
:1087E0008F93C801029621E030E02C0F3D1F820FCD
:1087F000931F9F938F930E94628B080F191FC801CC
:108800000E94FF3C0FB6F894DEBF0FBECDBF892B90
:1088100009F076C920E030E0C657DF4F4881CA58DA
:10882000D04050E060E070E080E090E0A0E00E9486
:108830009A8641F183E00E94D5099F938F937F939D
:108840006F9381E297E09F938F931F9287E78F93B7
:10885000C8010296E1E0F0E0EC0FFD1F8E0F9F1FB4
:108860009F938F930E94628B080F191F8C98C801E9
:108870000E94FF3C0FB6F894DEBF0FBECDBF892B20
:1088800009F03EC920E030E04A2D487050E060E039
:1088900070E080E090E0A0E00E949A8671F1809103
:1088A0008F1F87FF2AC021E042E161E080ED0E9436
:1088B000EF599F938F937F936F938EE297E09F93EF
:1088C0008F931F9287E78F93C801029641E050E093
:1088D0004C0F5D1F840F951F9F938F930E94628B97
:1088E000080F191FC8010E94FF3C0FB6F894DEBFA5
:1088F0000FBECDBF892B09F003C920E030E04A2D1F
:10890000407150E060E070E080E090E0A0E00E9404
:108910009A8671F180918F1F87FF2AC021E042E182
:1089200062E080ED0E94EF599F938F937F936F9346
:108930008CE397E09F938F931F9287E78F93C801F3
:10894000029621E030E02C0F3D1F820F931F9F9372
:108950008F930E94628B080F191FC8010E94FF3C71
:108960000FB6F894DEBF0FBECDBF892B09F0C8C883
:1089700020E030E04A2D407250E060E070E080E09E
:1089800090E0A0E00E949A8671F180918F1F87FF8E
:108990002AC021E042E163E080ED0E94EF599F93FD
:1089A0008F937F936F938AE497E09F938F931F92A7
:1089B00087E78F93C8010296E1E0F0E0EC0FFD1F1E
:1089C0008E0F9F1F9F938F930E94628B080F191F1A
:1089D000C8010E94FF3C0FB6F894DEBF0FBECDBFAA
:1089E000892B09F08DC820E030E04A2D407450E01A
:1089F00060E070E080E090E0A0E00E949A8671F173
:108A000080918F1F87FF2AC021E042E164E080ED62
:108A10000E94EF599F938F937F936F9388E597E020
:108A20009F938F931F9287E78F93C801029641E02F
:108A300050E04C0F5D1F840F951F9F938F930E94F2
:108A4000628B080F191FC8010E94FF3C0FB6F894F3
:108A5000DEBF0FBECDBF892B09F052C8FA2DF078CA
:108A6000EF2E20E030E04F2F50E060E070E080E03B
:108A700090E0A0E00E949A8649F080918F1F82FFCB
:108A800005C046E061E083E00E94DF122B2D2170DB
:108A9000F22E20E030E040E05F2D60E070E080E00A
:108AA00090E0A0E00E949A8651F080918F1F82FF93
:108AB00006C021E046E061E083E00E94DF1220E092
:108AC00030E04E2D50E060E070E080E090E0A0E00B
:108AD0000E949A8689F180918F1F82FF2DC080911C
:108AE0007D1B8F9380917C1B8F9380917B1B8F9339
:108AF00080917A1B8F9386E697E09F938F931F92C6
:108B000087E78F93C801029641E050E04C0F5D1F4C
:108B1000840F951F9F938F930E94628B080F191FDC
:108B2000C8010E94FF3C0FB6F894DEBF0FBECDBF58
:108B3000892B11F00C94803D20E030E040E05F2D67
:108B400060E070E080E090E0A0E00E949A8689F109
:108B500080918F1F82FF2DC08091811B8F93809108
:108B6000801B8F9380917F1B8F9380917E1B8F93AF
:108B70008EE697E09F938F931F9287E78F93C801AC
:108B8000029621E030E02C0F3D1F820F931F9F9330
:108B90008F930E94628B080F191FC8010E94FF3C2F
:108BA0000FB6F894DEBF0FBECDBF892B11F00C9429
:108BB000803D20E030E040E05B2D527060E070E0EE
:108BC00080E090E0A0E00E949A8679F180918F1F6A
:108BD0009091901F90FF29C080E090E00E94761D48
:108BE0009F938F937F936F9389E797E09F938F93E2
:108BF0001F9287E78F93C8010296E1E0F0E0EC0F47
:108C0000FD1F8E0F9F1F9F938F930E94628B080FF3
:108C1000191FC8010E94FF3C0FB6F894DEBF0FBEBB
:108C2000CDBF892B11F00C94803D20E030E040E076
:108C30005B2D547060E070E080E090E0A0E00E9466
:108C40009A8679F180918F1F9091901F90FF29C093
:108C500081E090E00E94761D9F938F937F936F93A6
:108C600089E897E09F938F931F9287E78F93C801BE
:108C7000029641E050E04C0F5D1F840F951F9F93BB
:108C80008F930E94628B080F191FC8010E94FF3C3E
:108C90000FB6F894DEBF0FBECDBF892B11F00C9438
:108CA000803D20E030E040E05B2D507160E070E0FE
:108CB00080E090E0A0E00E949A86D9F180918F1F19
:108CC0009091901F90FF35C081E090E00E94761D4A
:108CD0006B017C0180E090E00E94761D9B01AC015D
:108CE000C701B6010E94DC1B9F938F937F936F9304
:108CF0008AE997E09F938F931F9287E78F93C8012C
:108D0000029621E030E02C0F3D1F820F931F9F93AE
:108D10008F930E94628B080F191FC8010E94FF3CAD
:108D20000FB6F894DEBF0FBECDBF892B11F00C94A7
:108D3000803D20E030E040E05B2D507260E070E06C
:108D400080E090E0A0E00E949A86D9F180918F1F88
:108D50009091901F90FF35C081E090E00E94761DB9
:108D60006B017C0180E090E00E94761D9B01AC01CC
:108D7000C701B6010E943D1C9F938F937F936F9311
:108D800085EA97E09F938F931F9287E78F93C8019F
:108D90000296E1E0F0E0EC0FFD1F8E0F9F1F9F9306
:108DA0008F930E94628B080F191FC8010E94FF3C1D
:108DB0000FB6F894DEBF0FBECDBF892B11F00C9417
:108DC000803D20E030E040E05B2D507460E070E0DA
:108DD00080E090E0A0E00E949A86D9F180918F1FF8
:108DE0009091901F90FF35C081E090E00E94761D29
:108DF0006B017C0180E090E00E94761D9B01AC013C
:108E0000C701B6010E949E1C9F938F937F936F931F
:108E100083EB97E09F938F931F9287E78F93C8010F
:108E2000029641E050E04C0F5D1F840F951F9F9309
:108E30008F930E94628B080F191FC8010E94FF3C8C
:108E40000FB6F894DEBF0FBECDBF892B11F00C9486
:108E5000803D20E030E040E05B2D587060E070E045
:108E600080E090E0A0E00E949A8669F180918F1FD7
:108E70009091901F91FF27C00E9429179F938F9375
:108E80007F936F9386EC97E09F938F931F9287E772
:108E90008F93C801029621E030E02C0F3D1F820F16
:108EA000931F9F938F930E94628B080F191FC80115
:108EB0000E94FF3C0FB6F894DEBF0FBECDBF892BDA
:108EC00011F00C94803D20E030E040E0CD56DF4FC3
:108ED0005881C359D04060E070E080E090E0A0E0AD
:108EE0000E949A8671F1F10186811F928F9385818C
:108EF0001F928F9383811F928F9382811F928F93F2
:108F000087ED97E09F938F931F9287E78F93C80118
:108F1000029621E030E02C0F3D1F820F931F9F939C
:108F20008F930E94628B080F191FC8010E94FF3C9B
:108F30000FB6F894DEBF0FBECDBF892B11F00C9495
:108F4000803D779A80915B0990915C0992FD749ABB
:108F50009401A501C257DF4F6881CE58D040C15758
:108F6000DF4F7881CF58D040C057DF4F8881C0593C
:108F7000D040CF56DF4F9881C159D040A0E0FE01CC
:108F800033967F010E949A8651F180915B099091FE
:108F90005C0982FD08C080914A0280FD04C081FF07
:108FA0001EC01D9B1CC0FF92EF928EEE97E09F9318
:108FB0008F930E94FF8A80916C020F900F900F9008
:108FC0000F90882361F01F928F9389E09EE09F931A
:108FD0008F930E94118B0F900F900F900F908091A4
:108FE00048028061898380917B098A83F701E00FC1
:108FF000F11F108280915B0990915C0998012D5FAF
:109000003F4F790180FF0CC0FF922F9385EF97E0CF
:109010009F938F930E94FF8A0F900F900F900F9055
:10902000B701CE0101960E94365480914A0282FF18
:109030000AC02DEE33E2A701BE016F5F7F4F8AE5C4
:1090400092E00E94BC5880915B0990915C0982FD7E
:1090500073980E94516087E899E00E94094B8091C3
:109060004A0290914B0290FD02C00C94B23D0F5FFA
:109070001F4FE0905002F09051020E944F61D82E95
:10908000109251021092500289E190E00E946761B3
:109090000C94853D83E799E00E946A4F892B11F477
:1090A0000C94E33D0E94096080914A0287FD02C052
:1090B0000C94803D2B9A0C94803DCB56DF4F0FB61D
:1090C000F894DEBF0FBECDBFDF91CF911F910F91FE
:1090D000FF90EF90DF90CF90BF90AF909F908F90D8
:1090E0007F906F905F904F903F902F9008950C94D9
:1090F000304B4F925F926F927F928F929F92AF927E
:10910000BF92CF92DF92EF92FF920F931F93CF9374
:10911000DF93CDB7DEB760970FB6F894DEBF0FBE12
:10912000CDBF6B010E944F61FC01EE0FFF1FEE7F70
:10913000F170ED54F54E8081918101969183808389
:1091400080915B0990915C0981FD749880904A023E
:1091500090904B020E948A537C01FC018081982FE1
:1091600092959F70913099F48F7051F48091BF1A4D
:109170009091C01A01969093C01A8093BF1A08C1AB
:10918000B60182E198E20E94A64A892B51F08091B3
:10919000BD1A9091BE1A01969093BE1A8093BD1A83
:1091A000F7C0C40184E0989F812D99271124F82FDE
:1091B000F1708F2E82E999E00E94B14D8C010097E9
:1091C00009F448C0B601C80102960E94A64A892B3C
:1091D000E9F198014FE059E060E074E6C8010F96AC
:1091E0000E943150F7019181F8018481981321C0C8
:1091F00082858F5F82878091BB1A9091BC1A0196FD
:109200009093BC1A8093BB1A84E00E94A754F80183
:10921000208530E02817390708F074C184E00E94E7
:10922000A754F8018087F70180818F70F80181874A
:10923000AFC0F801128684E00E94A754F80180872D
:10924000F70180818F70F80181875DC1C8010E949C
:10925000594EB4CF84E092E00E94464D8C010097B5
:1092600009F496C0B601C80102960E949D4AF70112
:1092700081818150F801848380E091E0A0E0B0E03A
:1092800083879487A587B687128684E00E94A754B7
:10929000F8018087F70180818F70F8018187B8011C
:1092A00082E999E00E94114E98014FE059E060E098
:1092B00074E6C8010F960E94315099249394F701E7
:1092C0008181F8018483F70180818F70F8018783A1
:1092D00084E00E94A754F801858383E00E94A7548C
:1092E0005C01F801868387818F3009F0912CF701AA
:1092F0004180F8018481481A512C612C712C46E080
:10930000440C551C661C771C4A95D1F7238534857F
:1093100045855685A0ECB0E00E944884BB27A92F64
:10932000982F872F480E591E6A1E7B1E438654862F
:109330006586768680915B0990915C0981FD32C0DB
:1093400080914A0280FD2EC081FD2AC0992001F142
:1093500082E08093A22381E08093A3231092A42330
:109360001092A52380E88093A6231092A723109241
:10937000A8231092A9231092AA231093AC23009340
:10938000AB2342EA53E262E18AE292E00E94C44CDB
:1093900080915B0990915C0981FFB7C0749AB5C058
:1093A0001D9BD4CFA4E6B0E0A30192010E944884A3
:1093B000672F782F892F992724E630E040E050E08E
:1093C0000E9493847F936F93452C562C672C7724AF
:1093D0005F924F92BB24BF92AF92F80185811F929A
:1093E0008F93F70180818F701F928F9381811F92DD
:1093F0008F93F60181811F928F9380811F928F93AB
:10940000C70102969F938F9386E098E09F938F9376
:109410000E94FF8A80916C020FB6F894DEBF0FBEE7
:10942000CDBF882361F01F928F9386E09EE09F93CB
:109430008F930E94118B0F900F900F900F9080913F
:109440004A0290914B0296FF2DC0882059F1F701F6
:109450002081322F3F70832F90E00297D4F08FEF5E
:10946000830F207F822B808387E899E00E947748D2
:109470008091B91A9091BA1A01969093BA1A809372
:10948000B91A80915B0990915C0996FF0BC07398A3
:1094900009C08091BF1A9091C01A01969093C01A8A
:1094A0008093BF1A80918F1F86FF50CF0E943E5934
:1094B000C70105960E940A59F70181811F928F9377
:1094C000F80186811F928F9385811F928F938AE482
:1094D00098E09F938F931F9280E18F939E012F5F5F
:1094E0003F4F7901FF922F930E94628B82E00E948E
:1094F0002459C7010E940A590FB6F894DEBF0FBE67
:10950000CDBF24CF812C912CDACE60960FB6F89483
:10951000DEBF0FBECDBFDF91CF911F910F91FF90A6
:10952000EF90DF90CF90BF90AF909F908F907F9003
:109530006F905F904F9008950895FB012081FC018A
:109540002083FB012181FC0121830895FC0190818E
:10955000DB018C91981309C081E090E03181119674
:109560002C91321721F080E0089580E090E008957A
:10957000BC0182E198E20C949D4ADC011996ED91C0
:10958000FC911A970280F381E02D309709F009943D
:1095900008950F931F93CF93DF9300D0CDB7DEB71D
:1095A0008C0188E10E94BA54BC01CE0101960E9450
:1095B0009D4AD8011996ED91FC911A970190F0817E
:1095C000E02DBE016F5F7F4FC80109950F900F908E
:1095D000DF91CF911F910F910895EF92FF920F931A
:1095E0001F93CF93DF93EC018B017A0143EF52E09D
:1095F0000E94164BFA86E98667EF72E0C801DF9198
:10960000CF911F910F91FF90EF900C946F4B0C94A2
:109610002E4BCF93DF93EC0162E178E288E10E9468
:10962000B054CE01DF91CF910C94304BEF92FF926A
:109630000F931F93CF93DF93EC018B017A010E946C
:109640004B4BF886EF826BEF72E0C801DF91CF9150
:109650001F910F91FF90EF900C946F4B0C94534B14
:109660000C94CB65DC011796ED91FC911897019055
:10967000F081E02D0994DC011796ED91FC9118978B
:109680000280F381E02D309709F00994089586E96E
:1096900091E10C94AD4DFC0173836283BC0186E9BA
:1096A00091E10C94114EBC0186E991E10C94F64DC8
:1096B000CF93DF93EC0186E991E10E94B14D0097D1
:1096C00049F0FC01228133812C173D0729F00E94CB
:1096D000594EF5CF80E090E0DF91CF9108950F9340
:1096E0001F93CF93DF938B010E94584BEC0100979F
:1096F00031F01D830C83C8010E94FC678E83DF91CB
:10970000CF911F910F9108951F93CF93DF93EC0199
:10971000162FEC81FD813097D1F0909399118093B1
:10972000981182E08887CE0106960995992787FDD2
:1097300090950297029710F0133839F4BE01CE01CC
:10974000DF91CF911F910C94B14B81E08887DF911D
:10975000CF911F910895FC01208520FD0C94844B2E
:109760000895CF92DF92EF92FF920F931F93CF93C2
:10977000DF93EC016B01E0909811F090991100914A
:109780009A1110919B11F801EC17FD0739F03097F1
:1097900009F44AC00190F081E02DF6CF209709F43A
:1097A00043C08885882309F118860115110561F0E9
:1097B000C017D10729F0AE0167E8C8010E94AB4B82
:1097C000F80100811181F1CFEC81FD81309769F0C2
:1097D000CC15DD0551F0D0939911C093981140E05C
:1097E00050E063E8CE0106960995E0919A11F09158
:1097F0009B11CE17DF0769F48881998190939B11A3
:1098000080939A110DC0808191818C179D0721F062
:10981000FC013097C1F704C08881998191838083CE
:10982000F0929911E0929811DF91CF911F910F91D1
:10983000FF90EF90DF90CF9008951F93CF93DF9329
:109840001092A411C0919A11D0919B1111E0209710
:1098500079F08985882341F01887198640E050E027
:1098600062E8CE010E94844B0990D881C02DEFCFD1
:10987000DF91CF911F9108958091471291E0980F49
:1098800090934712089560919811709199110C94DA
:10989000B14B8AE8809347121092451210924612FB
:1098A00010929B1110929A11109299111092981186
:1098B00008958091A41181110E941D4C709146124F
:1098C000772309F451C0E09145122E2F30E085E056
:1098D000E89FF0011124EB55FE4E60816093A311C7
:1098E000418152815093A2114093A11183819481AF
:1098F0009093A01180939F112F5F3F4F2F713327BB
:1099000020934512715070934612009731F5809163
:109910009A1190919B1190939E1180939D1180912B
:109920009D1190919E11892BF9F08091A4118111C4
:109930000E941D4C4091A1115091A2116091A31160
:1099400080919D1190919E110E94AB4BE0919D11D1
:10995000F0919E1180819181DECF613819F421E070
:10996000FC0120870E94AB4B8091A41120914612EC
:1099700090E0820F911D08958091A41120914612CC
:1099800090E0820F911D0895209146122032B9F087
:10999000E0914512E20FEF71E0939C1135E0E39FF7
:1099A000F0011124EB55FE4E608352834183948372
:1099B00083832F5F2093461280E090E0089581E03A
:1099C00090E00895CF93DF93C0919811D0919911B1
:1099D0000E94AB4BD0939911C0939811DF91CF9116
:1099E0000895AB0130919A1120919B11E32FF22F32
:1099F000E817F907B1F0309721F00190F081E02DE0
:109A0000F7CF009771F0FC013083218390939B1175
:109A100080939A1121E020871782168261E80C94C6
:109A2000E24C0895009749F0FC0120852150223036
:109A300020F421E021872093A411089521E030E053
:109A4000FC018085811102C020E030E0C901089549
:109A5000CF93DF93EC014A815B8160E070E08C8101
:109A60009D810E946D8A2A813B8188819981289FEE
:109A7000A001299F500D389F500D112460E070E027
:109A80008E819F81DF91CF910C946D8AFC01828140
:109A9000938120E030E028173907D1F0A481B58107
:109AA000A20FB31F4C91411110C081E08C938081B3
:109AB0009181289FA001299F500D389F500D11249E
:109AC00086819781840F951F08952F5F3F4FE3CFC5
:109AD00080E090E00895FC01268137814281538126
:109AE00080E090E084179507C9F02617370781F4C6
:109AF000A481B581A80FB91F2C91121614F421501E
:109B00002C930480F581E02DE80FF91F80810895E2
:109B1000A081B1812A0F3B1F0196E4CF8FEF0895FA
:109B2000FC018681978168177907A0F0A081B18137
:109B300042815381A49F9001A59F300DB49F300DA9
:109B40001124280F391F81E090E06217730720F07D
:109B500080E0089580E090E00895FC011182108279
:109B60000895FC01808191810895FB01208131815C
:109B7000FC01318320830895DC01ED91FC91309745
:109B800031F080819181009729F0FC01FACF80E0CB
:109B900090E00895CF010895DC01ED91FC911197BB
:109BA0003097A9F020813181232B21F41D921C9242
:109BB000CF010895A081B1818D919C911197892B3E
:109BC00011F0FD01F7CF11821082CD01089580E0E0
:109BD00090E00895DC01ED91FC911197309721F010
:109BE000208131812D933C93CF010895DC01ED91CB
:109BF000FC913097A9F0A0E0B0E020813181E61718
:109C0000F70741F4109709F4DC012D933C9311827E
:109C1000108208952115310519F0DF01F901EDCF0A
:109C200008950F931F93CF93DF938C01EB010E9454
:109C3000F64D19821882C8010E94BC4D009711F49C
:109C4000F80101C0FC01D183C083DF91CF911F9146
:109C50000F9108950F931F93CF93DF93EC018B0126
:109C60000E94F64D88819981F80191838083198340
:109C70000883DF91CF911F910F910895DC01ED9141
:109C8000FC9180E090E0309729F001960190F081FE
:109C9000E02DF9CF0895FB01309719F4BA010C9427
:109CA0002A4E80819181DA018D939C935183408368
:109CB0000895009721F0FC0180819181089580E052
:109CC00090E0089580914A1290914B12892B29F4CB
:109CD000109249121092481208950E94565DE09128
:109CE0004A12F0914B122281338140815181240F1D
:109CF000351F281B390B0480F581E02D309769F062
:109D00004281538160817181460F571F481B590B57
:109D10004217530780F79A01EECF280F391F30936F
:109D200049122093481208958BE792E00C94124D4B
:109D3000EF92FF920F931F93CF93DF938C01FC015F
:109D400080819181009799F08A359105D9F0F801C9
:109D50001182108283E068C08681978184179507FD
:109D600009F049C00480F581E02D3097A9F71092E1
:109D70004B1210924A128AE590E0F8019183808399
:109D800081E052C0673891F16238A9F7C0914A1258
:109D9000D0914B12E12CF12C209769F3CE010E9457
:109DA000CD6B892BF1F0AE0168E88E819F810E9416
:109DB000C44C892BA1F41F821E828C819D81E114E9
:109DC000F10421F0F7019583848304C090934B1232
:109DD00080934A121D821C820E94624ED7CF0E943D
:109DE000944E7E010C80DD81C02DD6CFE0914A12C9
:109DF000F0914B12BACFF0934B12E0934A12A48128
:109E0000B581109709F4B7CF16968D919C9117974D
:109E10008417950711F0FD01F2CF14968D919C9156
:109E2000159795838483EBCFDF91CF911F910F918D
:109E3000FF90EF900895CF93DF93EC010E94944E32
:109E40008E819F8130914A1220914B12892B59F0BB
:109E5000E32FF22F309739F0EC17FD0781F00480E3
:109E6000F581E02DF7CF80919811909199119F8302
:109E70008E833C832D83D0934B12C0934A12DF9183
:109E8000CF910C94624ECF93DF93EC010E94AD6BA7
:109E9000CE01DF91CF910C941B4FCF93DF93EC0158
:109EA0000E94B96BCE01DF91CF910C941B4FCF93E1
:109EB000DF93EC010E94C36BCE01DF91CF910C9434
:109EC0001B4FFC0120813181260F371F31832083F6
:109ED0000C94624E21E030E0FC0186819781892B51
:109EE00011F020E030E0C9010895FC0122813381A6
:109EF00080819181820F931F0895FC01808191815F
:109F0000089581E090E020914A1230914B12232B6A
:109F100011F480E090E0089580914A1290914B12E4
:109F2000892B29F08091481290914912089580E080
:109F300090E00895CF93DF93EC01E0914A12F09105
:109F40004B128E179F0769F48C819D8190934B1261
:109F500080934A120DC0848195818C179D0721F052
:109F6000FC013097C1F706C08C819D819583848365
:109F70000E94624E1D821C821F821E82DF91CF9141
:109F80000895EF92FF920F931F93CF93DF938C016D
:109F90007A01FC0180819181009741F08B34910519
:109FA00001F1F8011182108283E048C08DE492E152
:109FB0000E94B14DEC01209751F06C817D81CE0162
:109FC00002960E94434F0990D881C02DF4CF81E0C2
:109FD00080934C128BE490E0F8019183808381E0C0
:109FE0002DC06838E1F78DE492E10E94B14DEC019B
:109FF000209781F3CE010296E816F906D9F4BE0146
:10A000008DE492E10E94F64DE0909811F090991144
:10A010008A859B859093991180939811EC85FD8595
:10A02000309719F08E859F850995F0929911E092ED
:10A030009811D0CF0990D881C02DDACFDF91CF9180
:10A040001F910F91FF90EF90089510924C128DE4A4
:10A0500092E10E94AD4D60E070E085E892E00C94E2
:10A06000F14C0F931F93CF93DF93EC010091981164
:10A07000109199111B870A875D874C873F872E8730
:10A0800080914C12882379F085E892E090939911A1
:10A0900080939811CE0102960E94434F109399111C
:10A0A0000093981102C07D836C83BE018DE492E120
:10A0B0000E94F64DBE018DE492E1DF91CF911F9198
:10A0C0000F910C94114E0F931F93CF93DF93EC01DC
:10A0D00080914C12882391F0009198111091991160
:10A0E00085E892E09093991180939811CE010296A1
:10A0F0000E944D4F1093991100939811BE018DE469
:10A1000092E10E94F64DBE018DE492E1DF91CF9184
:10A110001F910F910C94114E0F931F93CF93DF93C8
:10A12000EC0180914C12882391F0009198111091CC
:10A13000991185E892E09093991180939811CE013E
:10A1400002960E94574F1093991100939811BE01E7
:10A150008DE492E10E94F64DBE018DE492E1DF9123
:10A16000CF911F910F910C94114ECF93DF93EC017F
:10A1700080914C12882329F0CE0102960E949A4FBA
:10A1800004C01F821E8219861886BE018DE492E1EA
:10A19000DF91CF910C94F64DCF93DF93EC0180913A
:10A1A0004C12882331F0CE010296DF91CF910C94AE
:10A1B0006A4F8DE492E10E94B14D009739F08C17FF
:10A1C0009D0739F0FC0180819181F7CF81E090E01B
:10A1D00002C080E090E0DF91CF9108952F923F92EE
:10A1E0004F925F926F927F928F929F92AF92BF92A7
:10A1F000CF92DF92EF92FF920F931F93CF93DF9353
:10A20000CDB7DEB7E8970FB6F894DEBF0FBECDBF6F
:10A21000E9E4FAE22081318142815381E5E4FAE206
:10A220005080418032802380E1E4FAE2808189839A
:10A2300091819A83A281AB836380EDE3FAE2B081DE
:10A24000BC8381818D8392819E83A381AF83E9E367
:10A25000FAE2B081B8878181898792819A87A38148
:10A26000AB87E5E3FAE2B081BC8781818D8792817B
:10A270009E87A381AF87E1E3FAE2B081B88B818149
:10A28000898B92819A8BA381AB8BEDE2FAE2B0814C
:10A29000BC8B81818D8B92819E8BA381AF8BE9E2F8
:10A2A000FAE2B081B88F8181898F92819A8FA381E0
:10A2B000AB8FE5E2FAE2B081BC8F81818D8F928114
:10A2C0009E8FA381AF8FE1E2FAE2B081B8A38181D2
:10A2D00089A392819AA3A381ABA3EDE1FAE2B081B5
:10A2E000BCA381818DA392819EA3A381AFA3E9E149
:10A2F000FAE2B081B8A7818189A792819AA7A38148
:10A30000ABA7E5E1FAE2B081BCA781818DA792817C
:10A310009EA7A381AFA7E1E1FAE2B081B8AB81814A
:10A3200089AB92819AAB7380EDE0FAE2B080A180B4
:10A3300092808380E9E0FAE2F080E180D280C380FD
:10A34000E5E0FAE2A081AFABB181B8AF1281038141
:10A350002BAB3CAB4DAB5EAB0E94845D5EA95F93C3
:10A360004DA94F933CA93F932BA92F932F923F9236
:10A370004F925F926F922B812F932A812F93298185
:10A380002F932F812F932E812F932D812F932C810B
:10A390002F932B852F932A852F9329852F932885FB
:10A3A0002F932F852F932E852F932D852F932C85DB
:10A3B0002F932B892F932A892F9329892F932889CB
:10A3C0002F932F892F932E892F932D892F932C89AB
:10A3D0002F932B8D2F932A8D2F93298D2F93288D9B
:10A3E0002F932F8D2F932E8D2F932D8D2F932C8D7B
:10A3F0002F932BA12F932AA12F9329A12F9328A12B
:10A400002F932FA12F932EA12F932DA12F932CA10A
:10A410002F932BA52F932AA52F9329A52F9328A5FA
:10A420002F932FA52F932EA52F932DA52F932CA5DA
:10A430002F937F922AA92F9329A92F9328A92F938D
:10A440008F929F92AF92BF92CF92DF92EF92FF9244
:10A450000F931F9328AD2F932FA92F939F938F9323
:10A460007F936F93A3E1B8E28C911F928F93E2E107
:10A47000F8E280811F928F9381E89EE09F938F93F3
:10A480000E94118BE9E7FAE22081318142815381F8
:10A49000E5E7FAE25080418032802380E9E6FAE283
:10A4A0009080818072806380E5E6FAE28081898312
:10A4B00091819A83A281AB83B381BC83E1E6FAE206
:10A4C00080818D8391819E83A281AF83B381B88780
:10A4D000EDE5FAE28081898791819A87A281AB8735
:10A4E000B381BC87E9E5FAE280818D8791819E87FF
:10A4F000A281AF87B381B88BE5E5FAE28081898BD1
:10A5000091819A8BB280A380E1E5FAE2F080E1804C
:10A51000D280C380EDE4FAE2A081AB8BB181BC8B29
:10A52000128103810FB6F894DEBF0FBECDBF2BABF7
:10A530003CAB4DAB5EAB0E94845D5EA95F934DA9C1
:10A540004F933CA93F932BA92F932F923F924F9269
:10A550005F926F927F928F929F922C812F932B818B
:10A560002F932A812F9329812F9328852F932F8131
:10A570002F932E812F932D812F932C852F932B8515
:10A580002F932A852F9329852F9328892F932F8501
:10A590002F932E852F932D852F93AF92BF922A89CB
:10A5A0002F9329892F93CF92DF92EF92FF920F93EF
:10A5B0001F932C892F932B892F939F938F937F9396
:10A5C0006F93A3E1B8E28C911F928F93E2E1F8E2DE
:10A5D00080811F928F9382E19EE09F938F930E94D0
:10A5E000118B0FB6F894DEBF0FBECDBFE8960FB645
:10A5F000F894DEBF0FBECDBFDF91CF911F910F91B9
:10A60000FF90EF90DF90CF90BF90AF909F908F9092
:10A610007F906F905F904F903F902F90089580E3D0
:10A62000809303130895CF93DF936091031370E039
:10A63000C0E3D0E0C61BD70B6F5A7D4EAE010E941F
:10A64000648ACE01DF91CF910895CF92DF92EF928D
:10A65000FF920F931F93CF93DF937C01C09006135B
:10A66000D09007136091031370E0E601E096C61BDB
:10A67000D70BC138D105D8F400E310E0061B170B47
:10A680006F5A7D4EA8010E94648A60914F127091AA
:10A6900050128091041390910513680F791FA60141
:10A6A000C701800F911F0E94648ACE0102C080E022
:10A6B00090E0DF91CF911F910F91FF90EF90DF908D
:10A6C000CF90089590910313980F909303130895DA
:10A6D00040910613509107134817590798F020919D
:10A6E000041330910513280F391F3093051320935D
:10A6F0000413481B590B509307134093061381E032
:10A7000090E0089580E090E008959093071380937F
:10A710000613089580910413909105138F579D4E51
:10A7200008958091031390E08F5A9D4E089581E023
:10A7300090E020914F12309150122158324111F483
:10A7400080E090E008950E949753892B61F060911A
:10A750004F1270915012409106135091071381E8E7
:10A7600092E10C94648A2091041330910513211511
:10A770003105B9F08091061390910713C096E1E876
:10A78000F2E1AF01415552414817590734F4DF0156
:10A79000A20FB31F4C914193F4CF10920513109266
:10A7A0000413089580914F12909150120895809152
:10A7B00006139091071308959091031380E3891B6A
:10A7C000089520E380910313281B80910613909134
:10A7D0000713820F911D08951F93CF93DF93EC0110
:10A7E00010910313812F90E08C179D076CF00E944D
:10A7F000E1538C0F9D1F8138910530F41C1B109381
:10A80000031381E090E002C080E090E0DF91CF91FF
:10A810001F910895CF93DF93ECE1F8E2119211922A
:10A8200088E2EC34F807D1F7C4E1D8E261EF72E0D6
:10A83000CE010E949D4A229688E2CC31D807B1F71A
:10A84000DF91CF9108951092051310920413109286
:10A8500007131092061380E38093031381E892E1BB
:10A860009093501280934F120C940A54EF92FF92DF
:10A870000F931F93CF93DF9300D0CDB7DEB78C013A
:10A8800069837A830E9423546981E62E7A81F72EA8
:10A8900081E8E816F10418F080E8E82EF12CA70111
:10A8A000B80180914F12909150120E94648AF092E8
:10A8B0000713E0920613C7010F900F90DF91CF911D
:10A8C0001F910F91FF90EF9008950F931F93CF93D7
:10A8D000DF938C01EB010E942354109350120093DC
:10A8E0004F12D0930713C0930613DF91CF911F919E
:10A8F0000F91089520E3ECE1F8E2DC0101900D9264
:10A900002A95E1F788E0E4E1F8E2DB0101900D929D
:10A910008A95E1F7089520E3FC01ACE1B8E20190EB
:10A920000D922A95E1F788E0FB01A4E1B8E20190DD
:10A930000D928A95E1F70895E82FF0E0EE0FFF1FE2
:10A94000E45EF74D7183608381E090E00895E82F25
:10A95000F0E0EE0FFF1FE45EF74D808191810895D6
:10A9600090E0880F991F8C51984D0E949D4A81E07C
:10A9700090E0089590E0880F991F8C51984D0895AC
:10A980008115910511F00197F1F70895E0914F2895
:10A99000F0915028908180914E2889230895E0916C
:10A9A0004C28F0914D28808190914E28892B8083EE
:10A9B000E0915128F0915228808190914E28892B66
:10A9C00080830895E0914C28F0914D2890818091EA
:10A9D0004E28809589238083E0915128F091522858
:10A9E000908180914E2880958923808308951F93BC
:10A9F000CF93DF93E0914C28F0914D289081809186
:10AA00004E28809589238083E0915128F091522827
:10AA1000808190914E28892B80838FEB93E00E9458
:10AA2000C0541FB7F894E0915128F09152289081BA
:10AA300080914E2880958923808383E890E00E944E
:10AA4000C054E0914F28F0915028D081C0914E28F9
:10AA50001FBF78948BE393E00E94C054E0914F288D
:10AA6000F0915028908180914E28982319F08D2FD5
:10AA70008C2301C081E0DF91CF911F910895509305
:10AA800052284093512870934D2860934C289093FE
:10AA9000502880934F2881E001C0880F2A95EAF75B
:10AAA00080934E280C94F754CF93DF93C82FDFB7D1
:10AAB000F894E0915128F0915228808190914E288D
:10AAC000892B808383E090E00E94C054CC2351F016
:10AAD000E0915128F0915228808190914E289095D4
:10AAE0009823908387E190E00E94C054E0914F2822
:10AAF000F0915028808190914E28892309F4C0E07C
:10AB000089E590E00E94C054E0915128F0915228CC
:10AB1000808190914E28909598239083DFBF8BE39E
:10AB200090E00E94C0548C2FDF91CF910895CF9375
:10AB3000DF93C82FD8E08C2F81700E945455C695A2
:10AB40008111C068D150B9F78C2FDF91CF91089552
:10AB50008FEF0C949755DF92EF92FF920F931F9314
:10AB6000CF93DF93E82EEB010E94F75481112FC0A1
:10AB700080EF0E949755F12C10E488EFD82ED10E6B
:10AB800081E00E945455082F81E00E94545588238B
:10AB900019F0002361F01DC0011109C01E1528F035
:10ABA000888180FF04C0E11611F0F12E01E0802FB2
:10ABB0000E94545598819695011190689883115080
:10ABC0001D11DECF21961111D8CF8F2D03C08FEF2D
:10ABD00001C08EEFDF91CF911F910F91FF90EF9009
:10ABE000DF900895FF920F931F93CF93DF93F82E7A
:10ABF000EB010E94F754209769F085E50E94975574
:10AC00008E01085F1F4F89910E949755C017D10789
:10AC1000D1F703C08CEC0E9497558F2DDF91CF9117
:10AC20001F910F91FF900C9497550F931F93CF9303
:10AC3000DF93DB01EC9111969C911197F0E0F92BD9
:10AC4000803181F4BF016E7FE3E0660F771FEA95E4
:10AC5000E1F716969C911697ECE0F0E0E91BF109FC
:10AC6000E60FF71FF7FF07C091E0EA019883F1951F
:10AC7000E195F10902C0EA011882883279F414964C
:10AC80008C91982F9076903649F086FF02C0EE7F27
:10AC900005C085FF02C0EC7F01C0E87FCF0144E022
:10ACA000969587954A95E1F7D9018C93EF70E80165
:10ACB000E88380E0DF91CF911F910F9108950F936A
:10ACC0001F93CF93DF93EC018B01B80188810E9421
:10ACD000AB55888381508D3F30F4F80180818832F4
:10ACE00011F0803191F7DF91CF911F910F9108956D
:10ACF000CF93DF93EC010E94F754BE0184EB0E94D6
:10AD0000F25581E00E945455C82F0E94F75481E00B
:10AD1000C11101C080E0DF91CF9108951F93CF93BF
:10AD2000DF9300D0CDB7DEB7182F69837A830E94F6
:10AD3000F7540E94C65469817A81882341F084E4E3
:10AD40000E94F255113029F00E94CF5402C082E0D7
:10AD500001C080E00F900F90DF91CF911F91089577
:10AD60004F925F926F927F928F929F92AF92BF921B
:10AD7000CF92DF92EF92FF920F931F93CF93DF93C7
:10AD8000CDB7DEB729970FB6F894DEBF0FBECDBFA3
:10AD90006C015B014A0189010E94F754B6018EEBF8
:10ADA0000E94F255CE0101967C013E019AE0690EA7
:10ADB000711C27010E94A855F70181937F01E615B8
:10ADC000F705C1F769E070E0C2010E943E70811191
:10ADD00009C09401A501B201F60180810E941556B7
:10ADE00080E001C083E029960FB6F894DEBF0FBE65
:10ADF000CDBFDF91CF911F910F91FF90EF90DF902A
:10AE0000CF90BF90AF909F908F907F906F905F900A
:10AE10004F9008955F926F927F928F929F92AF9220
:10AE2000BF92CF92DF92EF92FF920F931F93CF9337
:10AE3000DF93CDB7DEB729970FB6F894DEBF0FBE0C
:10AE4000CDBF582E6B015A01890160E070E08EEB96
:10AE50000E94F255CE0101967C014E019AE0890EC6
:10AE6000911C37010E94A855F70181937F01E815D5
:10AE7000F905C1F769E070E0C3010E943E708111DD
:10AE800008C09501A601B301852D0E94155680E0EA
:10AE900001C083E029960FB6F894DEBF0FBECDBF88
:10AEA000DF91CF911F910F91FF90EF90DF90CF90A6
:10AEB000BF90AF909F908F907F906F905F9008951C
:10AEC0000F931F93CF93DF93CDB7DEB728970FB6BD
:10AED000F894DEBF0FBECDBF182F062F98E0EDEF20
:10AEE000F2E0DE01119601900D929A95E1F7242F80
:10AEF000332727FD309541E752E0249FC001259F6D
:10AF0000900D349F900D112464E670E00E947F84C0
:10AF1000CB0144E6049F800D911D1124FE01319662
:10AF2000AE01475F5F4F619170E02617370711F45C
:10AF3000019603C0E417F507B1F7112319F09195B5
:10AF40008195910928960FB6F894DEBF0FBECDBF4C
:10AF5000DF91CF911F910F910895EF92FF920F9380
:10AF60001F93CF93DF93CDB7DEB72B970FB6F8942F
:10AF7000DEBF0FBECDBFF82EE92E682F792F88E0F7
:10AF80008F0D0E948E56882319F084E391E243C00E
:10AF900066E471E48FE090E00E9418588E01075F2C
:10AFA0001F4F9801AE01465F5F4FBE01655F7F4F47
:10AFB0008F2D9E2D0E94B0568111E7CF88E0EDEFD6
:10AFC000F2E0DE01119601900D928A95E1F7498534
:10AFD00021E732E0429FC001439F900D112464E6B7
:10AFE00070E00E947F848A8594E6899F600D711DC0
:10AFF0001124FE0131968191481303C06F5F7F4F8A
:10B0000003C0E017F107B9F78B85882319F0719514
:10B0100061957109CB012B960FB6F894DEBF0FBE78
:10B02000CDBFDF91CF911F910F91FF90EF900895C9
:10B03000DC01CB0181159105A105B10529F08150F5
:10B040009040A040B040D9F708951092B90080E236
:10B050008093B800089594EA9093BC0040EA56E8C3
:10B0600061E070E09091BC0097FD0BC04150510928
:10B0700061097109411551056105710599F781E073
:10B0800008959091B900987F983011F09031B9F7F8
:10B090008093BB0084E88093BC0080EA96E8A1E03E
:10B0A000B0E02091BC0027FD08C00197A109B109BB
:10B0B0000097A105B105A9F7E2CF8091B900887F7B
:10B0C000883111F08034D9F680E0089524EA34E81C
:10B0D00044E92093BC009091BC0097FFFCCF909175
:10B0E000B900987F983011F0903199F78093BB00A8
:10B0F0003093BC009091BC0097FFFCCF9091B900B9
:10B10000987F903211F0983539F44093BC009091BB
:10B11000BC0094FDFCCFDDCF08950C942B5884E93E
:10B120008093BC008091BC0084FDFCCF0895809387
:10B13000BB0084E88093BC008091BC0087FFFCCFFB
:10B140009091B900987F81E0983209F480E00895E9
:10B1500084EC8093BC008091BC0087FFFCCF809181
:10B16000BB00089584E88093BC008091BC0087FFF9
:10B17000FCCF8091BB000895E0E1DC01FD91CD01A1
:10B18000F0933F01E150C9F780913C018F7D80939E
:10B190003C0180913C01877F80933C01FB0180E171
:10B1A000919190933E018150D9F780913C01806844
:10B1B00080933C0180913D0180FFFCCF40515109BB
:10B1C00080913C01806280933C0180913C01877FAB
:10B1D00080933C01141615069CF4FB0180E19191CB
:10B1E00090933E018150D9F780913C018068809313
:10B1F0003C0180913D0180FFFCCF40515109EACFD5
:10B20000F90180E190913E0191938150D9F781E05D
:10B2100090E008950F931F93CF93DF93EC018CE799
:10B220000E9466588CE70E9497588E01005F1F4F5E
:10B2300089910E949758C017D107D1F7DF91CF911C
:10B240001F910F910C948F58813019F440E050E019
:10B2500002C040EC50E060E070E08CE790E00C94BD
:10B260000C11813019F44EE050E002C048E050E08B
:10B2700060E070E08CE790E00C940C1141E050E04D
:10B2800060E070E08CE790E00E940C116AE67AE0E2
:10B2900080E090E00C94185848E350E060E070E0E3
:10B2A0008CE790E00E940C1149E350E060E070E010
:10B2B0008CE790E00E940C1144E150E060E070E007
:10B2C0008CE790E00E940C1148E750E060E070E0ED
:10B2D0008CE790E00E940C114EE550E060E070E0D9
:10B2E0008CE790E00E940C114DE650E060E070E0C9
:10B2F0008CE790E00E940C116CE17AE186E090E02E
:10B300000E9418584CE050E060E070E08CE790E05C
:10B310000E940C1141E050E060E070E08CE790E0AA
:10B320000E940C1146E050E060E070E08CE790E095
:10B330000E940C116AE67AE080E090E00C941858C4
:10B34000CF93DF93CDB7DEB7A2970FB6F894DEBFE9
:10B350000FBECDBF81E1E6EDF8E0DE01529601902F
:10B360000D928A95E1F781E1E7EEF8E0DE011196B2
:10B3700001900D928A95E1F70E944C59CE014296B8
:10B380000E940A5982E00E9424596AE67AE080E02D
:10B3900090E00E941858CE0101960E940A5960E17F
:10B3A0007EEA88E290E00E94185880E00E943159BD
:10B3B00060E17EEA88E290E00E9418584EE050E09A
:10B3C00060E070E08CE790E00E940C11A2960FB64E
:10B3D000F894DEBF0FBECDBFDF91CF910895CF921D
:10B3E000DF92EF92FF920F931F93CF93DF9300D0E2
:10B3F0001F92CDB7DEB7F82E042F122F213031F077
:10B40000223031F0243031F0283031F090E005C0A6
:10B4100091E003C092E001C093E00C3059F00E308F
:10B4200011F4946007C0003111F4986003C0023138
:10B4300009F49C60613059F0623011F4906207C0E9
:10B44000633011F4906403C0643009F4906690682E
:10B45000692F70E023E030E0AE014F5F5F4F8F2D2A
:10B4600090E00E94231169E07AE180E090E00E9480
:10B4700018588F2D8160F82E0E942B580E94A858D2
:10B4800089830E94A8588A83023119F40E94A8581F
:10B490008B830E94A85887FDF1CF0E94B2580E946A
:10B4A0008F5869E07AE180E090E00E9418588F2D73
:10B4B0000E942B580E94A85889830E94A8588A830A
:10B4C000023119F40E94B2588B830E94B2580E9434
:10B4D0008F5839812A81023149F5832F90E0A0E00D
:10B4E000B0E04B817727662731FF0EC030E0322F66
:10B4F0002227620F731F811D911D640F711D811D15
:10B50000911D8C6F9F6F0BC030E0322F2227620F8E
:10B51000731F811D911D640F711D811D911D0E945E
:10B520008C8120E83FEF4FEF57E420C0632F70E09D
:10B53000762F6627620F711D882777FD8095982FDB
:10B540000E948C810C3029F420E030EE4FEF54E45F
:10B550000DC00E3029F420E038EF4FEF55E406C05F
:10B56000003131F420E03EEF4FEF56E40E94ED80D1
:10B570002FE632E143E050E40E946A836B017C01D4
:10B58000612F70E080E090E00E948C819B01AC0113
:10B59000C701B6010E94ED800F900F900F90DF91D0
:10B5A000CF911F910F91FF90EF90DF90CF90089572
:10B5B000E6E4F1E08081208190813081829586955A
:10B5C0008695837022952F70822B832B92959F7086
:10B5D000892B08950F931F93CF93DF9300D0CDB79E
:10B5E000DEB746E06CE080E00E941A5E89E180935D
:10B5F000C4001092C50082E08093C00080E00E94E9
:10B60000A55E0E94465D84B784B784B784B784B7CB
:10B61000E3EDF0E322E432E4318320833A968DB700
:10B620009EB70A97E817F907B8F388EF98E09F9359
:10B630008F938EEC9FE09F938F930E94118B0E94BB
:10B64000816C0E94494C60E070E08BE792E00E94C0
:10B65000F14C0E942550E0910503F09106030995F5
:10B660000E94D85A90E00E94BD6CCE0101960E94C3
:10B670007B5C0F900F900F900F90882341F08EEA23
:10B680009FE09F938F930E94118B0F900F90CE019C
:10B6900001960E94B84A0E94895C8C010E94855CD8
:10B6A000AE014F5F5F4FB8010E9471610E94F55B70
:10B6B0000E9452610E948D5C0E94AB6281EA9FE011
:10B6C0009F938F930E94118B8A811F928F930DE914
:10B6D0001FE01F930F930E94118B89811F928F93FC
:10B6E0001F930F930E94118B8BE99FE09F938F9381
:10B6F0000E94118B0E94C16CE0914203F0914303C0
:10B700000995E0913403F09135030995E0911B030D
:10B71000F0911C0309950E94B262182F0E944F619C
:10B720001F921F931F928F93809141038F9380915B
:10B7300040038F93809133038F93809132038F93D3
:10B7400080E89FE09F938F930E94118BE0914C03C0
:10B75000F0914D030FB6F894DEBF0FBECDBF30970A
:10B7600091F00995BC0180E890E00E946B847F9382
:10B770006F938DE69FE09F938F930E94118B0F90A4
:10B780000F900F900F908BE69FE09F938F930E94F6
:10B79000118B60E070E081ED92E00E94F14C83EE4D
:10B7A00092E00E94916B83E69FE09F938F930E94AB
:10B7B000118B0F900F900F900F900F900F90DF91C3
:10B7C000CF911F910F9108957F936F939F938F93C4
:10B7D0008DE59FE09F938F930E94118B0F900F90A8
:10B7E0000F900F900F900F9008951F93CF93DF93BA
:10B7F000CDB7DEB7A0970FB6F894DEBF0FBECDBFB2
:10B8000085E390E00E944E8C182F282F35EF380FDB
:10B81000303108F0982F9095291709F461C089EE0E
:10B820009FE09F938F930E94118BEEE2F0E10F90C7
:10B830000F90DE01119684918D93319680E1E6336D
:10B84000F807C9F7F89448E050E061E570E0CE01F0
:10B8500001960E94548CE0E2F0E1DE0111968491A1
:10B860008D93319680E1EE32F807C9F74EE050E053
:10B8700063E470E0CE0101960E94548CE6E1F0E1B1
:10B88000DE01119684918D93319680E1E032F807C4
:10B89000C9F74AE050E069E370E0CE0101960E94EA
:10B8A000548C6DEC7BEA83E390E00E946C8C60E04A
:10B8B00070E081E390E00E946C8C60E080E390E0B7
:10B8C0000E945E8C60E070E087E390E00E946C8CE8
:10B8D0001AE16AE175EE85E390E00E946C8C789441
:10B8E000812FA0960FB6F894DEBF0FBECDBFDF91BB
:10B8F000CF911F910895F89442E050E061E570E027
:10B900000E94368C789480E0089583E390E00C9454
:10B910004E8C81E390E00C944E8C80E390E00C948C
:10B92000468C409161285091622860916328709103
:10B93000642890E0A0E0B0E0480F591F6A1F7B1F09
:10B940004093612850936228609363287093642821
:10B9500040915D2850915E2860915F287091602829
:10B96000480F591F6A1F7B1F40935D2850935E2824
:10B9700060935F28709360282091012A2223A1F010
:10B980004091592850915A2860915B2870915C2809
:10B99000480F591F6A1F7B1F4093592850935A28FC
:10B9A00060935B2870935C2808951F920F920FB6E6
:10B9B0000F9211240BB60F922F933F934F935F93E7
:10B9C0006F937F938F939F93AF93BF93EF93FF9367
:10B9D00080910A1390910B13019690930B1380930F
:10B9E0000A13809109138F5F809309138038A9F49B
:10B9F000109209138091612890916228A091632888
:10BA0000B09164280196A11DB11D80936128909387
:10BA10006228A0936328B09364288091012A882328
:10BA2000E1F0809108138F5F809308138038A9F4A8
:10BA3000109208138091592890915A28A0915B2860
:10BA4000B0915C280196A11DB11D80935928909357
:10BA50005A28A0935B28B0935C280E94814F892BC1
:10BA600011F00E94944EFF91EF91BF91AF919F9181
:10BA70008F917F916F915F914F913F912F910F9097
:10BA80000BBE0F900FBE0F901F901895F894109258
:10BA9000B60016BC83EF87BD82E084BD94E095BDFF
:10BAA00095B395BB80936E007894089580910A13A6
:10BAB00090910B1320910A1330910B138217930767
:10BAC000A9F70895009751F022E330E000002150DB
:10BAD000310921153105D1F70197F4CF08950F935E
:10BAE0001F93CF93DF93EC010E94565D8C010E945F
:10BAF000565D801B910B8C179D07C8F3DF91CF918A
:10BB00001F910F91089508950F931F9360916128DD
:10BB10007091622880916328909164280091612837
:10BB20001091622820916328309164286017710772
:10BB30008207930759F71F910F9108951F920F9253
:10BB40000FB60F9211241092A7020F900FBE0F9004
:10BB50001F9018951F920F920FB60F9211240BB6DB
:10BB60000F922F933F934F935F936F937F938F9396
:10BB70009F93AF93BF93EF93FF93E0919D02F0915A
:10BB80009E028081E091A802F091A902309709F00D
:10BB90000995FF91EF91BF91AF919F918F917F9107
:10BBA0006F915F914F913F912F910F900BBE0F902E
:10BBB0000FBE0F901F9018951F920F920FB60F9205
:10BBC00011241092B4020F900FBE0F901F90189581
:10BBD0001F920F920FB60F9211240BB60F922F9354
:10BBE0003F934F935F936F937F938F939F93AF9305
:10BBF000BF93EF93FF93E091AA02F091AB02808193
:10BC0000E091B502F091B602309709F00995FF91E5
:10BC1000EF91BF91AF919F918F917F916F915F91C4
:10BC20004F913F912F910F900BBE0F900FBE0F9031
:10BC30001F9018959DE0899FF0011124E356FD4F58
:10BC4000A281B3811C92A481B5816C93A681B78136
:10BC500088ED8C93A085B1854C931286148613864B
:10BC600008959DE0899FF0011124E356FD4F81E086
:10BC70008287A081B1816C933A9680818111FDCF3A
:10BC800008951F93CF93DF93182FEB01FE0164916A
:10BC9000662329F0812F0E94315E2196F7CFDF9134
:10BCA000CF911F9108951F93CF93DF93182FEB012E
:10BCB0008881882369F08A3021F46DE0812F0E9409
:10BCC000315E69916D30A1F3812F0E94315EF0CF1A
:10BCD000DF91CF911F910895CF93DF93CDB7DEB75A
:10BCE0009E01285F3F4F4E815F8160E470E08CE0F1
:10BCF00093E10E949F8B6CE073E18D810E94535E03
:10BD0000DF91CF910895CF93C82F8A3031F46DE041
:10BD100080914C130E94315E02C08D3029F06C2F4F
:10BD200080914C130E94315E80E090E0CF910895A5
:10BD30009DE0899FF0011124E356FD4F74876387CE
:10BD40000895682F80E00C94315E80934C138FE847
:10BD500092E09093CE308093CD30089584B7877F62
:10BD600084BF88E10FB6F894809360001092600061
:10BD70000FBE08952FE088E190E00FB6F894A895E3
:10BD8000809360000FBE209360000895A8950895E9
:10BD900088E10FB6F89480936000109260000FBEA7
:10BDA0000895F89428E088E190E00FB6F894A895FB
:10BDB000809360000FBE20936000FFCF80916C28BD
:10BDC00080916C2890E0089540E06FE181E491E07B
:10BDD0000C944764E9E3F1E0808180818D7F80836A
:10BDE0008DE090E00197F1F723E040E06FE182E41D
:10BDF00091E00E94516483E090E00197F1F708958B
:10BE00009091390191FD0AC0282F803108F02FE070
:10BE100040E06FE085E491E00C94516408958091D6
:10BE2000390181FD0EC040E06FE181E491E00E94A4
:10BE30004764282F2F7E81E090E0213021F080E0C0
:10BE4000089580E090E008958091390181FD10C04F
:10BE500040E06FE181E491E00E9447648F3131F06E
:10BE6000982F9F7E915081E0923018F480E00895E1
:10BE700081E008950E94245F8823E1F30895CF9321
:10BE8000DF93C82F0E943A5F0E94E45ED82FC81744
:10BE900089F1C83019F40E94EA5E25C0C93121F445
:10BEA000863189F429E005C0C63169F4893159F435
:10BEB00026E040E06FE182E491E00E945164E3E01B
:10BEC000F0E03197F1F72C2F40E06FE182E491E050
:10BED0000E945164D83019F4E9E6F1E002C0E3E0D1
:10BEE000F0E03197F1F70E94E45E8C1719F083E4DB
:10BEF00090E002C080E490E0DF91CF9108950E942D
:10BF00003A5F1092012A0E94EA5E809139018260B4
:10BF1000809339018091842A8823D9F180919400FB
:10BF2000909195004091952A5091962A84179507F3
:10BF3000A0F48091612A9091622AA091632AB09125
:10BF4000642A8C57914EAF4FBF4F8093612A9093D4
:10BF5000622AA093632AB093642A209194003091BE
:10BF60009500241B350B8091612A9091622AA09143
:10BF7000632AB091642A820F931FA11DB11D809383
:10BF8000612A9093622AA093632AB093642A109244
:10BF9000842A8091862A8823D9F1809194009091F7
:10BFA00095004091992A50919A2A84179507A0F4F8
:10BFB0008091692A90916A2AA0916B2AB0916C2A8B
:10BFC0008C57914EAF4FBF4F8093692A90936A2A46
:10BFD000A0936B2AB0936C2A209194003091950025
:10BFE000241B350B8091692A90916A2AA0916B2AB3
:10BFF000B0916C2A820F931FA11DB11D8093692AF5
:10C0000090936A2AA0936B2AB0936C2A1092862A86
:10C0100008958091012A882381F08091D0138111A5
:10C0200004C00E94245F811106C081E08093CE137A
:10C0300081E090E008950E947F5F80E090E00895A5
:10C04000809194009091950090939A2A8093992AD8
:10C0500021E02093862A8091390181FD08C08091DA
:10C06000390181FD1AC086E10E943F5F16C020930E
:10C07000002A80919400909195009093962A809345
:10C08000952A2093842A809139018D7F80933901EC
:10C090008091002A8111FCCFE2CF81E08093012AB8
:10C0A00008958091012A81110AC08091D0138823BC
:10C0B00021F081E08093CF1302C00E94206081E0D4
:10C0C00090E008951F93CF93DF931F92CDB7DEB713
:10C0D0008FB789838091D013811126C0F894809105
:10C0E000012A882351F08091390181FD1BC00E94F3
:10C0F000245F8823B9F080E003C00E94516081E092
:10C100002091470191E02E3008F090E0192F119511
:10C1100081110E940960107429F089818FBF81E02C
:10C1200090E004C089818FBF80E090E00F90DF91A4
:10C13000CF911F9108958091CF13882321F00E9401
:10C1400020601092CF138091CE13882321F00E949B
:10C150007F5F1092CE131092D01308950F931F9308
:10C16000AB0121E02093D0130091452A1091462A7B
:10C170002091472A3091482A0F5F1F4F2F4F3F4F82
:10C180000093452A1093462A2093472A3093482A41
:10C1900022E0260F27FF0CC08091FE299091FF29F5
:10C1A00001969093FF298093FE290FEF1FEF07C0A0
:10C1B000BC018DE493E10E94648A00E010E00E94DB
:10C1C0009B60C8011F910F9108958093D213089529
:10C1D0000E94E45E823011F0823111F480E0089513
:10C1E00081E0089508958FEF80934E0122E044E0AE
:10C1F00060EF8CE691E00E94516425E041E06EE042
:10C200008CE290E00E94516480E880936F018091FD
:10C21000460180936D0121E045E060E284E491E015
:10C220000C9451648DEF93E00197F1F70E943D6407
:10C23000109275281092F72810927929109274287C
:10C2400010927328E9E3F1E080818E7F8083808102
:10C250008D7F80838DE090E00197F1F7E9E3F1E0D5
:10C2600080818160808323E040E06FE182E491E09F
:10C270000E9451648DEF93E00197F1F780915D0189
:10C2800080915E010E94F36060E070E087EB92E0D5
:10C290000E94F14C0E94206081E090E0089580911E
:10C2A000D1130895CF93DF931F92CDB7DEB7898363
:10C2B0000E943A5F89818093D113282F40E06FE17B
:10C2C00088E491E00F90DF91CF910C9451640E942B
:10C2D00052618091390181FD03C086E00C943F5F7B
:10C2E0000895FA0180936201909363016093600165
:10C2F000709361013097C1F0808180936B018181DF
:10C3000080936A01828180936901838180936801AF
:10C310008481809367018581809366018681809303
:10C320006501878180936401089587EB92E00E9404
:10C33000124D81E080936C2880916D2890916E2839
:10C34000019690936E2880936D2881E090E0089587
:10C350008091742892E8899FF0011124EB58F74DE1
:10C3600010828F5F833018F48093742802C010927B
:10C370007428E091742882E8E89FF0011124EB58BA
:10C38000F74D808181110C94956110926C2808956D
:10C390001F93CF93DF932091742812E8129F90018E
:10C3A0001124D901AB58B74D4C91411103C00E94E3
:10C3B000A86193C05091390151FD8FC05091012A5D
:10C3C000552309F48AC047FF16C00E94A8618091D6
:10C3D000352A9091362AA091372AB091382A0196B1
:10C3E000A11DB11D8093352A9093362AA093372A38
:10C3F000B093382A72C04330B0F40E94A861809193
:10C40000312A9091322AA091332AB091342A019690
:10C41000A11DB11D8093312A9093322AA093332A13
:10C42000B093342A5AC050E0EA0122976C177D0776
:10C43000B0F40E94A86180912D2A90912E2AA0919B
:10C440002F2AB091302A0196A11DB11D80932D2A6B
:10C4500090932E2AA0932F2AB093302A3EC0B90180
:10C460006A58774D0E94648AE09174281E9FF001FB
:10C470001124EB50F74D8081809365280E94A861BC
:10C48000809147018093662890916B28992311F041
:10C49000891710F480936B286091662870E084E01F
:10C4A0000E949C546091652870E083E00E949C5437
:10C4B0004091492A50914A2A60914B2A70914C2A06
:10C4C0004F5F5F4F6F4F7F4F4093492A50934A2AE7
:10C4D00060934B2A70934C2A02C0C0E0D0E0CE019A
:10C4E000DF91CF911F910895CF93DF93EC01888165
:10C4F00099810097E9F08730954021F019821882E0
:10C5000083E026C06238C1F410926C280E94235444
:10C510000E948A5360E870E00E94C86118161906EC
:10C520006CF40E948553E0914603F091470309950E
:10C5300087E095E09983888381E00AC0809169282B
:10C5400090916A28019690936A2880936928F0CF89
:10C55000DF91CF91089591E09093D0130E94005FF6
:10C560000C949B608091390181FD06C040E06FE032
:10C5700085E491E00C94476480E108950F931F9344
:10C58000CF93DF93182F21E02093D0130091012A3D
:10C590008091390181FF16C080919400909195009F
:10C5A0009093962A8093952A2093842A2093002A98
:10C5B000809139018D7F809339018091002A81110A
:10C5C000FCCF00E00E943A5F8091012A882309F4A1
:10C5D0003FC08091862A8823D9F180919400909160
:10C5E0009500E091992AF0919A2A8E179F07A0F45E
:10C5F0004091692A50916A2A60916B2A70916C2A45
:10C600004C57514E6F4F7F4F4093692A50936A2A7F
:10C6100060936B2A70936C2A20919400309195005E
:10C620002E1B3F0B4091692A50916A2A60916B2A18
:10C6300070916C2A420F531F611D711D4093692A2E
:10C6400050936A2A60936B2A70936C2A1092862A00
:10C650008091390181FD03C089E10E943F5F86E03E
:10C660000E94A754892B51F00E94B262C82F86E025
:10C670000E94A75481500E94005F02C0C0E0D0E039
:10C6800020919400309195003093982A2093972A16
:10C6900081E08093852AF8948091390182608093AB
:10C6A0003901809139018D7F8093390162E0610FFA
:10C6B0008DE493E10E94826478942091FB2930916B
:10C6C000FC292F5F3F4F3093FC292093FB290E94C8
:10C6D0003A5F45E060EE82E491E00E944764182FE3
:10C6E00086E00E94A754892B19F08C2F0E94005FCE
:10C6F000002319F00E94206002C00E947F5F809199
:10C70000852A8823D9F18091940090919500E09139
:10C71000972AF091982A8E179F07A0F44091652AD6
:10C720005091662A6091672A7091682A4C57514E41
:10C730006F4F7F4F4093652A5093662A6093672A14
:10C740007093682A20919400309195002E1B3F0B26
:10C750004091652A5091662A6091672A7091682AF3
:10C76000420F531F611D711D4093652A5093662A25
:10C770006093672A7093682A1092852A8091012A13
:10C78000882361F0209194003091950030939A2A8B
:10C790002093992A81E08093862A07C023E040E015
:10C7A0006FE182E491E00E9451640E949B6011302D
:10C7B000E9F01330A9F480913D2A90913E2AA0918E
:10C7C0003F2AB091402A0196A11DB11D80933D2AB8
:10C7D00090933E2AA0933F2AB093402A12E009C0CA
:10C7E000153031F0173029F411E003C010E001C01A
:10C7F00013E0812F90E0DF91CF911F910F91089569
:10C80000CF93DF93EB010E94AE60009729F4CE0135
:10C810000E94BE62009751F02091FE293091FF29BD
:10C820002F5F3F4F3093FF292093FE29DF91CF9157
:10C830000895CF93DF938091012A811104C00E9453
:10C840005160D1E001C0D0E00E94E45E863111F079
:10C85000813119F4C091470109C040E06FE186E4DD
:10C8600091E00E944764C82FCC0FC80FD1110E94DD
:10C8700009608C2FDF91CF9108951092D4131092FC
:10C88000D313EFE6F0E08081806280830895FC019D
:10C890008081862390E002C0959587954A95E2F7BE
:10C8A0000895F894FC015081362F30955323042EBF
:10C8B00001C0220F0A94EAF72623522B5083789462
:10C8C000089540917B01FC014193A0E8B1E050E85C
:10C8D000540F9D012F5F3F4F6C916193521711F0E0
:10C8E000D901F7CF4150E42FF0E0E058FE4F21810D
:10C8F000FC01E058FF4F2083FC01EF57FF4F21E080
:10C900002083089560938001E1E8F1E061589F0180
:10C910002F5F3F4FDC014D91CD014083621711F035
:10C92000F901F5CF08951F920F920FB60F921124BF
:10C930000BB60F922F933F934F935F936F937F9319
:10C940008F939F93AF93BF93EF93FF938091470192
:10C95000809366288091732822E8829FC001112469
:10C960008B58974D0E946164809173288F5F83304C
:10C9700018F48093732802C0109273280E94956166
:10C98000FF91EF91BF91AF919F918F917F916F91A7
:10C990005F914F913F912F910F900BBE0F900FBE63
:10C9A0000F901F9018951F920F920FB60F9211249F
:10C9B0000F900FBE0F901F9018951F920F920FB6F9
:10C9C0000F9211240F900FBE0F901F9018951F9279
:10C9D0000F920FB60F9211240F900FBE0F901F9061
:10C9E00018951F920F920FB60F9211241092002AE1
:10C9F0000F900FBE0F901F9018951F920F920FB6B9
:10CA00000F9211241092002A0F900FBE0F901F90CA
:10CA100018951F920F920FB60F9211248F9381E0F9
:10CA200080936C288F910F900FBE0F901F901895D8
:10CA30001F920F920FB60F9211241092002A0F909E
:10CA40000FBE0F901F9018951F920F920FB60F9266
:10CA500011248F939F938091D3139091D4130196B7
:10CA60009093D4138093D3139F918F910F900FBE07
:10CA70000F901F901895CF92DF92EF92FF920F9335
:10CA80001F93CF93DF937C018B016A0185ED93E1C6
:10CA90000E94B14DEC01009751F0EC81FD8130977F
:10CAA00011F0C8010995CE010E94594EF3CFA6019D
:10CAB000B801C701DF91CF911F910F91FF90EF90C7
:10CAC000DF90CF900C943B4B0F931F93CF93DF934A
:10CAD00000D0CDB7DEB78091092A90910A2AA091A3
:10CAE0000B2AB0910C2A0196A11DB11D8093092A31
:10CAF00090930A2AA0930B2AB0930C2A0E94CE6727
:10CB00008C0185ED93E10E94B14D009779F0DC0135
:10CB10001296ED91FC911397309729F089839A83AF
:10CB200009959A8189810E94594EEFCF011511050F
:10CB300049F0C8010F900F90DF91CF911F910F9195
:10CB40000C94324B0F900F90DF91CF911F910F916A
:10CB500008950E94C16C0E9423540E94F56582E3EF
:10CB600093E09093042A8093032A0E94CC672FEFCE
:10CB700031E040E05EE160E074E082E090E00C943F
:10CB80009567BC0185ED93E10C94114EBC0185EDD8
:10CB900093E10C94F64DCF93DF93EC014091052A7D
:10CBA0005091062A6091072A7091082A4F5F5F4FC3
:10CBB0006F4F7F4F4093052A5093062A6093072AB0
:10CBC0007093082A0E94E167009761F00E94A353C6
:10CBD000E0913603F0913703BE018BE395E60995AA
:10CBE00081E090E0DF91CF9108958BED93E10C947B
:10CBF000AD4D0F93CF93DF93EC017B836A8318864F
:10CC00005F834E83BC018BED93E10E94114EE09156
:10CC1000D713F091D813309749F04C815D8101E032
:10CC200020E030E068858A819B810995DF91CF9172
:10CC30000F910895BC018BED93E10C94F64D0F9389
:10CC4000DC0118961C921897E091D713F091D81335
:10CC5000309759F000E020E030E040E050E060E044
:10CC600012968D919C91139709950F9108950F93AA
:10CC7000DC01AB0114962D913C91159781E018963B
:10CC80008C93189715967C936E931497E091D71315
:10CC9000F091D813309739F000E061E012968D9151
:10CCA0009C91139709950F9108950F93DC01E091E2
:10CCB000D713F091D813309771F014964D915C9181
:10CCC000159701E09A0118966C91189712968D911C
:10CCD0009C91139709950F910895E091D913F091C4
:10CCE000DA13309709F0099408959093DA1380933A
:10CCF000D91308959093D8138093D71308958BED8B
:10CD000093E10C94B14DEF92FF920F931F93CF9349
:10CD1000DF938C01EB017A018BED93E10E94B14D21
:10CD20000097D9F0DC0112962D913C9113972C17A6
:10CD30003D0781F41696ED91FC911797309769F0B5
:10CD40009701AE01B801DF91CF911F910F91FF9034
:10CD5000EF9009940E94594EE3CFDF91CF911F913C
:10CD60000F91FF90EF9008950895CF93DF93CEE059
:10CD7000D4E16881798120E030E044ED56E688EF27
:10CD800093E10E9431500E94BF6C688179810E94BA
:10CD90006B8420E030E048EE56E6BC0188EE93E17B
:10CDA000DF91CF910C94315080910E1490910F141B
:10CDB00020910C1430910D14880F991F28173907F2
:10CDC00008F4C90190930F1480930E140C94B56667
:10CDD000CF93DF930E9423540E948A53EC0119825F
:10CDE00018820E947F6628813981009719F1FC0121
:10CDF00040854423F9F0FC0142815381F901EE0F93
:10CE0000FF1FEE0FFF1FEC0FFD1F53834283FC013A
:10CE1000448155812F5F3F4FF901EE0FFF1FEE0F49
:10CE2000FF1FEC0FFD1F51834083398328830E942D
:10CE3000594ED9CFC901880F991F880F991F0296A3
:10CE40000E94855388819981892B31F08DED93E182
:10CE5000DF91CF910C94094BDF91CF910895AF9260
:10CE6000BF92CF92DF92EF92FF920F931F93CF93D7
:10CE7000DF9300D0CDB7DEB76B010E948A53FC016F
:10CE8000008111811A8309830C30110518F4E12CFB
:10CE9000F12C0DC01F930F9386E199E09F938F9320
:10CEA0000E94FF8A0F900F900F900F9021C0E01604
:10CEB000F106F1F00E948A53F701EE0FFF1FEE0F0B
:10CEC000FF1FE80FF91FA280B3800E948A53FFEF73
:10CED000EF1AFF0AF701EE0FFF1FEE0FFF1FE80F1B
:10CEE000F91F40815181B501C6010E948366DFCFE1
:10CEF0000F900F90DF91CF911F910F91FF90EF90C6
:10CF0000DF90CF90BF90AF9008950F93013059F408
:10CF1000809108149091091490930F1480930E142B
:10CF20000F910C94B5660F910895EF92FF920F93B5
:10CF30001F93CF93DF938B01EA0179014FE153E017
:10CF4000BC018DED93E10E94ED4A1093091400930A
:10CF50000814D0930B14C0930A14F0920D14E092AD
:10CF60000C1485E897E6DF91CF911F910F91FF9008
:10CF7000EF900C947A6688EF93E10E94B55088EEAA
:10CF800093E10E94B5508DED93E10C94074B809195
:10CF90000E1490910F1408950C94474BCF93DF9388
:10CFA000E0912303F09124030995EC01009729F007
:10CFB0006A817B8181E00E949C54CE01DF91CF91F8
:10CFC00008950F931F93CF93DF93EC01E091250316
:10CFD000F091260309958C016A817B8181E00E9492
:10CFE0009C5481E090E0012B11F480E090E0DF910F
:10CFF000CF911F910F910895E0912703F09128039D
:10D00000099420E030E00296FC01329740814423ED
:10D0100031F0FC0131974081240F311DF4CFC9015B
:10D020000895FC01208130E0322F22278181282BB6
:10D0300002C0220F331F6A95E2F7832F9927FA0166
:10D04000E75DFC4F208130E08223932328E030E02D
:10D05000241B350B02C0969587952A95E2F7089513
:10D060006F927F928F929F92AF92BF92CF92DF92F8
:10D07000EF92FF920F931F93CF93DF938C01EB01FD
:10D080006A0179012830310524F4A901B601CE01E5
:10D090004AC0590123E0B594A7942A95E1F74115B8
:10D0A000510521F04801612C712C03C0D801FB010E
:10D0B00020C048E050E0B601CE01860D971D0E94C9
:10D0C0001168F40181934F01FFEF6F1A7F0A6A1410
:10D0D0007B047CF3C501B7FE02C080E090E0A701AD
:10D0E000477055274115510511F1080F191FB60159
:10D0F00018C0CF018C1B9D0B8A159B051CF48191D8
:10D100008D93F7CFC501B7FE02C080E090E0A70184
:10D11000477055274115510551F0080F191F60E060
:10D1200070E08C0F9D1F0E941168F8018083DF91D1
:10D13000CF911F910F91FF90EF90DF90CF90BF9014
:10D14000AF909F908F907F906F9008958F929F9255
:10D15000AF92BF92CF92DF92EF92FF920F931F9305
:10D16000CF93DF9300D0CDB7DEB70E948A538C01F6
:10D1700082E090E00E946853892B19F480E090E0EF
:10D180005DC0F801818190E0982F88272081820F6F
:10D19000911D0E94584B7C01009781F30E948A5395
:10D1A0004C01F7012681822F86958695869590E021
:10D1B000422F477021E030E011F420E030E0820F90
:10D1C000931F0E946853892BC9F2F70104811581CE
:10D1D000C12CD12CF8018081882379F1F801A1803C
:10D1E000B12CB60133E0759567953A95E1F7A60144
:10D1F00047705527680D791D883168F09501CE017B
:10D2000001960E943068BE016F5F7F4FF8018081F8
:10D210000E94B0540DC01A8219829501CE01019668
:10D220000E94306869817A81F80180810E949C5453
:10D23000CA0CDB1C0E5F1F4FCDCFC7010F900F90A4
:10D24000DF91CF911F910F91FF90EF90DF90CF90E2
:10D25000BF90AF909F908F900895DC0150E0E0E187
:10D26000F0E0E61BF70BE21BF30B02C0440F551F67
:10D27000EA95E2F78C91852B8C9311968C911197FE
:10D28000842B11968C9308956F927F928F929F9228
:10D29000AF92BF92CF92DF92EF92FF920F931F93C4
:10D2A000CF93DF938C016B01EA01790128303105BE
:10D2B0001CF44881C8015CC0390153E0759467943F
:10D2C0005A95E1F76115710521F04E01A12CB12CA1
:10D2D00003C0D801FE0127C0F40141914F0128E0AD
:10D2E00030E0B601C8018A0D9B1D0E942D69FFEF39
:10D2F000AF1ABF0AA614B7047CF3C30177FE02C0BD
:10D3000080E090E09701277033272115310509F45B
:10D310003FC0C80FD91F488150E0B601621B730B94
:10D32000685F7F4F1CC0CF018C1B9D0B8615970536
:10D330001CF481918D93F7CFC30177FE02C080E08A
:10D3400090E09701277033272115310509F1C80FA7
:10D35000D91F488150E068E070E0621B730B02C087
:10D36000559547956A95E2F760E070E0800F911F50
:10D37000DF91CF911F910F91FF90EF90DF90CF90B1
:10D38000BF90AF909F908F907F906F900C942D697D
:10D39000DF91CF911F910F91FF90EF90DF90CF9091
:10D3A000BF90AF909F908F907F906F9008956F92F5
:10D3B0007F928F929F92AF92BF92CF92DF92EF9225
:10D3C000FF920F931F93CF93DF9300D0CDB7DEB7BB
:10D3D0008C01FC018681E82EE694E694E694F12C1B
:10D3E000282F277081E090E011F480E090E0E80EB3
:10D3F000F91EC70102960E94EC53009709F445C03C
:10D400000E949153F8012281FC012083F8012381BD
:10D41000FC0121830E94915302965C01A70160E008
:10D4200070E00E946D8AF80104811581E12CF12CD5
:10D43000F8018081882339F1F8018180912C6701FE
:10D4400063E0D594C7946A95E1F73701F7E06F225E
:10D450007724CA0CDB1C883128F00E94BA5494014E
:10D46000AC0108C00E94A7549A8389839401AE013D
:10D470004F5F5F4FB301C6010E944469E80CF91C7D
:10D480000E5F1F4FD5CF81E090E00F900F90DF919E
:10D49000CF911F910F91FF90EF90DF90CF90BF90B1
:10D4A000AF909F908F907F906F900895E09144038C
:10D4B000F09145030994E0911D03F0911E03099436
:10D4C000E0914803F09149030994E0914A03F091F7
:10D4D0004B03099480E090E008950895E0911503CE
:10D4E000F0911603099480E090E008950F931F9344
:10D4F000CF93DF93CDB7DEB7E0970FB6F894DEBFDA
:10D500000FBECDBF0E94D7538C010E948A53AE013B
:10D510004F5F5F4F602F0E944672882309F446C018
:10D5200088A99801281B3109C9010E946853892BD9
:10D53000E9F12E8121110CC0BE016A5E7F4F88E1A6
:10D540000E94B054E0913803F091390309952EC040
:10D550008A859B858D3C3BEA930711F0019631F556
:10D56000223019F088E090E002C082E090E001975C
:10D570009C012F5F3F4F12161306F4F6E1E0F0E036
:10D58000EC0FFD1FE80FF91F23852F3F81F3BE012C
:10D59000645F7F4F89E10E94B05489E10E94BA54D0
:10D5A00062E178E20E94A64A892B31F6E0960FB636
:10D5B000F894DEBF0FBECDBFDF91CF911F910F91C9
:10D5C0000895AF92BF92CF92DF92EF92FF920F93A6
:10D5D0001F93CF93DF93CDB7DEB7E0970FB6F894E4
:10D5E000DEBF0FBECDBF8C016B01CE0101967C0169
:10D5F00080E3F70111928A95E9F781E089838CE055
:10D600000E94A7548C831D821F828091121491E086
:10D61000980F90931214898783E0B82EB8868DEC0A
:10D620009BEA9B878A8789E10E94BA5461EF72E086
:10D630000E94A64A892B31F082E08E838FEF8C877F
:10D640008D8709C089E10E94BA54BC01CE010C96B5
:10D650000E949D4ABE828DEC9BEA9D8B8C8B62E181
:10D6600078E2CE0146960E949D4A0E948A539FA767
:10D670008EA70E94D75388ABC7010E943F71B82E76
:10D6800090E00E94EC53892B31F10E949153BC0130
:10D690004B2DC7010E945D71E0900B03F0900C03CD
:10D6A0000E94E1535C010E949153B501F701099575
:10D6B0000115110581F0009739F0019761F441E0FF
:10D6C00050E064E070E004C041E050E060E070E0F1
:10D6D000C601F8010995E0960FB6F894DEBF0FBEBB
:10D6E000CDBFDF91CF911F910F91FF90EF90DF9011
:10D6F000CF90BF90AF9008950E94BF6C809312149A
:10D70000E0911503F09116030994892B29F0E0911B
:10D710001503F091160304C0E0911703F09118036C
:10D720000994CF93DF93EC0189919991009729F0A7
:10D7300060E070E00E94F14CF7CFDF91CF91089547
:10D74000CF93DF93EC0189919991009719F00E9492
:10D75000434CF9CFDF91CF910895CF93DF93EC0144
:10D760007B836A830E94565D99838883DF91CF9182
:10D770000895FC018081918122813381820F931F62
:10D78000918380830895CF93DF93EC010E94565DCF
:10D7900099838883DF91CF910895CF93DF93EC0134
:10D7A0000E94565D28813981821B930B9C012F5F5B
:10D7B0003F4F81E090E04A815B814217530710F0B0
:10D7C00080E090E0DF91CF910895CF93DF93FC014B
:10D7D000C281D38180819181C80FD91F0E94565D7B
:10D7E0009E01281B390BC901DF91CF910895CF937A
:10D7F000DF93EBE8FAE2CDE4DAE2AFE7BAE21192C6
:10D80000119219921992199219921D928AE2E33A91
:10D81000F807A9F7DF91CF910895CF93DF93FC012B
:10D82000E158F54D40819C01220F331F220F331F19
:10D83000442301F1A0919400B0919500FC01EE0FFA
:10D84000FF1FE557F54D80819181AD01481B590BB4
:10D85000CA01E901C35BD54D488159816A817B8149
:10D86000480F591F611D711D488359836A837B834B
:10D87000B183A083F901E35BF54D60817181828101
:10D880009381DF91CF91089560E070E0CB0108951E
:10D89000FC01EE0FFF1FEE0FFF1FE35BF54D408312
:10D8A0005183628373830895CF93DF932FE73AE226
:10D8B000CDE4DAE2EBE8FAE2D9018D919D0188230B
:10D8C000B9F0409194005091950080819181BA0106
:10D8D000681B790B88819981AA81BB81860F971F6C
:10D8E000A11DB11D88839983AA83BB835183408383
:10D8F00024963296BAE22B383B07F1F6DF91CF91AE
:10D9000008950C94CE700F931F93FC01CB014091AE
:10D910001314509114143383228315830483718369
:10D920006083F0931414E0931314452B11F40E94B8
:10D93000E87080E090E01F910F910895809113149A
:10D94000909114140097C1F01092141410921314B3
:10D95000DC0114966D917C9115971296ED91FC91D6
:10D9600013970995E0911314F0911414309721F056
:10D97000808191810C94E87008950C94F7860C9442
:10D98000F38689EC92E00E94284D81EC92E00C94A1
:10D99000284DCF93DF930E949753892BA9F081ECF8
:10D9A00092E00E94464DEC01009721F10E94D7536E
:10D9B000998388830E94D2539B838A83CE010496E5
:10D9C0000E9413538CAB14C089EC92E00E94464D28
:10D9D000EC01009779F002960E9425539983888381
:10D9E000BE016E547F4FCE018E579F4F0E947A54D6
:10D9F000CE0102C080E090E0DF91CF910895BC019C
:10DA00006E547F4F8E579F4F0C947A54CF93DF9371
:10DA1000EC01BC0189EC92E00E94904DBE01892B83
:10DA200019F089EC92E009C081EC92E00E94904DDF
:10DA3000892B39F0BE0181EC92E0DF91CF910C94FB
:10DA40006B4DDF91CF9108950F931F93CF93DF9389
:10DA5000EC01BC0189EC92E00E94904D892B91F081
:10DA6000FE0161917191CF010E943654BE016E5446
:10DA70007F4FCE018E579F4FDF91CF911F910F9116
:10DA80000C948B54BE0181EC92E00E94904D892B46
:10DA9000D1F00E942354688179818A819B810E9400
:10DAA00036548CA990E00E94EC530CA910E00E941F
:10DAB0009153BE016C5F7F4FA801DF91CF911F9101
:10DAC0000F910C94648ADF91CF911F910F9108956B
:10DAD000CF93DF93EC01BC0189EC92E00E94904D62
:10DAE000892B19F0CE0102960CC0BE0181EC92E0A8
:10DAF0000E94904D892B19F08A819B8102C080E0A1
:10DB000090E0DF91CF910895FC018081918108958B
:10DB1000860F911D860F911D8E579F4F0895860F7A
:10DB2000911D860F911D8E579F4FFC018081918121
:10DB30000895089582E79AE10E946A4F892B21F0A7
:10DB400082E79AE10C94574F0895E0915E1AF091A4
:10DB50005F1A309709F0099480E00895EF92FF92E0
:10DB60000F931F93CF93DF937C01EA01FC01808127
:10DB70009181009741F08C30934071F1F70111824F
:10DB8000108283E0F2C080E024E0829FF001112443
:10DB9000E05AF54E118210828F5F8430A8F3809393
:10DBA0005D1A80919811909199119093711A8093B8
:10DBB000701A0E943C4C8093A32A60E470E082E7D4
:10DBC0009AE10E94434F0E94BC738CE093E0F701FE
:10DBD0009183808381E0C9C06230D9F48091A42A06
:10DBE0009091A52A892B89F38091B52A863029F452
:10DBF0008091CD2A81FD0E949A6D81E00E94FA7485
:10DC00008091A42A9091A52A892BF9F20E94BE6FD7
:10DC1000DCCF633060F5611114C02097B1F2D0936E
:10DC2000B22FC093B12F83E00E94FA748091A42A8E
:10DC30009091A52A892B11F00E94A56D0E949A6DE2
:10DC4000C4CF613011F6209709F4BFCFD093AE2F27
:10DC5000C093AD2F85E00E94FA748091A42A909120
:10DC6000A52A892B09F4B1CF0E94A56DAECF6738E4
:10DC7000E9F510925C1A00E61AE180915C1A843092
:10DC8000B8F4F801828193818C179D0749F4808153
:10DC900091810E94C774F80111821082138212824E
:10DCA0000C5F1F4F80915C1A8F5F80935C1AE5CFE9
:10DCB000ECECFFE2838194818C179D0719F41482A8
:10DCC00013821082B09620E3EC34F20799F7E9E46E
:10DCD000F0E3818592858C179D0711F415821482DB
:10DCE0003D9680E3EB3CF807A1F76FCF683809F069
:10DCF0006CCFC257DA4109F068CF82E79AE10E94FF
:10DD00006A4F892B09F461CF10925C1AE0915C1A7A
:10DD1000E43008F05ACF20E2E29FF0011124ED54E4
:10DD2000F04D818D8823D9F082E79AE10E94574F08
:10DD300080915C1AE0E28E9FC00111248D54904DB9
:10DD40009093B22F8093B12F82E00E94FA74809159
:10DD5000A42A9091A52A892B11F00E94A56D80918B
:10DD60005C1A8F5F80935C1AD1CFDF91CF911F91A6
:10DD70000F91FF90EF90089590935F1A80935E1A31
:10DD80000895209198113091991160E0E0E6FAE150
:10DD9000643098F4408151814817590759F4428101
:10DDA00053814217530731F460935B1A118210823A
:10DDB0000C94C77434966F5FEBCF60935B1A089531
:10DDC00040E0E0E6FAE14430A8F451E0540F20814D
:10DDD0003181232B61F440935A1A918380832091DF
:10DDE000981130919911338322830C94E174349605
:10DDF000452FE9CF40935A1A0895209198113091F8
:10DE00009911FC01358F248F778F668F08952091AB
:10DE1000981130919911FC013287218774876387AB
:10DE20000895CF93DF93EA010E946A74009749F046
:10DE30002091981130919911FC0132872187D48764
:10DE4000C387DF91CF9108950F931F93CF93DF93F3
:10DE500000D000D0CDB7DEB78C01AB018FEF898346
:10DE60008A838B838C83B801CE0101960E94116F47
:10DE7000009719F0FC01158304830F900F900F9009
:10DE80000F90DF91CF911F910F91089540E050E0E6
:10DE900062E081ED92E00E94E24C1092A52A10927D
:10DEA000A42A0895AC0161E081ED92E00C94C44C89
:10DEB000AC0160E081ED92E00C94C44C0F931F9391
:10DEC000CF93DF938A010E94E873EC01009759F029
:10DED00080919811909199119D8F8C8F1F8F0E8F2B
:10DEE000CE010E94586FCE01DF91CF911F910F910B
:10DEF0000895CF93DF93A091B12FB091B22F1097D7
:10DF000019F0ED016C9605C0C091AD2FD091AE2FE8
:10DF100029968091AC2F86FF22C01092591A40E0BA
:10DF2000E0E6FAE14430B8F42081318114968D9115
:10DF30009C9115972817390759F48281938100978E
:10DF400039F04093591A998388831B821A8205C03D
:10DF500034964F5FE7CF4093591A0E949A6D88819B
:10DF60009981009741F04A815B816091A32ADF91FA
:10DF7000CF910C94E24CDF91CF9108950F931F93B2
:10DF8000CF93DF938091B52A863009F071C08091DC
:10DF9000A42A9091A52A8115954009F069C0C4E989
:10DFA000D2E0D093A52AC093A42A02E00093AE2A1F
:10DFB00014E91093AF2A1092D12A1092D02A0E940D
:10DFC000B673809590959093D12A8093D02A109221
:10DFD000B72A1092B62A0E94A573809590959093C7
:10DFE000B72A8093B62A0E94A56DD093A52AC09324
:10DFF000A42A0093AE2A1093AF2AA091AF2FB0911C
:10E00000B02FFD01E459FD4F8CE692E001900D9296
:10E010000197E1F76CE672E084EC9AE20E94647387
:10E020008091A82A8093C42A8091A92A8093C52A26
:10E030008091AA2A8093C62A8091AB2A8093C72A0E
:10E040001092D12A1092D02A0E94B6738095909592
:10E050009093D12A8093D02A1092B72A1092B62A90
:10E060000E94A573809590959093B72A8093B62AC5
:10E07000DF91CF911F910F910C94A56DFC01680F5A
:10E08000791F80E048E1E617F70781F0219198E0D9
:10E09000322F3827532F517030FD84278695513009
:10E0A00009F480682695915099F7EDCF08951F9255
:10E0B0000F920FB60F9211240BB60F922F933F932E
:10E0C0004F935F936F937F938F939F93AF93BF9380
:10E0D000EF93FF9380919400909195009093902AF4
:10E0E00080938F2A81E08093812A80917100807DC6
:10E0F000809371000E949E6C8091812A8823D9F1BF
:10E10000809194009091950040918F2A5091902A8F
:10E1100084179507A0F48091552A9091562AA091D2
:10E12000572AB091582A8C57914EAF4FBF4F8093CA
:10E13000552A9093562AA093572AB093582A209193
:10E14000940030919500241B350B8091552A9091B5
:10E15000562AA091572AB091582A820F931FA11DC9
:10E16000B11D8093552A9093562AA093572AB093B5
:10E17000582A1092812AFF91EF91BF91AF919F9100
:10E180008F917F916F915F914F913F912F910F9060
:10E190000BBE0F900FBE0F901F9018959FB7F8946D
:10E1A000E1E7F0E08081807D808388B38F6288BB67
:10E1B00010929000E1E9F0E010821092920010922B
:10E1C0009500109294008081856080839FBF0895A0
:10E1D0002FB7F894909399008093980088B38F623A
:10E1E00088BBE1E7F0E08081826080832FBF0895E3
:10E1F000CF93DF93FC01DB0185E0EB0119928A9557
:10E20000E9F78581837011F082E08C9387818370B8
:10E2100021F082E012968C9312978581837081F0B1
:10E220008781837069F023893489818592852817D5
:10E23000390731F481E0848312961C92129701C051
:10E24000148285818370823021F0833021F080E058
:10E2500003C082E001C088E011968C9311978781FA
:10E260008370823021F0833021F080E003C082E0AF
:10E2700001C088E013968C93DF91CF910895CF93DE
:10E28000DF9300D000D01F92CDB7DEB7BE016F5F25
:10E290007F4F0E94F87089819A81890F8D5F9B81E1
:10E2A000890F9C81890F9D81890F0F900F900F908E
:10E2B0000F900F90DF91CF9108954F925F926F92E0
:10E2C0007F928F929F92AF92BF92CF92DF92EF9206
:10E2D000FF920F931F93CF93DF9300D000D000D015
:10E2E000CDB7DEB78C017B01BE016F5F7F4F4E83E0
:10E2F0000E94F870B981AA815B804C808B2F90E0DE
:10E3000003962A2F30E0820F931F850D911D642DF7
:10E3100070E0860F971F5D81850F911D4E8150E043
:10E32000481759070CF49AC0F801818180FB6624D4
:10E3300060F8712C43E0660C771C4A95E1F7828106
:10E3400080FB882480F8912C54E0880C991C5A9505
:10E35000E1F7862880818770882A838180FBAA2440
:10E36000A0F8B12C85E0AA0CBB1C8A95E1F78A289D
:10E37000848180FBCC24C0F8D12C96E0CC0CDD1C31
:10E380009A95E1F78C28F7018082F8014581437066
:10E39000F4E04F9FA0011124F80186818370F0E121
:10E3A0008F9FC0011124482BF8018781F0E48F9FD3
:10E3B000C0011124482BF7014183F8018085F70142
:10E3C0008283B23059F4F8018185F7018383F80123
:10E3D0008285F701848395E0C92E02C083E0C82EB0
:10E3E000B0E080E090E0200F311FDB2EDC0C0197C5
:10E3F000BA1761F0A901480F591FFA01B384A701A8
:10E400004D0D511DFA01B082BF5FEFCF9D2DF2E09F
:10E410005F120EC0D701AD0DB11DF80183898C9339
:10E4200081E08D0DD701A80FB11D9E5F84898C936B
:10E4300040E020E030E0060F171F842F890F2150A5
:10E440003109441561F0D801A20FB31F55965C91B4
:10E45000D701A80FB11D5C934F5FEFCF80E02696E8
:10E460000FB6F894DEBF0FBECDBFDF91CF911F91E5
:10E470000F91FF90EF90DF90CF90BF90AF909F9063
:10E480008F907F906F905F904F900895BF92CF9242
:10E49000DF92EF92FF920F931F93CF93DF937C0154
:10E4A000D62EEA0182E0861708F0B2C0F70180811B
:10E4B00086FBBB24B0F89181292F269526952370E1
:10E4C000C92EC294C694C69453E0C522382F377023
:10E4D000388383FB332730F9398384FB332730F9C2
:10E4E0003A8385FB882780F98B83BC822D83892F13
:10E4F000829583708E83CF8282818887222391F1D7
:10E500003381848190E0982F8827830F911D9A870B
:10E51000898787010B5F1F4F223079F461EF72E02A
:10E52000CE010B960E949D4AF70186818B878581DB
:10E530008C878701095F1F4F20C02330F1F4F7015A
:10E540003D9680E090E03E2F2F2F4291DE01A80FF4
:10E55000B91F1B964C93019688309105B1F7032F94
:10E56000122F0BC087010D5F1F4F61EF72E0CE01CC
:10E570000B960E949D4A1A861986CC20B9F1B110DB
:10E580000DC0F8012081818190E0982F8827820FAB
:10E59000911D9C8B8B8B0E5F1F4F04C089859A85C4
:10E5A0009C8B8B8BF2E0CF120EC061EF72E0CE013C
:10E5B00045960E949D4AF80181818D8B80818E8BCA
:10E5C0000E5F1F4F1BC0F3E0CF1218C0085F1F4F34
:10E5D000F80180E090E02291DE01A80FB91F559666
:10E5E0002C93019688309105B1F708C061EF72E075
:10E5F000CE0145960E949D4A1C8A1B8AC8018E192D
:10E600009F092D2D281B2FA71EA70DA7D81608F48C
:10E6100080E0DF91CF911F910F91FF90EF90DF90FD
:10E62000CF90BF900895FB0141505109460F571FED
:10E63000E417F50778F4208130E0322F222761813A
:10E64000260F311D820F931F8217930708F401963E
:10E650003296EECFE417F50751F4208130E0322FE7
:10E660002227820F931F8217930708F401960895BB
:10E67000CF93DF93C091AF2AD0E064972091AE2A68
:10E6800030E0322F2227C20FD31F48E050E068EB62
:10E690007AE29E01280F311DC9010E941373AE0159
:10E6A00060EC7AE20E941373009721F09827892783
:10E6B000982702C08FEF9FEFDF91CF91089590933D
:10E6C0008B1A80938A1A0895FC015381560F509338
:10E6D000AB2A872F99274281480F4093AA2AA1810C
:10E6E000A093A92AE081E093A82A242F30E02817DC
:10E6F000390748F481E08A0F8093A92A811103C069
:10E70000EF5FE093A82A852F90E077278617970779
:10E7100088F44F5F4093AA2A41110CC08091A92A26
:10E720008F5F8093A92A811105C08091A82A8F5FED
:10E730008093A82A0895AB01BC0180E090E00E947C
:10E740001373982789279827089544E150E06CEACD
:10E750007AE280E090E00E941373009721F09827FE
:10E760008927982708958FEF9FEF089586E00C94EE
:10E77000387381E10C94387380E0E82FF0E0EE0FFD
:10E78000FF1FED5CFF4C118210828F5F8430A8F375
:10E7900080E090E2899FF0011124ED54F04D118E3C
:10E7A0008F5F8430B0F380E094E09093851A80937B
:10E7B000841A80E09DE0989FF0011124E75BFF4CF4
:10E7C000158214828F5F8A30B0F38093831A089584
:10E7D000CF932091841A3091851A2F5F3F4F2115D6
:10E7E0004DE7340710F020E030E1522F432FE3EBE8
:10E7F000FFE2C0E0C43059F0A18DAA2329F0A48122
:10E80000B581A417B50749F3CF5FB096F3CF309326
:10E81000851A2093841A1092831A20E0E0E0F0E039
:10E820002430E8F430E2239FD0011124AD54B04DE0
:10E8300059963C915997311104C02093831AFD01D8
:10E8400010C0373041F4309739F05A964C915A97AE
:10E85000328D341708F0DF012F5FFD01E1CF2093E7
:10E86000831A3097A1F122E0218F2091861A248704
:10E870002091871A25872091881A26872091891A46
:10E88000278728ED34E0338B228B358B248B21E0D6
:10E8900030E0318B208B138E21E0228F23E0208FFC
:10E8A000168A20E1278B2091841A3091851A32270D
:10E8B000232732273583248377836683DC014D91B8
:10E8C0005D916D917C914083518362837383CF010D
:10E8D000CF910895CF93DF932091841A3091851AB8
:10E8E0002F5F3F4F21154DE7340710F020E030E156
:10E8F000522F432FEDE4F0E3C0E0CA3041F0A08195
:10E90000B181CF5F3D96A417B507B9F7E9CF309332
:10E91000851A2093841A40E05DE04A30A0F4A1E01B
:10E92000A40F549FF0011124E75BFF4C2481358133
:10E93000232B39F44093831A309741F480E090E020
:10E9400023C04A2FEACF4093831AF8CF2091841A2C
:10E950003091851A32272327322735832483778302
:10E960006683009729F4108211821282138209C0F3
:10E97000EC0188819981AA81BB8180839183A283E4
:10E98000B38380E48087CF01DF91CF91089540E089
:10E990004430A0F4E42FF0E051E0540FEE0FFF1FDD
:10E9A000ED5CFF4C208131812817390729F4409311
:10E9B000831A118210820895452FEACF4093831A5B
:10E9C000089540E0443098F4E42FF0E051E0540F13
:10E9D000EE0FFF1FED5CFF4C20813181232B29F4CA
:10E9E0004093831A918380830895452FEBCF409302
:10E9F000831A0895AF92BF92CF92DF92EF92FF9267
:10EA00000F931F93CF93DF93C091B12FD091B22F6B
:10EA1000843009F4DCC124ED3AE23093B02F209326
:10EA2000AF2F3093A72A2093A62A833059F4898DDB
:10EA30008F70833009F06BC088899989892B09F020
:10EA4000DFC67FC0823009F080C08091891A8F5F55
:10EA50008093891A811113C08091881A8F5F8093E7
:10EA6000881A81110CC08091871A8F5F8093871A52
:10EA7000811105C08091861A8F5F8093861A10924B
:10EA8000A52A1092A42A1092483010924730298D5E
:10EA9000822F8D7F853041F48A8D8F5F8A8F8431FC
:10EAA00009F0AEC6198EACC6222309F4A9C688891E
:10EAB0009989892B09F441C08A8D9FEF980F9A8F0D
:10EAC00081119EC68B8D883031F09FEF920F92306E
:10EAD00048F4853039F4198E80E88093AC2F0E9479
:10EAE000796F47C5853038F493E0082E01C0990F3F
:10EAF0000A94EAF701C090E39A8F8F5F8B8F822F81
:10EB00008F708330A1F048F4813009F44FC3823014
:10EB100009F076C61092CD2A4CC3863009F4C8C4D9
:10EB2000883009F4C5C4843009F06AC6C1C484E0E1
:10EB30008093AC2F0E94796F4EC52F70233009F05F
:10EB40005FC688E08093AC2F09C5853019F5E09148
:10EB5000AD2FF091AE2F84819581892B09F450C699
:10EB60001092B22F1092B12F88EC9AE29093B02FAE
:10EB70008093AF2F9093A72A8093A62A10924830B3
:10EB8000109247301092A52A1092A42A88E0809310
:10EB9000AC2F1BC18091AC2A853409F031C600919D
:10EBA000AE2A10E0102F00278091AF2A080F111D08
:10EBB0008091A42A9091A52A8017910708F420C675
:10EBC0001093A52A0093A42A8091B22A8F7309F08A
:10EBD00017C68091B32A811113C68091433090915A
:10EBE0004430C0914E03D0914F038C179D0759F4C8
:10EBF000409145305091463020915003309151035F
:10EC000042175307A1F02091BC2A3091BD2A281742
:10EC1000390709F0F5C52091BE2A3091BF2A8091AD
:10EC20004530909146302817390709F0E9C50E9410
:10EC3000A573019609F0E4C58091B52A863009F4E0
:10EC400029C18131E9F1813009F0DAC58091C02A0A
:10EC5000883009F0D5C51092C02A8091C22A9091BF
:10EC6000C32A873F3FEF930710F0099601C008962B
:10EC70009093C32A8093C22A8091B82A9091B92A8E
:10EC8000A091BA2AB091BB2A8093BC2A9093BD2A46
:10EC9000A093BE2AB093BF2A809143309091443014
:10ECA000A0914530B09146308093B82A9093B92A0C
:10ECB000A093BA2AB093BB2A80E48093B42A7DC57E
:10ECC0000C5111091093A52A0093A42A88EC9AE20A
:10ECD0009093B02F8093AF2F8091C62A9091C72A2E
:10ECE000892B29F00E94B973019609F089C52091FA
:10ECF000C22A3091C32A2115310509F481C589E45E
:10ED000090E39093AE2F8093AD2FA090C02AB09047
:10ED1000C12A409150035091510360915203709168
:10ED20005303A0915403B09155030091B82A109158
:10ED3000B92AE090BA2AF090BB2AE091AD2FF09169
:10ED4000AE2F80E3EB3CF80708F05AC5848195812B
:10ED5000009721F12817390709F5868197810097D7
:10ED600019F0A816B906D1F4808191818C179D07FE
:10ED700029F4C280D380C416D506B1F08617970750
:10ED800029F4C280D380CA16DB0671F00817190770
:10ED900029F482819381E816F90631F03D96F093CB
:10EDA000AE2FE093AD2FC9CF1092B22F1092B12F9A
:10EDB00082E08093AC2F88EC9AE29093A72A80930C
:10EDC000A62A10924830109247300E94796F8091A5
:10EDD000473090914830009709F412C59C01245E99
:10EDE0003F4F3093A52A2093A42A3093AE2A209334
:10EDF000AF2AE091AD2FF091AE2F20852093B42A59
:10EE000021E12093B52A089698278927982790937F
:10EE1000C52A8093C42A1092C72A1092C62A8481D8
:10EE200095819093C12A8093C02A8681978190937F
:10EE3000C32A8093C22A8091433090914430A0919C
:10EE40004530B09146308093B82A9093B92AA09368
:10EE5000BA2AB093BB2A80819181A281B381809329
:10EE6000BC2A9093BD2AA093BE2AB093BF2A84EDFA
:10EE70009AE29093B02F8093AF2F0E94B973809540
:10EE80009095009711F48FEF9FEF9093C72A80938E
:10EE9000C62A93C40E94B673019609F0B1C480914A
:10EEA000C22A9091C32A009709F4AAC42091C02ACB
:10EEB0003091C12A2115310509F4A2C44091B82A24
:10EEC0005091B92A6091BA2A7091BB2AECECFFE20A
:10EED000C3EBDFE2F080FF20A9F0AC81BD818A178F
:10EEE0009B0781F4AE81BF812A173B0759F4A881A3
:10EEF000B9814A175B0731F4AA81BB816A177B0786
:10EF000009F46FC1A096B096A0E3C333DA0711F7F6
:10EF10002091CD2A2F732230D9F49093811A8093B7
:10EF2000801A40E0443090F4E42FF0E0EE0FFF1F31
:10EF3000ED5CFF4C208131814F5F8217930791F781
:10EF40001092831A20E0C0E0D0E07EC04093831A84
:10EF50008091CD2A82FD54C484E18093CD2A88E239
:10EF600090E09093A52A8093A42A80E58093CC2AF0
:10EF70008091C72A9091CB2A9093C72A3091C62AB4
:10EF80009091CA2A9093C62A3093CA2A2091C52A02
:10EF90009091C92A9093C52A2093C92A9091C42A96
:10EFA0009093831A4091C82A4093C42A9093C82A08
:10EFB0008F5F8093CB2A81110FC081E0830F8093F4
:10EFC000CA2A811109C081E0820F8093C92A811168
:10EFD00003C09F5F9093C82A8091C02A9091C12A54
:10EFE0009093811A8093801A2091C22A3091C32A6B
:10EFF0003093C12A2093C02A9093C32A8093C22AB7
:10F000008091B82A9091B92AA091BA2AB091BB2ACE
:10F010008093BC2A9093BD2AA093BE2AB093BF2AA6
:10F020008091433090914430A0914530B09146306A
:10F030008093B82A9093B92AA093BA2AB093BB2A96
:10F04000A1C3373089F02F5F2430C0F430E2239F12
:10F05000C0011124FC01ED54F04D318D3111F1CF7F
:10F060002093831AEF010CC0209721F0428D3A8D36
:10F07000341748F7EC01CD54D04DE5CF2093831AD7
:10F08000209709F4BDC3D093B22FC093B12F83E072
:10F090008A8F888F1E8A84E08F8B1B8E8091C22A74
:10F0A0009091C32A9D838C838091C02A9091C12A1C
:10F0B0009F838E838091B82A9091B92AA091BA2A11
:10F0C000B091BB2A88839983AA83BB8381E0898F0F
:10F0D0008091861A8C878091871A8D878091881AF3
:10F0E0008E878091891A8F8781E090E0998B888B39
:10F0F0008091C72A8B878091C62A8A878091C52AEA
:10F1000089878091C42A888781E090E00E94647C8E
:10F110008091CC2A282F207F30E0213531050CF456
:10F1200045C082958F7090E00597880F991F880FD2
:10F13000991F3091821A20E0E22FF0E0E817F907DA
:10F140008CF5E455F54D30A5311105C02093831A97
:10F150001092821A2BC0313011F42F5FEDCF323074
:10F16000E1F441A54430C9F42093831A3093821A04
:10F1700082A590E0982F882723A5822B9093811A4F
:10F180008093801A893DA4E09A0710F088ED94E0FE
:10F190009B8B8A8B9D8B8C8B09C041A5442311F0DE
:10F1A000240FCACF2093831A3093821A80E1809370
:10F1B000CD2A8091CD2A82608093CD2A82E08093EF
:10F1C000D42A84E08093D52A8093D62A88ED809330
:10F1D000D72A8CE290E09093A52A8093A42A80E617
:10F1E0007EC2D093B22FC093B12F1092AC2F9091CA
:10F1F000CD2A92FF03C0198E80E21AC28091CC2AD8
:10F2000082958F70880F880F8093831A081B1109CD
:10F21000045111091093A52A0093A42A8F2D8F70F1
:10F22000823029F4892F8F73823139F41FC08130E5
:10F2300021F4892F8F738230C9F0012B19F4892FA3
:10F240008370A1F02091C42A888528133EC22091A2
:10F25000C52A8985281339C22091C62A8A85281390
:10F2600034C22091C72A8B8528132FC294FF4AC02D
:10F27000688979896115710509F444C0CE010C963D
:10F280000E9464733091C82A8091A82A38133AC02A
:10F290002091C92A8091A92A281334C09091CA2AA2
:10F2A0008091AA2A98132EC08091CB2A4091AB2A34
:10F2B000841328C03C872D879E878F878B8D811173
:10F2C0001AC02E89888D9A8D891B922F96959695B6
:10F2D0009695891B280F2E8B87FD81959F89392F45
:10F2E00036953695931B980F9F8B822F8695869522
:10F2F0008695890F888F81E08093AC2F888D8A8FC7
:10F30000198A188A498D842F8F7090E0FC013197FB
:10F31000E830F10508F074C2E057FF4F0C942F86D7
:10F320008091AC2F80FF14C083E0898F80E48093AC
:10F33000AC2F198A188A8091A42A9091A52A009747
:10F3400009F408C122E42093AC2F0E94647C02C11E
:10F350008091CD2A8F73823009F052C227CF8091DD
:10F36000AC2F80FF70C08091CD2A8F73823109F05D
:10F370006AC08091CC2A282F207F30E021353105CA
:10F380000CF445C082958F7090E00597880F991F07
:10F39000880F991F3091821A20E0E22FF0E0E817E1
:10F3A000F9078CF5E455F54D30A5311105C02093D2
:10F3B000831A1092821A2BC0313011F42F5FEDCFD7
:10F3C0003230E1F441A54430C9F42093831A3093DC
:10F3D000821A82A590E0982F882723A5822B9093EC
:10F3E000811A8093801A893D24E0920710F088EDFD
:10F3F00094E09B8B8A8B9D8B8C8B09C041A5442309
:10F4000011F0240FCACF2093831A3093821A83E01D
:10F41000898F8091C42A88878091C52A89878091A5
:10F42000C62A8A878091C72A8B8781E090E00E9454
:10F43000647C82E48093AC2F198A188A1092A52AE2
:10F440001092A42A87C080E28093AC2F0E94796F2B
:10F45000E091B12FF091B22F118E7ACD8091CD2A0B
:10F4600080FF28C044FD26C088899989892B09F02E
:10F47000C7C18091A42A9091A52A01960E94647C1C
:10F480002091AC2F822F80618093AC2F8091A42A91
:10F490009091A52A892B19F022612093AC2F0E940C
:10F4A000796F81E090E0998B888B88E0898F1B8E43
:10F4B00081E10CC185FF1CC08091D22A90E0982F79
:10F4C00088272091D32A822B2091AF2F3091B02F03
:10F4D000280F391F3093B02F2093AF2F2091A42AEB
:10F4E0003091A52A281B390B3093A52A2093A42AF2
:10F4F0008091A42A9091A52A009749F044FD07C065
:10F500002091AC2F22602093AC2F0E94647C8091CC
:10F51000CE2A90E0982F88272091CF2A820F911D24
:10F520009093811A8093801A2C893D892817390776
:10F5300010F0892B21F43093811A2093801A809146
:10F54000801A9091811A9B8B8A8B8091AC2F83704B
:10F5500009F456C110924830109247300E94796FDA
:10F560008091AC2F85FF07C0109248301092473031
:10F57000198E84E1ABC084FF0AC01092483010920B
:10F58000473081E090E0998B888B84E08FCF209189
:10F5900047303091483021153105E1F080FF02C03D
:10F5A000198A188A88899989009781F48A899B89A0
:10F5B0008217930720F490934830809347308091CE
:10F5C000473090914830998B888B04C09093483095
:10F5D000809347301B8E8091A62A9091A72A909302
:10F5E000B02F8093AF2F8091473090914830892B76
:10F5F00059F088899989009739F088969093A52ABF
:10F600008093A42A88E10BC08091AC2F81FFF8C0C1
:10F6100088E290E09093A52A8093A42A80E18093C9
:10F62000CD2A5CC08091AC2F80FFEAC0198E80E1AA
:10F630008093AC2F0E94796FE3C08091A42A9091AF
:10F64000A52A009711F00E94647C9091CD2A8091A8
:10F65000AC2F90FF0BC080FF06C087E0898F1A8E09
:10F66000198A188A19C086E0898F16C080FF1EC0CB
:10F6700085E0898F198A188AC3C08091A42A909145
:10F68000A52A009711F00E94647C8091CD2A80FF0A
:10F690000DC087E0898F1A8E81E090E00E94647C23
:10F6A00080E18093AC2F0E94796F0FC08091A42AD3
:10F6B0009091A52A892B49F4A3C08091AC2F80FF9B
:10F6C0009FC087E0898F1A8E9BC080E18093CD2AEE
:10F6D00088E290E09093A52A8093A42A80E5809305
:10F6E000CC2A88858093C82A89858093C92A8A85EF
:10F6F0008093CA2A8B858093CB2A8C858093C42AD9
:10F700008D858093C52A8E858093C62A8F858093A8
:10F71000C72A86E08093B52A8C819D819093C12A67
:10F720008093C02A8E819F819093C32A8093C22A9E
:10F730008091433090914430A0914530B091463053
:10F740008093B82A9093B92AA093BA2AB093BB2A7F
:10F7500088819981AA81BB818093BC2A9093BD2A1C
:10F76000A093BE2AB093BF2A898D84FF05C0109252
:10F77000CF2A1092CE2A06C084E08093CE2A88ED4C
:10F780008093CF2A80E48093B42A8091A42A909118
:10F79000A52A9093AE2A8093AF2A1092D32A109272
:10F7A000D22A1092D12A1092D02A0E94B673809544
:10F7B00090959093D12A8093D02A85E48093AC2AA7
:10F7C0001092AD2A1092B32A1092B22A80918A1A0E
:10F7D00090918B1A019690938B1A80938A1A90932A
:10F7E000B02A8093B12A1092B72A1092B62A0E94AA
:10F7F000A573809590959093B72A8093B62A04C0FC
:10F800001092A52A1092A42A1092AC2FDF91CF91CA
:10F810001F910F91FF90EF90DF90CF90BF90AF902E
:10F82000089598278927982708950E943586089576
:10F83000FC018091A62A9091A72A2CEA3FE2281B7E
:10F84000390BAB01261737070CF4A901141615065E
:10F8500054F45093483040934730E817F90719F0B3
:10F86000BF010C94648A089580E88093610010922F
:10F8700061000E94EA5A0E94594C0E94C65E809123
:10F88000532890915428009729F001979093542879
:10F8900080935328C0905528D0905628E090572840
:10F8A000F09058280E94845DC616D706E806F9062F
:10F8B00011F30E94845D60935528709356288093BD
:10F8C000572890935828D7CF2091B12F3091B22F3D
:10F8D000BC01C90108960E946473E091B12FF091B8
:10F8E000B22F8091A82A80878091A92A8187809150
:10F8F000AA2A82878091AB2A838708952F923F920C
:10F900004F925F926F927F928F929F92AF92BF922F
:10F91000CF92DF92EF92FF920F931F93CF93DF93DB
:10F92000CDB7DEB763970FB6F894DEBF0FBECDBF7D
:10F930007C011B016A01FC0117821682838181FF11
:10F9400066C3BE016F5F7F4F4B01F7019381F101E9
:10F9500093FD859193FF81911F01882309F453C37F
:10F96000853239F493FD859193FF81911F01853292
:10F9700039F4B70190E00E94CD8A56016501E5CFC8
:10F9800010E0512C20E02032A0F48B3269F030F4EA
:10F99000803259F0833269F420612CC08D3239F005
:10F9A000803339F4216026C02260246023C028609F
:10F9B00021C027FD27C030ED380F3A3078F426FFFC
:10F9C00006C0FAE01F9F300D1124132F13C06AE008
:10F9D000569E300D1124532E20620CC08E3221F41D
:10F9E00026FD11C3206406C08C3611F4206802C0C5
:10F9F000883641F4F10193FD859193FF81911F01B8
:10FA00008111C1CF9BEB980F933018F42061805E79
:10FA100006C09BE9980F933008F0AAC12F7E26FFFD
:10FA200016E02F73722E853621F4F22FF0647F2EAC
:10FA300008C0863621F4622F6068762E02C011114C
:10FA4000115077FE07C01C3348F444244394410E00
:10FA500027E00BC0183030F4212F06C027E04CE31C
:10FA6000442E03C027E017E0412C560174E0A70E96
:10FA7000B11CF6016081718182819381042DA40102
:10FA80000E946C896C01098100FF02C003FF06C05F
:10FA900071FC07C072FC08C0612C08C03DE2632EF7
:10FAA00005C02BE2622E02C090E2692E802F8C707E
:10FAB00099F1662011F084E001C083E0851510F013
:10FAC000512C0BC0581A73FC08C0B70180E290E0BB
:10FAD0000E94CD8A5A94C9F7F3CF662029F0B70166
:10FAE000862D90E00E94CD8A03FD03C00AE310E159
:10FAF00002C006E310E1F72DF0717F2EF80184912A
:10FB0000882309F476C271108052B70190E00E94F8
:10FB1000CD8A0F5F1F4FF2CF77FE0FC04C0C04FF52
:10FB200004C08A81813309F44A94141474F5F8E00E
:10FB3000F41578F588E0482E2CC076FC2AC0812F79
:10FB400090E08C159D059CF06CEFC6166FEFD60605
:10FB500074F0772D7068772E0AC0E2E0F0E0EC0FC9
:10FB6000FD1FE10FF11D8081803319F41150111137
:10FB7000F4CF77FE0EC044244394410E812F90E0D1
:10FB8000C816D9062CF41C1904C04424439401C09F
:10FB900010E077FE07C01C141D043CF496012F5F93
:10FBA0003F4F05C025E030E002C021E030E0662094
:10FBB00011F02F5F3F4F112331F0412F50E04F5F85
:10FBC0005F4F240F351F452D50E02417350714F4DF
:10FBD000521A01C0512C872D897049F4552039F0F3
:10FBE000B70180E290E00E94CD8A5A94F7CF662058
:10FBF00029F0B701862D90E00E94CD8A73FC09C0E0
:10FC0000552039F0B70180E390E00E94CD8A5A94E4
:10FC1000F7CF77FE5FC09C2D8D2DD7FE02C090E000
:10FC200080E0692E782E40E050E0C60184199109E9
:10FC30009D878C87960126193709280D391D812F3C
:10FC400090E0EE27FF27E81BF90BFF87EE87FFEF19
:10FC50006F167F0669F4B7018EE290E02B8B3A8B2A
:10FC6000488B598B0E94CD8A598948893A892B89BA
:10FC7000C614D70454F06C857D85661577052CF481
:10FC8000F901E40FF51F818101C080E371E0671A7B
:10FC900071084F5F5F4FEE85FF856E167F066CF033
:10FCA000B70190E02B8B3A8B488B598B0E94CD8A01
:10FCB0002B893A8948895989CACF6C147D0439F453
:10FCC0009A81963318F4953311F404FF81E3B70158
:10FCD00090E04BC08A81813309F00F7EB70190E03C
:10FCE0000E94CD8A111105C074FE18C085E490E011
:10FCF00017C0B7018EE290E00E94CD8A82E06624B0
:10FD00006394680EF401E80FF11D8081B70190E063
:10FD10000E94CD8A115041F3862DF1CF85E690E007
:10FD2000B7010E94CD8AD7FC05C0C114D10439F4B3
:10FD300004FF05C0D194C194D1088DE201C08BE2CB
:10FD4000B70190E00E94CD8A80E36AE0C616D10434
:10FD50002CF08F5FFAE0CF1AD108F7CFB70190E00F
:10FD60000E94CD8AB701C601C0960E94CD8A41C1CA
:10FD7000833631F0833779F0833509F058C021C0DC
:10FD8000560172E0A70EB11CF6018081898301E063
:10FD900010E0640114C05601F2E0AF0EB11CF60190
:10FDA000C080D18026FF03C0612F70E002C06FEFDA
:10FDB0007FEFC6012B8B0E94938A8C012B892F77B2
:10FDC00015C05601F2E0AF0EB11CF601C080D18023
:10FDD00026FF03C0612F70E002C06FEF7FEFC60106
:10FDE0002B8B0E94558A8C012B892068722E23FD53
:10FDF0001AC0852D90E008171907A8F4B70180E212
:10FE000090E00E94CD8A5A94F4CFF60177FC859158
:10FE100077FE81916F01B70190E00E94CD8A511069
:10FE20005A94015011090115110579F7E2C0843681
:10FE300011F0893651F5560127FF09C0F4E0AF0EE5
:10FE4000B11CF60160817181828193810AC0F2E068
:10FE5000AF0EB11CF60160817181882777FD809516
:10FE6000982F022F0F7697FF08C090958095709578
:10FE700061957F4F8F4F9F4F00682AE030E0A401CB
:10FE80000E94D88BC82EC8183EC0022F853721F497
:10FE90000F7E2AE030E01DC0097F8F3691F018F404
:10FEA000883559F0B0C0803719F0883711F0ABC0F1
:10FEB000006104FF09C0046007C024FF08C0066099
:10FEC00006C028E030E005C020E130E002C020E1BB
:10FED00032E0560107FF09C0F4E0AF0EB11CF60195
:10FEE000608171818281938108C0F2E0AF0EB11C04
:10FEF000F6016081718180E090E0A4010E94D88BBE
:10FF0000C82EC8180F7706FF0BC0202F2E7FC116F2
:10FF100050F404FF0AC002FD08C0202F2E7E05C049
:10FF2000DC2C202F03C0DC2C01C0D12E24FF0DC0FF
:10FF3000FE01EC0DF11D8081803311F4297E09C092
:10FF400022FF06C0D394D39404C0822F867809F090
:10FF5000D39423FD13C020FF06C01C2DD51418F424
:10FF6000150D1D19D52CD51468F4B70180E290E069
:10FF70002B8B0E94CD8AD3942B89F5CFD51410F406
:10FF80005D1801C0512C24FF12C0B70180E390E03E
:10FF90002B8B0E94CD8A2B8922FF17C021FF03C023
:10FFA00088E590E002C088E790E0B7010CC0822F9E
:10FFB000867859F021FD02C080E201C08BE227FD66
:10FFC0008DE2B70190E00E94CD8AC11638F4B701E6
:10FFD00080E390E00E94CD8A1150F7CFCA94F401DB
:10FFE000EC0DF11D8081B70190E00E94CD8AC11017
:10FFF000F5CF552009F4C2CCB70180E290E00E9411
:020000021000EC
:10000000CD8A5A94F6CFF7018681978102C08FEF8F
:100010009FEF63960FB6F894DEBF0FBECDBFDF91A2
:10002000CF911F910F91FF90EF90DF90CF90BF90F5
:10003000AF909F908F907F906F905F904F903F9088
:100040002F9008955058BB27AA270ED04EC23FD2FA
:1000500030F044D220F031F49F3F11F41EF4FFC180
:100060000EF4E095E7FBF5C1E92F50D280F3BA1703
:10007000620773078407950718F071F49EF568C24C
:100080000EF4E0950B2EBA2FA02D0B01B9019001B3
:100090000C01CA01A0011124FF27591B99F0593FF7
:1000A00050F4503E68F11A16F040A22F232F342F3F
:1000B0004427585FF3CF469537952795A795F0408D
:1000C0005395C9F77EF41F16BA0B620B730B840BA2
:1000D000BAF09150A1F0FF0FBB1F661F771F881F5A
:1000E000C2F70EC0BA0F621F731F841F48F48795B2
:1000F00077956795B795F7959E3F08F0B3CF9395A1
:10010000880F08F09927EE0F979587950895DFD10E
:1001100058F080E891E009F49EEFE0D128F040E843
:1001200051E059F45EEF09C09AC112C2E92FE0789C
:10013000EDD168F3092E052AC1F3261737074807C2
:10014000590738F00E2E07F8E02569F0E025E06445
:100150000AC0EF6307F8009407FADB01B9019D01BB
:10016000DC01CA01AD01EF9347D0BFD10AD05F9146
:10017000552331F02BED3FE049E450FD49EC63CFCE
:100180000895DF93DD27B92FBF7740E85FE31616A8
:10019000170648075B0710F4D92FE1D19F938F937F
:1001A0007F936F9346D3E0E3F1E06CD19ED12F9122
:1001B0003F914F915F919AD2DD2349F09058A2EA86
:1001C0002AED3FE049EC5FE3D0785D274DDFDF911A
:1001D0008CC11BD108F481E008950CD086C17ED17A
:1001E00040F075D130F021F45F3F19F032C1511168
:1001F000B0C135C18BD198F39923C9F35523B1F31D
:10020000951B550BBB27AA2762177307840738F085
:100210009F5F5F4F220F331F441FAA1FA9F333D0E4
:100220000E2E3AF0E0E830D091505040E695001C98
:10023000CAF729D0FE2F27D0660F771F881FBB1F54
:10024000261737074807AB07B0E809F0BB0B802D2E
:10025000BF01FF2793585F4F2AF09E3F510568F07A
:10026000F8C077C15F3FECF3983EDCF38695779555
:100270006795B795F7959F5FC9F7880F911D96957C
:10028000879597F90895E1E0660F771F881FBB1FD8
:10029000621773078407BA0720F0621B730B840B85
:1002A000BA0BEE1F88F7E095089519F40EF0D1C04F
:1002B0004FC1D5C033D1C8F39638C0F707F80F92B5
:1002C000E8942BE33AEA48EB5FE712D20F920F92E1
:1002D0000F924DB75EB70F92CAD1EDE5F1E0D2D0E3
:1002E0004F915F91EF91FF91E595EE1FFF1F49F050
:1002F000FE57E0684427EE0F441FFA95E1F7419559
:10030000550B36D10F9007FE2AC1089597FB0EF4C6
:10031000A9D03EC0E89409C097FB3EF49095809523
:10032000709561957F4F8F4F9F4F9923A9F0F92FBB
:1003300096E9BB279395F695879577956795B79539
:10034000F111F8CFFAF4BB0F11F460FF1BC06F5F1F
:100350007F4F8F4F9F4F16C0882311F096E911C031
:10036000772321F09EE8872F762F05C0662371F052
:1003700096E8862F70E060E02AF09A95660F771F66
:10038000881FDAF7880F9695879597F90895E8946E
:10039000F92F96EBFF2381F0121613061406440B77
:1003A0009395F69587957795679557954040FF23E8
:1003B000B9F71BC099270895882351F49850D2F7B4
:1003C000872B762F652F542F432F322F20E0B1F348
:1003D000121613061406440B88233AF09A95440F1C
:1003E000551F661F771F881FCAF755234AF4440F0D
:1003F000551F11F460FF04C06F5F7F4F8F4F9F4FF9
:10040000880F9695879597F90895990F0008550FCD
:10041000AA0BE0E8FEEF16161706E807F907C0F08A
:1004200012161306E407F50798F0621B730B840B92
:10043000950B39F40A2661F0232B242B252B21F46C
:1004400008950A2609F4A140A6958FEF811D811D0C
:10045000089597F99F6780E870E060E008959FEF46
:1004600080EC089590958095709560955095409595
:10047000309521953F4F4F4F5F4F6F4F7F4F8F4FBD
:100480009F4F0895DF93CF931F930F93FF92EF92A7
:10049000DF927B018C01689405C0DA2EEF0126D132
:1004A000FE01E894A5912591359145915591AEF3C2
:1004B000EF01DADDFE019701A801DA9479F7DF9008
:1004C000EF90FF900F911F91CF91DF91089500243D
:1004D0000A941616170618060906089500240A94A9
:1004E00012161306140605060895092E0394000C2F
:1004F00011F4882352F0BB0F40F4BF2B11F460FFBE
:1005000004C06F5F7F4F8F4F9F4F089557FD9058E6
:10051000440F551F59F05F3F71F04795880F97FBC7
:10052000991F61F09F3F79F0879508951216130681
:100530001406551FF2CF4695F1DF08C016161706B0
:100540001806991FF1CF86957105610508940895E5
:10055000E894BB2766277727CB0197F908959B017D
:10056000AC0160E070E080E89FE337CE72CF64C1F9
:10057000D5DFE8F39923D9F3940F511DBBF39150C4
:10058000504094F059F0882332F0660F771F881F8F
:1005900091505040C1F79E3F510544F7880F911D7F
:1005A0009695879597F908955F3FACF0983E9CF03B
:1005B000BB27869577956795B79508F4B1609395B5
:1005C000C1F7BB0F58F711F460FFE8CF6F5F7F4FA3
:1005D0008F4F9F4FE3CFBDCF0AD029ED3BE54EEDC6
:1005E0005EE378C00EF028C13ACF689432CF96DF30
:1005F000C8F39923D1F3C6F3DF93CF931F930F93DF
:10060000FF92C92FDD2788232AF02197660F771FD5
:10061000881FDAF720E030E040E85FEB9FE388399D
:1006200020F0803E30F021968F770DDDE5E8F1E097
:1006300003C009DDE2EBF1E025DF8B01BE01EC0137
:10064000FB2E6F5771097595771F880B990B64DE28
:1006500028E132E741E35FE349D0AF2D9801AE01D5
:10066000FF900F911F91CF91DF91FEDC3ECFFA01F9
:10067000DC01AA0FBB1F9B01AC01BF5728F4222746
:100680003327442750781FC0B75188F4AB2F00247C
:10069000469537952795011CA395D2F3002069F064
:1006A000220F331F441FB395DAF30DD0CBCC61304A
:1006B0007105A0E88A07B94630F49B01AC016627B2
:1006C000772788279078309621F0208331834283E2
:1006D000538308950BD009CFFADE28F0FFDE18F01F
:1006E000952309F0B6CEBBCE112433CF0FDFA0F394
:1006F000959FD1F3950F50E0551F629FF001729FB7
:10070000BB27F00DB11D639FAA27F00DB11DAA1FD5
:10071000649F6627B00DA11D661F829F2227B00D22
:10072000A11D621F739FB00DA11D621F839FA00DAD
:10073000611D221F749F3327A00D611D231F849FFD
:10074000600D211D822F762F6A2F11249F57504054
:100750008AF0E1F088234AF0EE0FFF1FBB1F661FEF
:10076000771F881F91505040A9F79E3F510570F0A8
:1007700070CEEFCE5F3FECF3983EDCF38695779535
:100780006795B795F795E7959F5FC1F7FE2B880FA3
:10079000911D9695879597F90895FA01EE0FFF1F21
:1007A00030962105310599F16115710561F48038A4
:1007B000BFE39B0749F168949038810561F0803868
:1007C000BFEF9B0741F0992342F5FF3FE10531055B
:1007D000210511F1E8940894E795D901AA2329F499
:1007E000AB2FBE2FF85FD0F310C0FF5F70F4A6955B
:1007F000E0F7F73950F019F0FF3A38F49F779F93FC
:100800000CD00F9007FC905808953EF028CE60E081
:1008100070E080E89FE308954FE79F775F934F93E1
:100820003F932F93E4DE2F913F914F915F9152DFE1
:1008300041CD9B01AC014ECF9F3F31F0915020F450
:10084000879577956795B795880F911D96958795AC
:1008500097F908950E943284332312F48A1B9B0B6C
:100860000C944384A29FB001B39FC001A39F700D5D
:10087000811D1124911DB29F700D811D1124911DA8
:1008800008950E943284B7FF0895821B930B089548
:100890000E943284A59F900DB49F900DA49F800D5F
:1008A000911D11240895B7FF0C9448840E94488438
:1008B000821B930B0895DB018F939F930E944884C2
:1008C000BF91AF91A29F800D911DA39F900DB29FEC
:1008D000900D11240895AA1BBB1B51E107C0AA1F4C
:1008E000BB1FA617B70710F0A61BB70B881F991FD1
:1008F0005A95A9F780959095BC01CD01089597FB75
:10090000072E16F4009407D077FD09D00E946B845F
:1009100007FC05D03EF4909581959F4F0895709502
:1009200061957F4F0895A1E21A2EAA1BBB1BFD0102
:100930000DC0AA1FBB1FEE1FFF1FA217B307E407BE
:10094000F50720F0A21BB30BE40BF50B661F771F16
:10095000881F991F1A9469F76095709580959095F6
:100960009B01AC01BD01CF010895052E97FB1EF43C
:1009700000940E94E08557FD07D00E94938407FCF5
:1009800003D04EF40C94E085509540953095219518
:100990003F4F4F4F5F4F0895689401C0E894F92F7F
:1009A000F12B12F00C940085A0E0B0E0EAEDF4E841
:1009B0000C94FE85092E059422F40E94E8851123EB
:1009C00092F4F0E80F26FFEFE094F0940095109574
:1009D000B094C094D094A194BF0ACF0ADF0AEF0A62
:1009E000FF0A0F0B1F0B0E948F8507FC0E94E885F2
:1009F000CDB7DEB7ECE00C941A86689401C0E89499
:100A00008F929F92CF93DF930E948F85DF91CF913A
:100A10009F908F900895DF93CF931F930F939A9D8C
:100A2000F02D219FF00D8B9DF00D8A9DE02DF10D95
:100A3000039FF00D029FE00DF11D4E9DE00DF11D95
:100A40005E9DF00D4F9DF00D7F936F93BF92AF921F
:100A50005F934F93D5010E9432848B01AC01D70183
:100A60000E943284EB01E80FF91FD6010E945B85DA
:100A70002F913F91D6010E943284C60FD71FE81FE5
:100A8000F91FAF91BF910E945B852F913F910E940A
:100A90003284C60FD71FE81FF91FD6010E94328487
:100AA000E60FF71F9801BE01CF0111240F911F918E
:100AB000CF91DF9108950E943284460F571FC81FBF
:100AC000D91F08F431960895E894DF93CF93FC0181
:100AD000DB010E9432847F936F93E9019A01AC019C
:100AE000BF93AF933F932F93DF010E94328426F48C
:100AF0006C1B7D0B820B930B9E01EB01FC010E9492
:100B00005B85AF91BF912F913F910E945B85BE01A4
:100B1000CF01F9012F913F91CF91DF910895882462
:100B20009924F401E401B0E49F93AA279A158B0459
:100B30009C04ED05FE05CF05D007A10798F4AD2F65
:100B4000DC2FCF2FFE2FE92D982C892E982F872F61
:100B5000762F652F542F432F322F2227B85031F78D
:100B6000BF9127C01B2EBF91BB27220F331F441FED
:100B7000551F661F771F881F991F881C991CEE1F21
:100B8000FF1FCC1FDD1FAA1FBB1F8A149B04EC058F
:100B9000FD05CE05DF05A007B10748F08A189B08C0
:100BA000EC09FD09CE09DF09A00BB10B21601A94F5
:100BB000E1F62EF49401AF01BE01CD01000C0895C1
:100BC00090958095709561957F4F8F4F9F4F0895B9
:100BD00060957095809590953095409550952195AC
:100BE0003F4F4F4F5F4F6F4F7F4F8F4F9F4F089536
:100BF0002F923F924F925F926F927F928F929F922D
:100C0000AF92BF92CF92DF92EF92FF920F931F931A
:100C1000CF93DF93CDB7DEB7CA1BDB0B0FB6F894CB
:100C2000DEBF0FBECDBF09942A88398848885F840B
:100C30006E847D848C849B84AA84B984C884DF807C
:100C4000EE80FD800C811B81AA81B981CE0FD11D60
:100C50000FB6F894DEBF0FBECDBFED010895EE0FC5
:100C6000FF1F0590F491E02D0994692796276927C5
:100C700078278727782708950F93083090F0982FCA
:100C8000872F762F652F542F432F322F222708507E
:100C9000F4CF220F331F441F551F661F771F881F75
:100CA000991F0A95B2F70F91089597FB10F81694C3
:100CB00000080F93083098F00850232F342F452F49
:100CC000562F672F782F892F902DF4CF0594979565
:100CD00087957795679557954795379527950A9501
:100CE000AAF70F9108952A0D3B1D4C1D5D1D6E1D29
:100CF0007F1D801F911F08950024A7FD00942A0FD7
:100D0000301D401D501D601D701D801D901D0895DB
:100D10002A193B094C095D096E097F09800B910B6B
:100D200008952A153B054C055D056E057F05800776
:100D3000910708950024A7FD00942A173005400567
:100D40005005600570058005900508958F929F926B
:100D5000AF92BF92CF92DF92EF92FF92CF93DF9349
:100D6000EC01688179818A819B816115710581051A
:100D7000910521F464E279ED8BE597E02DE133EF05
:100D800041E050E00E94B58449015A019B01AC0149
:100D9000A7EAB1E40E9448846B017C01ACEEB4EF99
:100DA000A50194010E945684C60ED71EE81EF91EA6
:100DB000F7FE06C081E0C81AD108E10880E8F80A09
:100DC000C882D982EA82FB82C6019F77DF91CF91E8
:100DD000FF90EF90DF90CF90BF90AF909F908F905B
:100DE00008950C94A6868BED92E00C94A686A0E064
:100DF000B0E08093DB029093DC02A093DD02B0931D
:100E0000DE0208952F923F925F926F927F928F92AF
:100E10009F92AF92BF92CF92DF92EF92FF920F9389
:100E20001F93CF93DF938B01EA016115710521F0C8
:100E3000DB018C9311969C93209739F09E012250F0
:100E400031092332310508F0FBC07C016701BFEF97
:100E5000CB1ADB0A5601F7016080862D90E00E94D4
:100E6000448A892B11F07601F1CFFDE26F120AC09E
:100E7000570182E0A80EB11CD70111966C9077241F
:100E800073940BC0BBE26B1207C05701E2E0AE0ED9
:100E9000B11CD70111966C90712CCE018F7E892BDD
:100EA00089F4B0E36B1222C0F50180818F7D883513
:100EB00041F56180F2E0AF0EB11C872D8260782E83
:100EC000C0E1D0E0C830D105F1F04CF4C230D1051A
:100ED00011F5C12CD12CE12CB0E4FB2E2FC0CA306F
:100EE000D10531F0C031D10521F115C0209751F75E
:100EF000CAE0D0E0ACECCA2EDC2CEC2CACE0FA2E34
:100F00001DC02097F9F6C8E0D0E0C12CD12CE12C0F
:100F1000F0E1FF2E13C060E070E080E090E89E01F9
:100F2000442737FD4095542F0E94938469017A012C
:100F300005C0C12CD12CE12CE8E0FE2EF50160E0CB
:100F400020E030E0A9014E01AA2497FCA094BA2C1D
:100F50001F0170ED572E560CA9E0A51570F48FEB0C
:100F6000860D8A3118F499EC592E06C08FE9860D4A
:100F70008A3130F589EA582E560C852D90E08C1771
:100F80009D07F4F467FD18C0C216D306E406F50603
:100F900080F0C501B4010E945B849B01AC01250D6A
:100FA000311D411D511D213031054105B0E85B0760
:100FB00010F06FEF01C061E03196D1016C90C8CFA5
:100FC000872D81700115110571F0662329F0319785
:100FD000D801ED93FC9307C071FE19C03297D80178
:100FE000ED93FC9314C067FF12C0882329F020E022
:100FF00030E040E050E804C02FEF3FEF4FEF5FE7F5
:1010000082E290E09093D2308093D13016C0882352
:1010100041F050954095309521953F4F4F4F5F4F90
:101020000CC057FF0AC082E290E09093D2308093C8
:10103000D1302FEF3FEF4FEF5FE7B901CA0104C096
:1010400060E070E080E090E0DF91CF911F910F9120
:10105000FF90EF90DF90CF90BF90AF909F908F90D8
:101060007F906F905F903F902F9008952F923F92C6
:101070005F926F927F928F929F92AF92BF92CF9228
:10108000DF92EF92FF920F931F93CF93DF938B0129
:10109000EA016115710521F0DB018C9311969C9397
:1010A000209739F09E01225031092332310508F092
:1010B000D8C07C016701BFEFCB1ADB0A5601F701EC
:1010C0006080862D90E00E94448A892B11F0760181
:1010D000F1CFFDE26F120AC0570182E0A80EB11CE9
:1010E000D70111966C90772473940BC0BBE26B12FE
:1010F00007C05701E2E0AE0EB11CD70111966C900B
:10110000712CCE018F7E892B89F4B0E36B1237C02E
:10111000F50180818F7D8835D1F46180F2E0AF0EDA
:10112000B11C872D8260782EC0E1D0E0CA30D10595
:1011300051F1C031D10521F0C830D10599F409C071
:10114000CC24CA94DC2CEC2CAFE0FA2E22C02097E1
:1011500069F7C8E0D0E0CC24CA94DC2CEC2CFFE189
:10116000FF2E17C06FEF7FEFCB019E01442737FDA5
:101170004095542F0E94938469017A010AC02097F8
:10118000A9F6CAE0D0E0E9E9CE2EDC2CEC2CE9E1AE
:10119000FE2EF50160E020E030E0A9014E01AA2416
:1011A00097FCA094BA2C1F0170ED572E560CA9E0A5
:1011B000A51570F48FEB860D8A3118F499EC592E31
:1011C00006C08FE9860D8A3148F589EA582E560CFB
:1011D000852D90E08C179D070CF56F3FD9F0C21656
:1011E000D306E406F50698F0C501B4010E945B84BD
:1011F0009B01AC01852D90E0A0E0B0E0280F391FE5
:101200004A1F5B1F281739074A075B0710F46FEF67
:1012100001C061E03196D1016C90C5CF0115110577
:1012200051F0662311F0319703C071FE04C032976C
:10123000D801ED93FC9370FE07C050954095309512
:1012400021953F4F4F4F5F4F67FF10C082E290E004
:101250009093D2308093D1306FEF7FEF8FEF9FEF7D
:1012600007C060E070E080E090E002C0B901CA0110
:10127000DF91CF911F910F91FF90EF90DF90CF9072
:10128000BF90AF909F908F907F906F905F903F90B6
:101290002F900895662777270C94718CFC0188277E
:1012A0009927E89421912032E9F3293010F02E306B
:1012B000C8F32B3241F02D3239F4689404C00E94F7
:1012C000C58A820F911D219120532A30C0F31EF44C
:1012D000909581959F4F0895283008F027E0332797
:1012E000DA01990F311D87FD916000966105710546
:1012F00039F432602E5F3D9330E32A95E1F708958B
:101300009F3F30F080387105610509F03C5F3C5F1C
:101310003D93913008F08068911DDF93CF931F9328
:101320000F93FF92EF92192F987F9695E92F96953C
:101330009695E90FFF27E856FF4E99273327EE24AD
:10134000FF24A701E70105900894079428F4360FBD
:10135000E71EF81E491F511D660F771F881F991F32
:101360000694A1F70590079428F4E70EF81E491F8C
:10137000561FC11D770F881F991F661F0694A1F77E
:101380000590079428F4F80E491F561FC71FD11D5A
:10139000880F991F661F771F0694A1F70590079481
:1013A00020F4490F561FC71FD81F990F661F771FBC
:1013B000881F0694A9F784911095177041F0D6956F
:1013C000C79557954795F794E7941A95C1F7EEE3BB
:1013D000F0E168941590159135916591959105907E
:1013E0007FE27395E118F10A430B560BC90BD00944
:1013F000C0F7E10CF11E431F561FC91FD01D7EF41C
:10140000703311F48A95E6CFE894015030F0080F5C
:101410000AF40027021708F4202F2395022F7A33AD
:1014200028F079E37D932A95E9F710C07D932A95FA
:1014300089F6069497956795379517951794E1184F
:10144000F10A430B560BC90BD00998F023957E91F6
:1014500073957A3308F070E37C932013B8F77E918C
:1014600070617D9330F0839571E37D9370E32A95ED
:10147000E1F71124EF90FF900F911F91CF91DF9131
:10148000992787FD909508959111A8C3803219F08E
:1014900089508550D0F70895FB01DC018D910590AE
:1014A00080190110D9F3990B0895FC010590615042
:1014B00070400110D8F7809590958E0F9F1F08956A
:1014C0004CE85AE10C949E8AFB01DC0102C00190B9
:1014D0000D9241505040D8F70895DC0101C06D9342
:1014E00041505040E0F70895FB01DC018D910190DF
:1014F00080190110D9F3990B0895FB01DC010190CB
:101500000D920020E1F70895FB01DC0141505040AD
:1015100048F001900D920020C9F701C01D92415082
:101520005040E0F70895FC016150704001900110B7
:10153000D8F7809590958E0F9F1F0895FA01A1917D
:10154000B081009719F41097E1F0CD01DC01CD01D5
:101550000D90002011F4C00113C0FB012191222342
:1015600019F02015D9F7F3CFFB012191201519F4BB
:101570001E92119606C02223C1F70D900020A1F7FC
:10158000D001FA01A193B08308957AE0979F902D3E
:10159000879F802D910D112408950F931F93CF9352
:1015A000DF93182F092FEB018B8181FD03C08FEF93
:1015B0009FEF20C082FF10C04E815F812C813D8152
:1015C000421753077CF4E881F9819F012F5F3F4F59
:1015D00039832883108306C0E885F985812F099512
:1015E000892B29F72E813F812F5F3F4F3F832E8329
:1015F000812F902FDF91CF911F910F910895CF935D
:10160000DF93CDB7DEB7FE01359661917191AF01E1
:101610008091CD309091CE300E947E7CDF91CF9131
:1016200008950F931F93CF93DF93CDB7DEB7FE01DD
:101630003796619171910DEC10E3D8018D919C91D9
:10164000DC0113962C911397286013962C93AF010D
:101650000E947E7CD801ED91FC912381277F23831A
:10166000DF91CF911F910F9108950F931F93CF9307
:10167000DF93E091CD30F091CE30238121FF1BC06C
:10168000EC0100E010E089916091CD307091CE3096
:10169000DB011896ED91FC911997882331F009959B
:1016A000892B89F30FEF1FEFEECF8AE00995892B85
:1016B00011F4C80102C08FEF9FEFDF91CF911F910E
:1016C0000F9108950F931F93CF93DF93CDB7DEB79C
:1016D0002E970FB6F894DEBF0FBECDBF0D891E89C1
:1016E0008F89988D26E02C831A83098397FF02C087
:1016F00080E090E801979E838D83AE01455E5F4F49
:10170000698D7A8DCE0101960E947E7C4D815E812D
:1017100057FD0AC02F813885421753070CF49A01F0
:10172000F801E20FF31F10822E960FB6F894DEBF79
:101730000FBECDBFDF91CF911F910F9108950F93F1
:101740001F93CF93DF93CDB7DEB72E970FB6F894E4
:10175000DEBF0FBECDBF8C01CA0146E04C831A83A9
:10176000098377FF02C060E070E8615071097E83F1
:101770006D83A901BC01CE0101960E947E7C4D8142
:101780005E8157FD0AC02F813885421753070CF43C
:101790009A01F801E20FF31F10822E960FB6F8940B
:1017A000DEBF0FBECDBFDF91CF911F910F91089586
:1017B000FA01AA27283051F1203181F1E8946F9382
:1017C0006E7F6E5F7F4F8F4F9F4FAF4FB1E03ED028
:1017D000B4E03CD0670F781F891F9A1FA11D680FC6
:1017E000791F8A1F911DA11D6A0F711D811D911DF9
:1017F000A11D20D009F468943F912AE0269F11246E
:101800003019305D3193DEF6CF010895462F4770D1
:10181000405D4193B3E00FD0C9F7F6CF462F4F702C
:10182000405D4A3318F0495D31FD4052419302D08A
:10183000A9F7EACFB4E0A695979587957795679530
:10184000BA95C9F700976105710508959B01AC0130
:101850000A2E06945795479537952795BA95C9F757
:10186000620F731F841F951FA01D0895DC01CB011B
:10187000FC01F999FECF06C0F2BDE1BDF89A3196A0
:1018800000B40D9241505040B8F70895F999FECF39
:1018900092BD81BDF89A992780B50895A8E1B0E07E
:1018A00042E050E00C94388CDC01CB0103C02D9158
:1018B0000E945F8C41505040D0F70895262FF9992F
:1018C000FECF1FBA92BD81BD20BD0FB6F894FA9A23
:1018D000F99A0FBE019608950E945E8C272F0C94F2
:1018E0005F8C4F925F926F927F928F929F92AF9296
:1018F000BF92CF92DF92EF92FF920F931F93CF93FD
:10190000DF938B016115710521F0DB018C9311963A
:101910009C93EC015E01BFEFAB1ABB0A7501C88056
:101920008C2D90E00E94448A892B11F0E501F2CFC2
:10193000EDE2CE1208C07E01F2E0EF0EF11CC9808C
:10194000DD24D39409C02BE2C21205C07E0142E01F
:10195000E40EF11CC980D12CE701219743E050E04F
:1019600060E471E1CE010E94F18D892BD1F4E70191
:10197000229645E050E06BE371E1CE010E94F18DCB
:10198000892B11F4E70127960115110519F0D801EB
:10199000CD93DC93D11008C160E070E080E89FE750
:1019A0000CC143E050E068E371E1CE010E94F18D8B
:1019B000892B59F40115110509F4FBC0B2E0EB0EB7
:1019C000F11CF801F182E082F4C0F70160E070E000
:1019D000CB01C0E0D0E07F01A0EDAA2EAC0C29E045
:1019E0002A1530F14D2D4260B42E2D2D2870D2FED7
:1019F00004C0211125C0219623C021112197A5E003
:101A0000B0E09B01AC010E944884660F771F881FDD
:101A1000991F6A0D711D811D911D6839A9E97A0709
:101A20008A07A9E19A0760F0BD2DB660BB2E08C0F9
:101A30002EEFA2120AC0D3FC50C04D2D4860B42E28
:101A40003196D701CC90DB2CC6CF2C2D2F7D2534A1
:101A500009F043C0A081AD3241F4BD2DB061DB2E51
:101A60007F0122E0E20EF11C0CC07F01AB3231F0AD
:101A70004FEFE41AF40A21E030E006C0A2E0EA0EDB
:101A8000F11CA18122E030E0A053AA3018F0E21A44
:101A9000F30A23C0F70120E030E02038BCE03B0728
:101AA0005CF4A901440F551F440F551F240F351F27
:101AB000220F331F2A0F311DAF014F5F5F4F7A0195
:101AC000A081A053AA3010F4FA01E7CFD4FE03C0DE
:101AD000319521953109C20FD31FD1FE09C00115DF
:101AE000110531F0E1E0EE1AF108D801ED92FC9217
:101AF0000E948A812D2D2370233019F06B017C0107
:101B000006C06B017C01F7FAF094F7F8F09420E03E
:101B100030E0A901C701B6010E94E980882309F4D9
:101B200040C0D7FF06C0D195C195D10907E511E1A5
:101B300002C00FE611E14801B8E18B1A910890E26A
:101B4000A92EB12CF8014590559065907490CA1556
:101B5000DB055CF0A3019201C701B6010E946A8314
:101B60006B017C01CA19DB09F2CF04501109B5944D
:101B7000A7940815190531F78E2D880F8F2D881F12
:101B80008F3F49F020E030E0A901C701B6010E9473
:101B9000E980811106C082E290E09093D230809378
:101BA000D130C701B60109C060E070E080E89FEF66
:101BB00004C060E070E080EC9FE7DF91CF911F915F
:101BC0000F91FF90EF90DF90CF90BF90AF909F90DC
:101BD0008F907F906F905F904F90089599278827FE
:101BE0000895FB01DC014150504088F08D91813413
:101BF0001CF08B350CF4805E659161341CF06B3504
:101C00000CF4605E861B611171F3990B0895881BBB
